Component: Arm Compiler for Embedded 6.19 Tool: armlink [5e73cb00]

==============================================================================

Section Cross References

    main.o(.text.periph_init) refers to sysclk.o(.text.sysclk_init) for sysclk_init
    main.o(.text.periph_init) refers to uart.o(.text.uart_init_first) for uart_init_first
    main.o(.text.periph_init) refers to tmr.o(.text.tmr_init_first) for tmr_init_first
    main.o(.text.periph_init) refers to gpio.o(.text.gpio_init) for gpio_init
    main.o(.text.periph_init) refers to uart.o(.bss.huart1) for huart1
    main.o(.text.periph_init) refers to main.o(.text.restart_receive) for restart_receive
    main.o(.text.periph_init) refers to uart.o(.text.uart_set_callback) for uart_set_callback
    main.o(.text.periph_init) refers to uart.o(.text.uart_start) for uart_start
    main.o(.text.periph_init) refers to tmr.o(.bss.htmr2) for htmr2
    main.o(.text.periph_init) refers to main.o(.text.heartbit) for heartbit
    main.o(.text.periph_init) refers to tmr.o(.text.tmr_set_callback) for tmr_set_callback
    main.o(.text.periph_init) refers to tmr.o(.bss.htmr0) for htmr0
    main.o(.text.periph_init) refers to tmr.o(.text.tmr_start) for tmr_start
    main.o(.text.periph_init) refers to tmr.o(.bss.htmr1) for htmr1
    main.o(.ARM.exidx.text.periph_init) refers to main.o(.text.periph_init) for [Anonymous Symbol]
    main.o(.text.restart_receive) refers to uart.o(.bss.huart1) for huart1
    main.o(.text.restart_receive) refers to main.o(.bss.rxbuff) for rxbuff
    main.o(.text.restart_receive) refers to uart.o(.text.uart_receive_it) for uart_receive_it
    main.o(.text.restart_receive) refers to uart.o(.text.uart_transmit_it) for uart_transmit_it
    main.o(.ARM.exidx.text.restart_receive) refers to main.o(.text.restart_receive) for [Anonymous Symbol]
    main.o(.text.heartbit) refers to uart.o(.bss.huart1) for huart1
    main.o(.text.heartbit) refers to main.o(.rodata.str1.1) for .L.str
    main.o(.text.heartbit) refers to uart.o(.text.uart_transmit) for uart_transmit
    main.o(.ARM.exidx.text.heartbit) refers to main.o(.text.heartbit) for [Anonymous Symbol]
    main.o(.text.main) refers to main.o(.text.periph_init) for periph_init
    main.o(.text.main) refers to uart.o(.bss.huart1) for huart1
    main.o(.text.main) refers to main.o(.bss.rxbuff) for rxbuff
    main.o(.text.main) refers to uart.o(.text.uart_receive_it) for uart_receive_it
    main.o(.text.main) refers to tmr.o(.bss.htmr0) for htmr0
    main.o(.text.main) refers to tmr.o(.text.tmr_delay_start) for tmr_delay_start
    main.o(.text.main) refers to tmr.o(.text.tmr_delay_done) for tmr_delay_done
    main.o(.text.main) refers to main.o(.text.GPIO_ToggleBits) for GPIO_ToggleBits
    main.o(.text.main) refers to tmr.o(.text.tmr_delay) for tmr_delay
    main.o(.ARM.exidx.text.main) refers to main.o(.text.main) for [Anonymous Symbol]
    main.o(.ARM.exidx.text.GPIO_ToggleBits) refers to main.o(.text.GPIO_ToggleBits) for [Anonymous Symbol]
    main.o(.ARM.exidx.text.Error_Handler) refers to main.o(.text.Error_Handler) for [Anonymous Symbol]
    gpio.o(.text.gpio_init) refers to gpio.o(.text.RCU_AHBClkCmd) for RCU_AHBClkCmd
    gpio.o(.text.gpio_init) refers to gpio.o(.text.RCU_AHBRstCmd) for RCU_AHBRstCmd
    gpio.o(.text.gpio_init) refers to plib035_gpio.o(.text.GPIO_DeInit) for GPIO_DeInit
    gpio.o(.text.gpio_init) refers to gpio.o(.data.gpioa_config) for gpioa_config
    gpio.o(.text.gpio_init) refers to plib035_gpio.o(.text.GPIO_Init) for GPIO_Init
    gpio.o(.text.gpio_init) refers to gpio.o(.data.gpiob_config) for gpiob_config
    gpio.o(.ARM.exidx.text.gpio_init) refers to gpio.o(.text.gpio_init) for [Anonymous Symbol]
    gpio.o(.ARM.exidx.text.RCU_AHBClkCmd) refers to gpio.o(.text.RCU_AHBClkCmd) for [Anonymous Symbol]
    gpio.o(.ARM.exidx.text.RCU_AHBRstCmd) refers to gpio.o(.text.RCU_AHBRstCmd) for [Anonymous Symbol]
    gpio.o(.text.gpio_get_init) refers to gpio.o(.data.gpioa_config) for gpioa_config
    gpio.o(.text.gpio_get_init) refers to gpio.o(.data.gpiob_config) for gpiob_config
    gpio.o(.ARM.exidx.text.gpio_get_init) refers to gpio.o(.text.gpio_get_init) for [Anonymous Symbol]
    tmr.o(.text.tmr_init_first) refers to tmr.o(.text.RCU_APBClkCmd) for RCU_APBClkCmd
    tmr.o(.text.tmr_init_first) refers to tmr.o(.text.RCU_APBRstCmd) for RCU_APBRstCmd
    tmr.o(.text.tmr_init_first) refers to tmr.o(.bss.htmr0) for htmr0
    tmr.o(.text.tmr_init_first) refers to tmr.o(.data.tmr0_config) for tmr0_config
    tmr.o(.text.tmr_init_first) refers to tmr.o(.text.tmr_init) for tmr_init
    tmr.o(.text.tmr_init_first) refers to tmr.o(.text.__NVIC_EnableIRQ) for __NVIC_EnableIRQ
    tmr.o(.text.tmr_init_first) refers to tmr.o(.bss.htmr1) for htmr1
    tmr.o(.text.tmr_init_first) refers to tmr.o(.data.tmr1_config) for tmr1_config
    tmr.o(.text.tmr_init_first) refers to tmr.o(.bss.htmr2) for htmr2
    tmr.o(.text.tmr_init_first) refers to tmr.o(.data.tmr2_config) for tmr2_config
    tmr.o(.ARM.exidx.text.tmr_init_first) refers to tmr.o(.text.tmr_init_first) for [Anonymous Symbol]
    tmr.o(.ARM.exidx.text.RCU_APBClkCmd) refers to tmr.o(.text.RCU_APBClkCmd) for [Anonymous Symbol]
    tmr.o(.ARM.exidx.text.RCU_APBRstCmd) refers to tmr.o(.text.RCU_APBRstCmd) for [Anonymous Symbol]
    tmr.o(.text.tmr_init) refers to tmr.o(.text.TMR_Init) for TMR_Init
    tmr.o(.ARM.exidx.text.tmr_init) refers to tmr.o(.text.tmr_init) for [Anonymous Symbol]
    tmr.o(.ARM.exidx.text.__NVIC_EnableIRQ) refers to tmr.o(.text.__NVIC_EnableIRQ) for [Anonymous Symbol]
    tmr.o(.text.TMR_Init) refers to plib035_tmr.o(.text.TMR_PeriodConfig) for TMR_PeriodConfig
    tmr.o(.text.TMR_Init) refers to plib035_tmr.o(.text.TMR_FreqConfig) for TMR_FreqConfig
    tmr.o(.text.TMR_Init) refers to tmr.o(.text.TMR_SetLoad) for TMR_SetLoad
    tmr.o(.text.TMR_Init) refers to tmr.o(.text.TMR_ITCmd) for TMR_ITCmd
    tmr.o(.text.TMR_Init) refers to tmr.o(.text.TMR_DMAReqCmd) for TMR_DMAReqCmd
    tmr.o(.text.TMR_Init) refers to tmr.o(.text.TMR_ADCSOCCmd) for TMR_ADCSOCCmd
    tmr.o(.text.TMR_Init) refers to tmr.o(.text.TMR_ExtInputConfig) for TMR_ExtInputConfig
    tmr.o(.ARM.exidx.text.TMR_Init) refers to tmr.o(.text.TMR_Init) for [Anonymous Symbol]
    tmr.o(.ARM.exidx.text.tmr_set_callback) refers to tmr.o(.text.tmr_set_callback) for [Anonymous Symbol]
    tmr.o(.text.tmr_start) refers to tmr.o(.text.TMR_Cmd) for TMR_Cmd
    tmr.o(.ARM.exidx.text.tmr_start) refers to tmr.o(.text.tmr_start) for [Anonymous Symbol]
    tmr.o(.ARM.exidx.text.TMR_Cmd) refers to tmr.o(.text.TMR_Cmd) for [Anonymous Symbol]
    tmr.o(.text.tmr_stop) refers to tmr.o(.text.TMR_Cmd) for TMR_Cmd
    tmr.o(.ARM.exidx.text.tmr_stop) refers to tmr.o(.text.tmr_stop) for [Anonymous Symbol]
    tmr.o(.ARM.exidx.text.tmr_delay) refers to tmr.o(.text.tmr_delay) for [Anonymous Symbol]
    tmr.o(.ARM.exidx.text.tmr_delay_start) refers to tmr.o(.text.tmr_delay_start) for [Anonymous Symbol]
    tmr.o(.ARM.exidx.text.tmr_delay_done) refers to tmr.o(.text.tmr_delay_done) for [Anonymous Symbol]
    tmr.o(.text.tmr_handler) refers to tmr.o(.text.TMR_ITStatus) for TMR_ITStatus
    tmr.o(.text.tmr_handler) refers to tmr.o(.text.TMR_ITStatusClear) for TMR_ITStatusClear
    tmr.o(.ARM.exidx.text.tmr_handler) refers to tmr.o(.text.tmr_handler) for [Anonymous Symbol]
    tmr.o(.ARM.exidx.text.TMR_ITStatus) refers to tmr.o(.text.TMR_ITStatus) for [Anonymous Symbol]
    tmr.o(.ARM.exidx.text.TMR_ITStatusClear) refers to tmr.o(.text.TMR_ITStatusClear) for [Anonymous Symbol]
    tmr.o(.ARM.exidx.text.TMR_SetLoad) refers to tmr.o(.text.TMR_SetLoad) for [Anonymous Symbol]
    tmr.o(.ARM.exidx.text.TMR_ITCmd) refers to tmr.o(.text.TMR_ITCmd) for [Anonymous Symbol]
    tmr.o(.ARM.exidx.text.TMR_DMAReqCmd) refers to tmr.o(.text.TMR_DMAReqCmd) for [Anonymous Symbol]
    tmr.o(.ARM.exidx.text.TMR_ADCSOCCmd) refers to tmr.o(.text.TMR_ADCSOCCmd) for [Anonymous Symbol]
    tmr.o(.ARM.exidx.text.TMR_ExtInputConfig) refers to tmr.o(.text.TMR_ExtInputConfig) for [Anonymous Symbol]
    uart.o(.text.uart_init_first) refers to uart.o(.text.uart1_gpio_init) for uart1_gpio_init
    uart.o(.text.uart_init_first) refers to uart.o(.text.RCU_UARTClkConfig) for RCU_UARTClkConfig
    uart.o(.text.uart_init_first) refers to uart.o(.text.RCU_UARTClkCmd) for RCU_UARTClkCmd
    uart.o(.text.uart_init_first) refers to plib035_uart.o(.text.UART_DeInit) for UART_DeInit
    uart.o(.text.uart_init_first) refers to uart.o(.text.__NVIC_EnableIRQ) for __NVIC_EnableIRQ
    uart.o(.text.uart_init_first) refers to uart.o(.bss.huart1) for huart1
    uart.o(.text.uart_init_first) refers to uart.o(.data.uart1_config) for uart1_config
    uart.o(.text.uart_init_first) refers to uart.o(.text.uart_init) for uart_init
    uart.o(.ARM.exidx.text.uart_init_first) refers to uart.o(.text.uart_init_first) for [Anonymous Symbol]
    uart.o(.text.uart1_gpio_init) refers to gpio.o(.text.gpio_get_init) for gpio_get_init
    uart.o(.text.uart1_gpio_init) refers to uart.o(.data.uart1_config) for uart1_config
    uart.o(.text.uart1_gpio_init) refers to plib035_gpio.o(.text.GPIO_StructInit) for GPIO_StructInit
    uart.o(.text.uart1_gpio_init) refers to plib035_gpio.o(.text.GPIO_Init) for GPIO_Init
    uart.o(.ARM.exidx.text.uart1_gpio_init) refers to uart.o(.text.uart1_gpio_init) for [Anonymous Symbol]
    uart.o(.ARM.exidx.text.RCU_UARTClkConfig) refers to uart.o(.text.RCU_UARTClkConfig) for [Anonymous Symbol]
    uart.o(.ARM.exidx.text.RCU_UARTClkCmd) refers to uart.o(.text.RCU_UARTClkCmd) for [Anonymous Symbol]
    uart.o(.ARM.exidx.text.__NVIC_EnableIRQ) refers to uart.o(.text.__NVIC_EnableIRQ) for [Anonymous Symbol]
    uart.o(.text.uart_init) refers to plib035_uart.o(.text.UART_Init) for UART_Init
    uart.o(.ARM.exidx.text.uart_init) refers to uart.o(.text.uart_init) for [Anonymous Symbol]
    uart.o(.text.uart_start) refers to uart.o(.text.UART_ITFIFOLevelRxConfig) for UART_ITFIFOLevelRxConfig
    uart.o(.text.uart_start) refers to uart.o(.text.UART_ITFIFOLevelTxConfig) for UART_ITFIFOLevelTxConfig
    uart.o(.text.uart_start) refers to uart.o(.text.UART_Cmd) for UART_Cmd
    uart.o(.ARM.exidx.text.uart_start) refers to uart.o(.text.uart_start) for [Anonymous Symbol]
    uart.o(.ARM.exidx.text.UART_ITFIFOLevelRxConfig) refers to uart.o(.text.UART_ITFIFOLevelRxConfig) for [Anonymous Symbol]
    uart.o(.ARM.exidx.text.UART_ITFIFOLevelTxConfig) refers to uart.o(.text.UART_ITFIFOLevelTxConfig) for [Anonymous Symbol]
    uart.o(.ARM.exidx.text.UART_Cmd) refers to uart.o(.text.UART_Cmd) for [Anonymous Symbol]
    uart.o(.text.uart_transmit) refers to sysclk.o(.text.millis) for millis
    uart.o(.text.uart_transmit) refers to uart.o(.text.__uart_fifo_transmit) for __uart_fifo_transmit
    uart.o(.ARM.exidx.text.uart_transmit) refers to uart.o(.text.uart_transmit) for [Anonymous Symbol]
    uart.o(.text.__uart_fifo_transmit) refers to uart.o(.text.UART_FlagStatus) for UART_FlagStatus
    uart.o(.text.__uart_fifo_transmit) refers to uart.o(.text.UART_SendData) for UART_SendData
    uart.o(.text.__uart_fifo_transmit) refers to uart.o(.text.UART_ITCmd) for UART_ITCmd
    uart.o(.ARM.exidx.text.__uart_fifo_transmit) refers to uart.o(.text.__uart_fifo_transmit) for [Anonymous Symbol]
    uart.o(.text.uart_receive) refers to sysclk.o(.text.millis) for millis
    uart.o(.text.uart_receive) refers to uart.o(.text.__uart_fifo_transmit) for __uart_fifo_transmit
    uart.o(.ARM.exidx.text.uart_receive) refers to uart.o(.text.uart_receive) for [Anonymous Symbol]
    uart.o(.text.uart_transmit_it) refers to uart.o(.text.UART_ITCmd) for UART_ITCmd
    uart.o(.text.uart_transmit_it) refers to uart.o(.text.__uart_fifo_transmit) for __uart_fifo_transmit
    uart.o(.ARM.exidx.text.uart_transmit_it) refers to uart.o(.text.uart_transmit_it) for [Anonymous Symbol]
    uart.o(.ARM.exidx.text.UART_ITCmd) refers to uart.o(.text.UART_ITCmd) for [Anonymous Symbol]
    uart.o(.text.uart_receive_it) refers to uart.o(.text.UART_ITCmd) for UART_ITCmd
    uart.o(.ARM.exidx.text.uart_receive_it) refers to uart.o(.text.uart_receive_it) for [Anonymous Symbol]
    uart.o(.text.uart_handler) refers to uart.o(.text.UART_ErrorStatusClear) for UART_ErrorStatusClear
    uart.o(.text.uart_handler) refers to uart.o(.text.UART_ITStatusClear) for UART_ITStatusClear
    uart.o(.text.uart_handler) refers to uart.o(.text.__uart_fifo_receive) for __uart_fifo_receive
    uart.o(.text.uart_handler) refers to uart.o(.text.UART_ITCmd) for UART_ITCmd
    uart.o(.text.uart_handler) refers to uart.o(.text.__uart_fifo_transmit) for __uart_fifo_transmit
    uart.o(.ARM.exidx.text.uart_handler) refers to uart.o(.text.uart_handler) for [Anonymous Symbol]
    uart.o(.ARM.exidx.text.UART_ErrorStatusClear) refers to uart.o(.text.UART_ErrorStatusClear) for [Anonymous Symbol]
    uart.o(.ARM.exidx.text.UART_ITStatusClear) refers to uart.o(.text.UART_ITStatusClear) for [Anonymous Symbol]
    uart.o(.text.__uart_fifo_receive) refers to uart.o(.text.UART_FlagStatus) for UART_FlagStatus
    uart.o(.text.__uart_fifo_receive) refers to uart.o(.text.UART_RecieveData) for UART_RecieveData
    uart.o(.text.__uart_fifo_receive) refers to uart.o(.text.UART_ITCmd) for UART_ITCmd
    uart.o(.ARM.exidx.text.__uart_fifo_receive) refers to uart.o(.text.__uart_fifo_receive) for [Anonymous Symbol]
    uart.o(.ARM.exidx.text.uart_set_callback) refers to uart.o(.text.uart_set_callback) for [Anonymous Symbol]
    uart.o(.ARM.exidx.text.uart0_gpio_init) refers to uart.o(.text.uart0_gpio_init) for [Anonymous Symbol]
    uart.o(.ARM.exidx.text.uart0_gpio_deinit) refers to uart.o(.text.uart0_gpio_deinit) for [Anonymous Symbol]
    uart.o(.text.uart1_gpio_deinit) refers to gpio.o(.text.gpio_get_init) for gpio_get_init
    uart.o(.text.uart1_gpio_deinit) refers to plib035_gpio.o(.text.GPIO_StructInit) for GPIO_StructInit
    uart.o(.text.uart1_gpio_deinit) refers to plib035_gpio.o(.text.GPIO_Init) for GPIO_Init
    uart.o(.ARM.exidx.text.uart1_gpio_deinit) refers to uart.o(.text.uart1_gpio_deinit) for [Anonymous Symbol]
    uart.o(.ARM.exidx.text.UART_FlagStatus) refers to uart.o(.text.UART_FlagStatus) for [Anonymous Symbol]
    uart.o(.ARM.exidx.text.UART_RecieveData) refers to uart.o(.text.UART_RecieveData) for [Anonymous Symbol]
    uart.o(.ARM.exidx.text.UART_SendData) refers to uart.o(.text.UART_SendData) for [Anonymous Symbol]
    sysclk.o(.text.sysclk_init) refers to sysclk.o(.data.SYSCLK_Oscil_Type) for SYSCLK_Oscil_Type
    sysclk.o(.text.sysclk_init) refers to plib035_rcu.o(.text.RCU_PLL_AutoConfig) for RCU_PLL_AutoConfig
    sysclk.o(.text.sysclk_init) refers to main.o(.text.Error_Handler) for Error_Handler
    sysclk.o(.text.sysclk_init) refers to system_k1921vk035.o(.text.SystemCoreClockUpdate) for SystemCoreClockUpdate
    sysclk.o(.text.sysclk_init) refers to sysclk.o(.text.RCU_ClkOutConfig) for RCU_ClkOutConfig
    sysclk.o(.text.sysclk_init) refers to sysclk.o(.text.RCU_ClkOutCmd) for RCU_ClkOutCmd
    sysclk.o(.text.sysclk_init) refers to sysclk.o(.text.SysTick_Config) for SysTick_Config
    sysclk.o(.ARM.exidx.text.sysclk_init) refers to sysclk.o(.text.sysclk_init) for [Anonymous Symbol]
    sysclk.o(.ARM.exidx.text.RCU_ClkOutConfig) refers to sysclk.o(.text.RCU_ClkOutConfig) for [Anonymous Symbol]
    sysclk.o(.ARM.exidx.text.RCU_ClkOutCmd) refers to sysclk.o(.text.RCU_ClkOutCmd) for [Anonymous Symbol]
    sysclk.o(.text.SysTick_Config) refers to sysclk.o(.text.__NVIC_SetPriority) for __NVIC_SetPriority
    sysclk.o(.ARM.exidx.text.SysTick_Config) refers to sysclk.o(.text.SysTick_Config) for [Anonymous Symbol]
    sysclk.o(.text.millis) refers to sysclk.o(.bss.uwTick) for uwTick
    sysclk.o(.ARM.exidx.text.millis) refers to sysclk.o(.text.millis) for [Anonymous Symbol]
    sysclk.o(.text.millis_inc) refers to sysclk.o(.bss.uwTick) for uwTick
    sysclk.o(.ARM.exidx.text.millis_inc) refers to sysclk.o(.text.millis_inc) for [Anonymous Symbol]
    sysclk.o(.ARM.exidx.text.micros) refers to sysclk.o(.text.micros) for [Anonymous Symbol]
    sysclk.o(.text.micros_inc) refers to sysclk.o(.bss.uwTick) for uwTick
    sysclk.o(.ARM.exidx.text.micros_inc) refers to sysclk.o(.text.micros_inc) for [Anonymous Symbol]
    sysclk.o(.ARM.exidx.text.__NVIC_SetPriority) refers to sysclk.o(.text.__NVIC_SetPriority) for [Anonymous Symbol]
    vk035_it.o(.ARM.exidx.text.WDT_IRQHandler) refers to vk035_it.o(.text.WDT_IRQHandler) for [Anonymous Symbol]
    vk035_it.o(.ARM.exidx.text.RCU_IRQHandler) refers to vk035_it.o(.text.RCU_IRQHandler) for [Anonymous Symbol]
    vk035_it.o(.ARM.exidx.text.MFLASH_IRQHandler) refers to vk035_it.o(.text.MFLASH_IRQHandler) for [Anonymous Symbol]
    vk035_it.o(.ARM.exidx.text.GPIOA_IRQHandler) refers to vk035_it.o(.text.GPIOA_IRQHandler) for [Anonymous Symbol]
    vk035_it.o(.ARM.exidx.text.GPIOB_IRQHandler) refers to vk035_it.o(.text.GPIOB_IRQHandler) for [Anonymous Symbol]
    vk035_it.o(.text.TMR0_IRQHandler) refers to tmr.o(.bss.htmr0) for htmr0
    vk035_it.o(.text.TMR0_IRQHandler) refers to tmr.o(.text.tmr_handler) for tmr_handler
    vk035_it.o(.ARM.exidx.text.TMR0_IRQHandler) refers to vk035_it.o(.text.TMR0_IRQHandler) for [Anonymous Symbol]
    vk035_it.o(.text.TMR1_IRQHandler) refers to tmr.o(.bss.htmr1) for htmr1
    vk035_it.o(.text.TMR1_IRQHandler) refers to tmr.o(.text.tmr_handler) for tmr_handler
    vk035_it.o(.ARM.exidx.text.TMR1_IRQHandler) refers to vk035_it.o(.text.TMR1_IRQHandler) for [Anonymous Symbol]
    vk035_it.o(.text.TMR2_IRQHandler) refers to tmr.o(.bss.htmr2) for htmr2
    vk035_it.o(.text.TMR2_IRQHandler) refers to tmr.o(.text.tmr_handler) for tmr_handler
    vk035_it.o(.ARM.exidx.text.TMR2_IRQHandler) refers to vk035_it.o(.text.TMR2_IRQHandler) for [Anonymous Symbol]
    vk035_it.o(.text.TMR3_IRQHandler) refers to tmr.o(.bss.htmr3) for htmr3
    vk035_it.o(.text.TMR3_IRQHandler) refers to tmr.o(.text.tmr_handler) for tmr_handler
    vk035_it.o(.ARM.exidx.text.TMR3_IRQHandler) refers to vk035_it.o(.text.TMR3_IRQHandler) for [Anonymous Symbol]
    vk035_it.o(.text.UART0_TD_IRQHandler) refers to uart.o(.bss.huart0) for huart0
    vk035_it.o(.text.UART0_TD_IRQHandler) refers to uart.o(.text.uart_handler) for uart_handler
    vk035_it.o(.ARM.exidx.text.UART0_TD_IRQHandler) refers to vk035_it.o(.text.UART0_TD_IRQHandler) for [Anonymous Symbol]
    vk035_it.o(.text.UART0_RX_IRQHandler) refers to uart.o(.bss.huart0) for huart0
    vk035_it.o(.text.UART0_RX_IRQHandler) refers to uart.o(.text.uart_handler) for uart_handler
    vk035_it.o(.ARM.exidx.text.UART0_RX_IRQHandler) refers to vk035_it.o(.text.UART0_RX_IRQHandler) for [Anonymous Symbol]
    vk035_it.o(.text.UART0_TX_IRQHandler) refers to uart.o(.bss.huart0) for huart0
    vk035_it.o(.text.UART0_TX_IRQHandler) refers to uart.o(.text.uart_handler) for uart_handler
    vk035_it.o(.ARM.exidx.text.UART0_TX_IRQHandler) refers to vk035_it.o(.text.UART0_TX_IRQHandler) for [Anonymous Symbol]
    vk035_it.o(.text.UART0_E_RT_IRQHandler) refers to uart.o(.bss.huart0) for huart0
    vk035_it.o(.text.UART0_E_RT_IRQHandler) refers to uart.o(.text.uart_handler) for uart_handler
    vk035_it.o(.ARM.exidx.text.UART0_E_RT_IRQHandler) refers to vk035_it.o(.text.UART0_E_RT_IRQHandler) for [Anonymous Symbol]
    vk035_it.o(.text.UART1_TD_IRQHandler) refers to uart.o(.bss.huart1) for huart1
    vk035_it.o(.text.UART1_TD_IRQHandler) refers to uart.o(.text.uart_handler) for uart_handler
    vk035_it.o(.ARM.exidx.text.UART1_TD_IRQHandler) refers to vk035_it.o(.text.UART1_TD_IRQHandler) for [Anonymous Symbol]
    vk035_it.o(.text.UART1_RX_IRQHandler) refers to uart.o(.bss.huart1) for huart1
    vk035_it.o(.text.UART1_RX_IRQHandler) refers to uart.o(.text.uart_handler) for uart_handler
    vk035_it.o(.ARM.exidx.text.UART1_RX_IRQHandler) refers to vk035_it.o(.text.UART1_RX_IRQHandler) for [Anonymous Symbol]
    vk035_it.o(.text.UART1_TX_IRQHandler) refers to uart.o(.bss.huart1) for huart1
    vk035_it.o(.text.UART1_TX_IRQHandler) refers to uart.o(.text.uart_handler) for uart_handler
    vk035_it.o(.ARM.exidx.text.UART1_TX_IRQHandler) refers to vk035_it.o(.text.UART1_TX_IRQHandler) for [Anonymous Symbol]
    vk035_it.o(.text.UART1_E_RT_IRQHandler) refers to uart.o(.bss.huart1) for huart1
    vk035_it.o(.text.UART1_E_RT_IRQHandler) refers to uart.o(.text.uart_handler) for uart_handler
    vk035_it.o(.ARM.exidx.text.UART1_E_RT_IRQHandler) refers to vk035_it.o(.text.UART1_E_RT_IRQHandler) for [Anonymous Symbol]
    vk035_it.o(.ARM.exidx.text.SPI_RO_RT_IRQHandler) refers to vk035_it.o(.text.SPI_RO_RT_IRQHandler) for [Anonymous Symbol]
    vk035_it.o(.ARM.exidx.text.SPI_RX_IRQHandler) refers to vk035_it.o(.text.SPI_RX_IRQHandler) for [Anonymous Symbol]
    vk035_it.o(.ARM.exidx.text.SPI_TX_IRQHandler) refers to vk035_it.o(.text.SPI_TX_IRQHandler) for [Anonymous Symbol]
    vk035_it.o(.ARM.exidx.text.I2C_IRQHandler) refers to vk035_it.o(.text.I2C_IRQHandler) for [Anonymous Symbol]
    vk035_it.o(.ARM.exidx.text.ECAP0_IRQHandler) refers to vk035_it.o(.text.ECAP0_IRQHandler) for [Anonymous Symbol]
    vk035_it.o(.ARM.exidx.text.ECAP1_IRQHandler) refers to vk035_it.o(.text.ECAP1_IRQHandler) for [Anonymous Symbol]
    vk035_it.o(.ARM.exidx.text.ECAP2_IRQHandler) refers to vk035_it.o(.text.ECAP2_IRQHandler) for [Anonymous Symbol]
    vk035_it.o(.ARM.exidx.text.PWM0_IRQHandler) refers to vk035_it.o(.text.PWM0_IRQHandler) for [Anonymous Symbol]
    vk035_it.o(.ARM.exidx.text.PWM0_HD_IRQHandler) refers to vk035_it.o(.text.PWM0_HD_IRQHandler) for [Anonymous Symbol]
    vk035_it.o(.ARM.exidx.text.PWM0_TZ_IRQHandler) refers to vk035_it.o(.text.PWM0_TZ_IRQHandler) for [Anonymous Symbol]
    vk035_it.o(.ARM.exidx.text.PWM1_IRQHandler) refers to vk035_it.o(.text.PWM1_IRQHandler) for [Anonymous Symbol]
    vk035_it.o(.ARM.exidx.text.PWM1_HD_IRQHandler) refers to vk035_it.o(.text.PWM1_HD_IRQHandler) for [Anonymous Symbol]
    vk035_it.o(.ARM.exidx.text.PWM1_TZ_IRQHandler) refers to vk035_it.o(.text.PWM1_TZ_IRQHandler) for [Anonymous Symbol]
    vk035_it.o(.ARM.exidx.text.PWM2_IRQHandler) refers to vk035_it.o(.text.PWM2_IRQHandler) for [Anonymous Symbol]
    vk035_it.o(.ARM.exidx.text.PWM2_HD_IRQHandler) refers to vk035_it.o(.text.PWM2_HD_IRQHandler) for [Anonymous Symbol]
    vk035_it.o(.ARM.exidx.text.PWM2_TZ_IRQHandler) refers to vk035_it.o(.text.PWM2_TZ_IRQHandler) for [Anonymous Symbol]
    vk035_it.o(.ARM.exidx.text.QEP_IRQHandler) refers to vk035_it.o(.text.QEP_IRQHandler) for [Anonymous Symbol]
    vk035_it.o(.ARM.exidx.text.ADC_SEQ0_IRQHandler) refers to vk035_it.o(.text.ADC_SEQ0_IRQHandler) for [Anonymous Symbol]
    vk035_it.o(.ARM.exidx.text.ADC_SEQ1_IRQHandler) refers to vk035_it.o(.text.ADC_SEQ1_IRQHandler) for [Anonymous Symbol]
    vk035_it.o(.ARM.exidx.text.ADC_DC_IRQHandler) refers to vk035_it.o(.text.ADC_DC_IRQHandler) for [Anonymous Symbol]
    vk035_it.o(.ARM.exidx.text.CAN0_IRQHandler) refers to vk035_it.o(.text.CAN0_IRQHandler) for [Anonymous Symbol]
    vk035_it.o(.ARM.exidx.text.CAN1_IRQHandler) refers to vk035_it.o(.text.CAN1_IRQHandler) for [Anonymous Symbol]
    vk035_it.o(.ARM.exidx.text.CAN2_IRQHandler) refers to vk035_it.o(.text.CAN2_IRQHandler) for [Anonymous Symbol]
    vk035_it.o(.ARM.exidx.text.CAN3_IRQHandler) refers to vk035_it.o(.text.CAN3_IRQHandler) for [Anonymous Symbol]
    vk035_it.o(.ARM.exidx.text.CAN4_IRQHandler) refers to vk035_it.o(.text.CAN4_IRQHandler) for [Anonymous Symbol]
    vk035_it.o(.ARM.exidx.text.CAN5_IRQHandler) refers to vk035_it.o(.text.CAN5_IRQHandler) for [Anonymous Symbol]
    vk035_it.o(.ARM.exidx.text.CAN6_IRQHandler) refers to vk035_it.o(.text.CAN6_IRQHandler) for [Anonymous Symbol]
    vk035_it.o(.ARM.exidx.text.CAN7_IRQHandler) refers to vk035_it.o(.text.CAN7_IRQHandler) for [Anonymous Symbol]
    vk035_it.o(.ARM.exidx.text.CAN8_IRQHandler) refers to vk035_it.o(.text.CAN8_IRQHandler) for [Anonymous Symbol]
    vk035_it.o(.ARM.exidx.text.CAN9_IRQHandler) refers to vk035_it.o(.text.CAN9_IRQHandler) for [Anonymous Symbol]
    vk035_it.o(.ARM.exidx.text.CAN10_IRQHandler) refers to vk035_it.o(.text.CAN10_IRQHandler) for [Anonymous Symbol]
    vk035_it.o(.ARM.exidx.text.CAN11_IRQHandler) refers to vk035_it.o(.text.CAN11_IRQHandler) for [Anonymous Symbol]
    vk035_it.o(.ARM.exidx.text.CAN12_IRQHandler) refers to vk035_it.o(.text.CAN12_IRQHandler) for [Anonymous Symbol]
    vk035_it.o(.ARM.exidx.text.CAN13_IRQHandler) refers to vk035_it.o(.text.CAN13_IRQHandler) for [Anonymous Symbol]
    vk035_it.o(.ARM.exidx.text.CAN14_IRQHandler) refers to vk035_it.o(.text.CAN14_IRQHandler) for [Anonymous Symbol]
    vk035_it.o(.ARM.exidx.text.CAN15_IRQHandler) refers to vk035_it.o(.text.CAN15_IRQHandler) for [Anonymous Symbol]
    vk035_it.o(.ARM.exidx.text.FPU_IRQHandler) refers to vk035_it.o(.text.FPU_IRQHandler) for [Anonymous Symbol]
    vk035_it.o(.ARM.exidx.text.DMA_CH0_IRQHandler) refers to vk035_it.o(.text.DMA_CH0_IRQHandler) for [Anonymous Symbol]
    vk035_it.o(.ARM.exidx.text.DMA_CH1_IRQHandler) refers to vk035_it.o(.text.DMA_CH1_IRQHandler) for [Anonymous Symbol]
    vk035_it.o(.ARM.exidx.text.DMA_CH2_IRQHandler) refers to vk035_it.o(.text.DMA_CH2_IRQHandler) for [Anonymous Symbol]
    vk035_it.o(.ARM.exidx.text.DMA_CH3_IRQHandler) refers to vk035_it.o(.text.DMA_CH3_IRQHandler) for [Anonymous Symbol]
    vk035_it.o(.ARM.exidx.text.DMA_CH4_IRQHandler) refers to vk035_it.o(.text.DMA_CH4_IRQHandler) for [Anonymous Symbol]
    vk035_it.o(.ARM.exidx.text.DMA_CH5_IRQHandler) refers to vk035_it.o(.text.DMA_CH5_IRQHandler) for [Anonymous Symbol]
    vk035_it.o(.ARM.exidx.text.DMA_CH6_IRQHandler) refers to vk035_it.o(.text.DMA_CH6_IRQHandler) for [Anonymous Symbol]
    vk035_it.o(.ARM.exidx.text.DMA_CH7_IRQHandler) refers to vk035_it.o(.text.DMA_CH7_IRQHandler) for [Anonymous Symbol]
    vk035_it.o(.ARM.exidx.text.DMA_CH8_IRQHandler) refers to vk035_it.o(.text.DMA_CH8_IRQHandler) for [Anonymous Symbol]
    vk035_it.o(.ARM.exidx.text.DMA_CH9_IRQHandler) refers to vk035_it.o(.text.DMA_CH9_IRQHandler) for [Anonymous Symbol]
    vk035_it.o(.ARM.exidx.text.DMA_CH10_IRQHandler) refers to vk035_it.o(.text.DMA_CH10_IRQHandler) for [Anonymous Symbol]
    vk035_it.o(.ARM.exidx.text.DMA_CH11_IRQHandler) refers to vk035_it.o(.text.DMA_CH11_IRQHandler) for [Anonymous Symbol]
    vk035_it.o(.ARM.exidx.text.DMA_CH12_IRQHandler) refers to vk035_it.o(.text.DMA_CH12_IRQHandler) for [Anonymous Symbol]
    vk035_it.o(.ARM.exidx.text.DMA_CH13_IRQHandler) refers to vk035_it.o(.text.DMA_CH13_IRQHandler) for [Anonymous Symbol]
    vk035_it.o(.ARM.exidx.text.DMA_CH14_IRQHandler) refers to vk035_it.o(.text.DMA_CH14_IRQHandler) for [Anonymous Symbol]
    vk035_it.o(.ARM.exidx.text.DMA_CH15_IRQHandler) refers to vk035_it.o(.text.DMA_CH15_IRQHandler) for [Anonymous Symbol]
    vk035_it.o(.ARM.exidx.text.NMI_Handler) refers to vk035_it.o(.text.NMI_Handler) for [Anonymous Symbol]
    vk035_it.o(.ARM.exidx.text.HardFault_Handler) refers to vk035_it.o(.text.HardFault_Handler) for [Anonymous Symbol]
    vk035_it.o(.ARM.exidx.text.MemManage_Handler) refers to vk035_it.o(.text.MemManage_Handler) for [Anonymous Symbol]
    vk035_it.o(.ARM.exidx.text.BusFault_Handler) refers to vk035_it.o(.text.BusFault_Handler) for [Anonymous Symbol]
    vk035_it.o(.ARM.exidx.text.UsageFault_Handler) refers to vk035_it.o(.text.UsageFault_Handler) for [Anonymous Symbol]
    vk035_it.o(.ARM.exidx.text.SVC_Handler) refers to vk035_it.o(.text.SVC_Handler) for [Anonymous Symbol]
    vk035_it.o(.ARM.exidx.text.DebugMon_Handler) refers to vk035_it.o(.text.DebugMon_Handler) for [Anonymous Symbol]
    vk035_it.o(.ARM.exidx.text.PendSV_Handler) refers to vk035_it.o(.text.PendSV_Handler) for [Anonymous Symbol]
    vk035_it.o(.text.SysTick_Handler) refers to sysclk.o(.text.millis_inc) for millis_inc
    vk035_it.o(.ARM.exidx.text.SysTick_Handler) refers to vk035_it.o(.text.SysTick_Handler) for [Anonymous Symbol]
    segger_rtt.o(.text.SEGGER_RTT_ReadUpBufferNoLock) refers to segger_rtt.o(.bss._SEGGER_RTT) for _SEGGER_RTT
    segger_rtt.o(.text.SEGGER_RTT_ReadUpBufferNoLock) refers to segger_rtt.o(.text._DoInit) for _DoInit
    segger_rtt.o(.text.SEGGER_RTT_ReadUpBufferNoLock) refers to rt_memcpy_v6.o(.text) for __aeabi_memcpy
    segger_rtt.o(.ARM.exidx.text.SEGGER_RTT_ReadUpBufferNoLock) refers to segger_rtt.o(.text.SEGGER_RTT_ReadUpBufferNoLock) for [Anonymous Symbol]
    segger_rtt.o(.text._DoInit) refers to segger_rtt.o(.bss._SEGGER_RTT) for _SEGGER_RTT
    segger_rtt.o(.text._DoInit) refers to rt_memclr_w.o(.text) for __aeabi_memclr4
    segger_rtt.o(.text._DoInit) refers to segger_rtt.o(.rodata.str1.1) for .L.str
    segger_rtt.o(.text._DoInit) refers to segger_rtt.o(.bss._acUpBuffer) for _acUpBuffer
    segger_rtt.o(.text._DoInit) refers to segger_rtt.o(.bss._acDownBuffer) for _acDownBuffer
    segger_rtt.o(.text._DoInit) refers to segger_rtt.o(.rodata._DoInit._aInitStr) for _DoInit._aInitStr
    segger_rtt.o(.ARM.exidx.text._DoInit) refers to segger_rtt.o(.text._DoInit) for [Anonymous Symbol]
    segger_rtt.o(.text.SEGGER_RTT_ReadNoLock) refers to segger_rtt.o(.bss._SEGGER_RTT) for _SEGGER_RTT
    segger_rtt.o(.text.SEGGER_RTT_ReadNoLock) refers to segger_rtt.o(.text._DoInit) for _DoInit
    segger_rtt.o(.text.SEGGER_RTT_ReadNoLock) refers to rt_memcpy_v6.o(.text) for __aeabi_memcpy
    segger_rtt.o(.ARM.exidx.text.SEGGER_RTT_ReadNoLock) refers to segger_rtt.o(.text.SEGGER_RTT_ReadNoLock) for [Anonymous Symbol]
    segger_rtt.o(.text.SEGGER_RTT_ReadUpBuffer) refers to segger_rtt.o(.text.SEGGER_RTT_ReadUpBufferNoLock) for SEGGER_RTT_ReadUpBufferNoLock
    segger_rtt.o(.ARM.exidx.text.SEGGER_RTT_ReadUpBuffer) refers to segger_rtt.o(.text.SEGGER_RTT_ReadUpBuffer) for [Anonymous Symbol]
    segger_rtt.o(.text.SEGGER_RTT_Read) refers to segger_rtt.o(.text.SEGGER_RTT_ReadNoLock) for SEGGER_RTT_ReadNoLock
    segger_rtt.o(.ARM.exidx.text.SEGGER_RTT_Read) refers to segger_rtt.o(.text.SEGGER_RTT_Read) for [Anonymous Symbol]
    segger_rtt.o(.text.SEGGER_RTT_WriteWithOverwriteNoLock) refers to segger_rtt.o(.bss._SEGGER_RTT) for _SEGGER_RTT
    segger_rtt.o(.text.SEGGER_RTT_WriteWithOverwriteNoLock) refers to rt_memcpy_v6.o(.text) for __aeabi_memcpy
    segger_rtt.o(.ARM.exidx.text.SEGGER_RTT_WriteWithOverwriteNoLock) refers to segger_rtt.o(.text.SEGGER_RTT_WriteWithOverwriteNoLock) for [Anonymous Symbol]
    segger_rtt.o(.text.SEGGER_RTT_WriteDownBufferNoLock) refers to segger_rtt.o(.bss._SEGGER_RTT) for _SEGGER_RTT
    segger_rtt.o(.text.SEGGER_RTT_WriteDownBufferNoLock) refers to segger_rtt.o(.text._GetAvailWriteSpace) for _GetAvailWriteSpace
    segger_rtt.o(.text.SEGGER_RTT_WriteDownBufferNoLock) refers to segger_rtt.o(.text._WriteNoCheck) for _WriteNoCheck
    segger_rtt.o(.text.SEGGER_RTT_WriteDownBufferNoLock) refers to segger_rtt.o(.text._WriteBlocking) for _WriteBlocking
    segger_rtt.o(.ARM.exidx.text.SEGGER_RTT_WriteDownBufferNoLock) refers to segger_rtt.o(.text.SEGGER_RTT_WriteDownBufferNoLock) for [Anonymous Symbol]
    segger_rtt.o(.ARM.exidx.text._GetAvailWriteSpace) refers to segger_rtt.o(.text._GetAvailWriteSpace) for [Anonymous Symbol]
    segger_rtt.o(.text._WriteNoCheck) refers to rt_memcpy_v6.o(.text) for __aeabi_memcpy
    segger_rtt.o(.ARM.exidx.text._WriteNoCheck) refers to segger_rtt.o(.text._WriteNoCheck) for [Anonymous Symbol]
    segger_rtt.o(.text._WriteBlocking) refers to rt_memcpy_v6.o(.text) for __aeabi_memcpy
    segger_rtt.o(.ARM.exidx.text._WriteBlocking) refers to segger_rtt.o(.text._WriteBlocking) for [Anonymous Symbol]
    segger_rtt.o(.text.SEGGER_RTT_WriteNoLock) refers to segger_rtt.o(.bss._SEGGER_RTT) for _SEGGER_RTT
    segger_rtt.o(.text.SEGGER_RTT_WriteNoLock) refers to segger_rtt.o(.text._GetAvailWriteSpace) for _GetAvailWriteSpace
    segger_rtt.o(.text.SEGGER_RTT_WriteNoLock) refers to segger_rtt.o(.text._WriteNoCheck) for _WriteNoCheck
    segger_rtt.o(.text.SEGGER_RTT_WriteNoLock) refers to segger_rtt.o(.text._WriteBlocking) for _WriteBlocking
    segger_rtt.o(.ARM.exidx.text.SEGGER_RTT_WriteNoLock) refers to segger_rtt.o(.text.SEGGER_RTT_WriteNoLock) for [Anonymous Symbol]
    segger_rtt.o(.text.SEGGER_RTT_WriteDownBuffer) refers to segger_rtt.o(.bss._SEGGER_RTT) for _SEGGER_RTT
    segger_rtt.o(.text.SEGGER_RTT_WriteDownBuffer) refers to segger_rtt.o(.text._DoInit) for _DoInit
    segger_rtt.o(.text.SEGGER_RTT_WriteDownBuffer) refers to segger_rtt.o(.text.SEGGER_RTT_WriteDownBufferNoLock) for SEGGER_RTT_WriteDownBufferNoLock
    segger_rtt.o(.ARM.exidx.text.SEGGER_RTT_WriteDownBuffer) refers to segger_rtt.o(.text.SEGGER_RTT_WriteDownBuffer) for [Anonymous Symbol]
    segger_rtt.o(.text.SEGGER_RTT_Write) refers to segger_rtt.o(.bss._SEGGER_RTT) for _SEGGER_RTT
    segger_rtt.o(.text.SEGGER_RTT_Write) refers to segger_rtt.o(.text._DoInit) for _DoInit
    segger_rtt.o(.text.SEGGER_RTT_Write) refers to segger_rtt.o(.text.SEGGER_RTT_WriteNoLock) for SEGGER_RTT_WriteNoLock
    segger_rtt.o(.ARM.exidx.text.SEGGER_RTT_Write) refers to segger_rtt.o(.text.SEGGER_RTT_Write) for [Anonymous Symbol]
    segger_rtt.o(.text.SEGGER_RTT_WriteString) refers to strlen.o(.text) for strlen
    segger_rtt.o(.text.SEGGER_RTT_WriteString) refers to segger_rtt.o(.text.SEGGER_RTT_Write) for SEGGER_RTT_Write
    segger_rtt.o(.ARM.exidx.text.SEGGER_RTT_WriteString) refers to segger_rtt.o(.text.SEGGER_RTT_WriteString) for [Anonymous Symbol]
    segger_rtt.o(.text.SEGGER_RTT_PutCharSkipNoLock) refers to segger_rtt.o(.bss._SEGGER_RTT) for _SEGGER_RTT
    segger_rtt.o(.ARM.exidx.text.SEGGER_RTT_PutCharSkipNoLock) refers to segger_rtt.o(.text.SEGGER_RTT_PutCharSkipNoLock) for [Anonymous Symbol]
    segger_rtt.o(.text.SEGGER_RTT_PutCharSkip) refers to segger_rtt.o(.bss._SEGGER_RTT) for _SEGGER_RTT
    segger_rtt.o(.text.SEGGER_RTT_PutCharSkip) refers to segger_rtt.o(.text._DoInit) for _DoInit
    segger_rtt.o(.ARM.exidx.text.SEGGER_RTT_PutCharSkip) refers to segger_rtt.o(.text.SEGGER_RTT_PutCharSkip) for [Anonymous Symbol]
    segger_rtt.o(.text.SEGGER_RTT_PutChar) refers to segger_rtt.o(.bss._SEGGER_RTT) for _SEGGER_RTT
    segger_rtt.o(.text.SEGGER_RTT_PutChar) refers to segger_rtt.o(.text._DoInit) for _DoInit
    segger_rtt.o(.ARM.exidx.text.SEGGER_RTT_PutChar) refers to segger_rtt.o(.text.SEGGER_RTT_PutChar) for [Anonymous Symbol]
    segger_rtt.o(.text.SEGGER_RTT_GetKey) refers to segger_rtt.o(.text.SEGGER_RTT_Read) for SEGGER_RTT_Read
    segger_rtt.o(.ARM.exidx.text.SEGGER_RTT_GetKey) refers to segger_rtt.o(.text.SEGGER_RTT_GetKey) for [Anonymous Symbol]
    segger_rtt.o(.text.SEGGER_RTT_WaitKey) refers to segger_rtt.o(.text.SEGGER_RTT_GetKey) for SEGGER_RTT_GetKey
    segger_rtt.o(.ARM.exidx.text.SEGGER_RTT_WaitKey) refers to segger_rtt.o(.text.SEGGER_RTT_WaitKey) for [Anonymous Symbol]
    segger_rtt.o(.text.SEGGER_RTT_HasKey) refers to segger_rtt.o(.bss._SEGGER_RTT) for _SEGGER_RTT
    segger_rtt.o(.text.SEGGER_RTT_HasKey) refers to segger_rtt.o(.text._DoInit) for _DoInit
    segger_rtt.o(.ARM.exidx.text.SEGGER_RTT_HasKey) refers to segger_rtt.o(.text.SEGGER_RTT_HasKey) for [Anonymous Symbol]
    segger_rtt.o(.text.SEGGER_RTT_HasData) refers to segger_rtt.o(.bss._SEGGER_RTT) for _SEGGER_RTT
    segger_rtt.o(.ARM.exidx.text.SEGGER_RTT_HasData) refers to segger_rtt.o(.text.SEGGER_RTT_HasData) for [Anonymous Symbol]
    segger_rtt.o(.text.SEGGER_RTT_HasDataUp) refers to segger_rtt.o(.bss._SEGGER_RTT) for _SEGGER_RTT
    segger_rtt.o(.ARM.exidx.text.SEGGER_RTT_HasDataUp) refers to segger_rtt.o(.text.SEGGER_RTT_HasDataUp) for [Anonymous Symbol]
    segger_rtt.o(.text.SEGGER_RTT_AllocDownBuffer) refers to segger_rtt.o(.bss._SEGGER_RTT) for _SEGGER_RTT
    segger_rtt.o(.text.SEGGER_RTT_AllocDownBuffer) refers to segger_rtt.o(.text._DoInit) for _DoInit
    segger_rtt.o(.ARM.exidx.text.SEGGER_RTT_AllocDownBuffer) refers to segger_rtt.o(.text.SEGGER_RTT_AllocDownBuffer) for [Anonymous Symbol]
    segger_rtt.o(.text.SEGGER_RTT_AllocUpBuffer) refers to segger_rtt.o(.bss._SEGGER_RTT) for _SEGGER_RTT
    segger_rtt.o(.text.SEGGER_RTT_AllocUpBuffer) refers to segger_rtt.o(.text._DoInit) for _DoInit
    segger_rtt.o(.ARM.exidx.text.SEGGER_RTT_AllocUpBuffer) refers to segger_rtt.o(.text.SEGGER_RTT_AllocUpBuffer) for [Anonymous Symbol]
    segger_rtt.o(.text.SEGGER_RTT_ConfigUpBuffer) refers to segger_rtt.o(.bss._SEGGER_RTT) for _SEGGER_RTT
    segger_rtt.o(.text.SEGGER_RTT_ConfigUpBuffer) refers to segger_rtt.o(.text._DoInit) for _DoInit
    segger_rtt.o(.ARM.exidx.text.SEGGER_RTT_ConfigUpBuffer) refers to segger_rtt.o(.text.SEGGER_RTT_ConfigUpBuffer) for [Anonymous Symbol]
    segger_rtt.o(.text.SEGGER_RTT_ConfigDownBuffer) refers to segger_rtt.o(.bss._SEGGER_RTT) for _SEGGER_RTT
    segger_rtt.o(.text.SEGGER_RTT_ConfigDownBuffer) refers to segger_rtt.o(.text._DoInit) for _DoInit
    segger_rtt.o(.ARM.exidx.text.SEGGER_RTT_ConfigDownBuffer) refers to segger_rtt.o(.text.SEGGER_RTT_ConfigDownBuffer) for [Anonymous Symbol]
    segger_rtt.o(.text.SEGGER_RTT_SetNameUpBuffer) refers to segger_rtt.o(.bss._SEGGER_RTT) for _SEGGER_RTT
    segger_rtt.o(.text.SEGGER_RTT_SetNameUpBuffer) refers to segger_rtt.o(.text._DoInit) for _DoInit
    segger_rtt.o(.ARM.exidx.text.SEGGER_RTT_SetNameUpBuffer) refers to segger_rtt.o(.text.SEGGER_RTT_SetNameUpBuffer) for [Anonymous Symbol]
    segger_rtt.o(.text.SEGGER_RTT_SetNameDownBuffer) refers to segger_rtt.o(.bss._SEGGER_RTT) for _SEGGER_RTT
    segger_rtt.o(.text.SEGGER_RTT_SetNameDownBuffer) refers to segger_rtt.o(.text._DoInit) for _DoInit
    segger_rtt.o(.ARM.exidx.text.SEGGER_RTT_SetNameDownBuffer) refers to segger_rtt.o(.text.SEGGER_RTT_SetNameDownBuffer) for [Anonymous Symbol]
    segger_rtt.o(.text.SEGGER_RTT_SetFlagsUpBuffer) refers to segger_rtt.o(.bss._SEGGER_RTT) for _SEGGER_RTT
    segger_rtt.o(.text.SEGGER_RTT_SetFlagsUpBuffer) refers to segger_rtt.o(.text._DoInit) for _DoInit
    segger_rtt.o(.ARM.exidx.text.SEGGER_RTT_SetFlagsUpBuffer) refers to segger_rtt.o(.text.SEGGER_RTT_SetFlagsUpBuffer) for [Anonymous Symbol]
    segger_rtt.o(.text.SEGGER_RTT_SetFlagsDownBuffer) refers to segger_rtt.o(.bss._SEGGER_RTT) for _SEGGER_RTT
    segger_rtt.o(.text.SEGGER_RTT_SetFlagsDownBuffer) refers to segger_rtt.o(.text._DoInit) for _DoInit
    segger_rtt.o(.ARM.exidx.text.SEGGER_RTT_SetFlagsDownBuffer) refers to segger_rtt.o(.text.SEGGER_RTT_SetFlagsDownBuffer) for [Anonymous Symbol]
    segger_rtt.o(.text.SEGGER_RTT_Init) refers to segger_rtt.o(.text._DoInit) for _DoInit
    segger_rtt.o(.ARM.exidx.text.SEGGER_RTT_Init) refers to segger_rtt.o(.text.SEGGER_RTT_Init) for [Anonymous Symbol]
    segger_rtt.o(.text.SEGGER_RTT_SetTerminal) refers to segger_rtt.o(.bss._SEGGER_RTT) for _SEGGER_RTT
    segger_rtt.o(.text.SEGGER_RTT_SetTerminal) refers to segger_rtt.o(.text._DoInit) for _DoInit
    segger_rtt.o(.text.SEGGER_RTT_SetTerminal) refers to segger_rtt.o(.rodata._aTerminalId) for _aTerminalId
    segger_rtt.o(.text.SEGGER_RTT_SetTerminal) refers to segger_rtt.o(.bss._ActiveTerminal) for _ActiveTerminal
    segger_rtt.o(.text.SEGGER_RTT_SetTerminal) refers to segger_rtt.o(.text._WriteBlocking) for _WriteBlocking
    segger_rtt.o(.text.SEGGER_RTT_SetTerminal) refers to segger_rtt.o(.text._GetAvailWriteSpace) for _GetAvailWriteSpace
    segger_rtt.o(.text.SEGGER_RTT_SetTerminal) refers to segger_rtt.o(.text._WriteNoCheck) for _WriteNoCheck
    segger_rtt.o(.ARM.exidx.text.SEGGER_RTT_SetTerminal) refers to segger_rtt.o(.text.SEGGER_RTT_SetTerminal) for [Anonymous Symbol]
    segger_rtt.o(.text.SEGGER_RTT_TerminalOut) refers to segger_rtt.o(.bss._SEGGER_RTT) for _SEGGER_RTT
    segger_rtt.o(.text.SEGGER_RTT_TerminalOut) refers to segger_rtt.o(.text._DoInit) for _DoInit
    segger_rtt.o(.text.SEGGER_RTT_TerminalOut) refers to strlen.o(.text) for strlen
    segger_rtt.o(.text.SEGGER_RTT_TerminalOut) refers to segger_rtt.o(.text._GetAvailWriteSpace) for _GetAvailWriteSpace
    segger_rtt.o(.text.SEGGER_RTT_TerminalOut) refers to segger_rtt.o(.text._PostTerminalSwitch) for _PostTerminalSwitch
    segger_rtt.o(.text.SEGGER_RTT_TerminalOut) refers to segger_rtt.o(.text._WriteBlocking) for _WriteBlocking
    segger_rtt.o(.text.SEGGER_RTT_TerminalOut) refers to segger_rtt.o(.bss._ActiveTerminal) for _ActiveTerminal
    segger_rtt.o(.ARM.exidx.text.SEGGER_RTT_TerminalOut) refers to segger_rtt.o(.text.SEGGER_RTT_TerminalOut) for [Anonymous Symbol]
    segger_rtt.o(.text._PostTerminalSwitch) refers to segger_rtt.o(.rodata._aTerminalId) for _aTerminalId
    segger_rtt.o(.text._PostTerminalSwitch) refers to segger_rtt.o(.text._WriteBlocking) for _WriteBlocking
    segger_rtt.o(.ARM.exidx.text._PostTerminalSwitch) refers to segger_rtt.o(.text._PostTerminalSwitch) for [Anonymous Symbol]
    segger_rtt.o(.text.SEGGER_RTT_GetAvailWriteSpace) refers to segger_rtt.o(.bss._SEGGER_RTT) for _SEGGER_RTT
    segger_rtt.o(.text.SEGGER_RTT_GetAvailWriteSpace) refers to segger_rtt.o(.text._GetAvailWriteSpace) for _GetAvailWriteSpace
    segger_rtt.o(.ARM.exidx.text.SEGGER_RTT_GetAvailWriteSpace) refers to segger_rtt.o(.text.SEGGER_RTT_GetAvailWriteSpace) for [Anonymous Symbol]
    segger_rtt.o(.text.SEGGER_RTT_GetBytesInBuffer) refers to segger_rtt.o(.bss._SEGGER_RTT) for _SEGGER_RTT
    segger_rtt.o(.ARM.exidx.text.SEGGER_RTT_GetBytesInBuffer) refers to segger_rtt.o(.text.SEGGER_RTT_GetBytesInBuffer) for [Anonymous Symbol]
    segger_rtt_printf.o(.text.SEGGER_RTT_vprintf) refers to segger_rtt_printf.o(.text._StoreChar) for _StoreChar
    segger_rtt_printf.o(.text.SEGGER_RTT_vprintf) refers to segger_rtt_printf.o(.text._PrintInt) for _PrintInt
    segger_rtt_printf.o(.text.SEGGER_RTT_vprintf) refers to segger_rtt_printf.o(.text._PrintUnsigned) for _PrintUnsigned
    segger_rtt_printf.o(.text.SEGGER_RTT_vprintf) refers to segger_rtt_printf.o(.rodata.str1.1) for .L.str
    segger_rtt_printf.o(.text.SEGGER_RTT_vprintf) refers to segger_rtt.o(.text.SEGGER_RTT_Write) for SEGGER_RTT_Write
    segger_rtt_printf.o(.ARM.exidx.text.SEGGER_RTT_vprintf) refers to segger_rtt_printf.o(.text.SEGGER_RTT_vprintf) for [Anonymous Symbol]
    segger_rtt_printf.o(.text._StoreChar) refers to segger_rtt.o(.text.SEGGER_RTT_Write) for SEGGER_RTT_Write
    segger_rtt_printf.o(.ARM.exidx.text._StoreChar) refers to segger_rtt_printf.o(.text._StoreChar) for [Anonymous Symbol]
    segger_rtt_printf.o(.text._PrintInt) refers to segger_rtt_printf.o(.text._StoreChar) for _StoreChar
    segger_rtt_printf.o(.text._PrintInt) refers to segger_rtt_printf.o(.text._PrintUnsigned) for _PrintUnsigned
    segger_rtt_printf.o(.ARM.exidx.text._PrintInt) refers to segger_rtt_printf.o(.text._PrintInt) for [Anonymous Symbol]
    segger_rtt_printf.o(.text._PrintUnsigned) refers to segger_rtt_printf.o(.text._StoreChar) for _StoreChar
    segger_rtt_printf.o(.text._PrintUnsigned) refers to segger_rtt_printf.o(.rodata._PrintUnsigned._aV2C) for _PrintUnsigned._aV2C
    segger_rtt_printf.o(.ARM.exidx.text._PrintUnsigned) refers to segger_rtt_printf.o(.text._PrintUnsigned) for [Anonymous Symbol]
    segger_rtt_printf.o(.text.SEGGER_RTT_printf) refers to segger_rtt_printf.o(.text.SEGGER_RTT_vprintf) for SEGGER_RTT_vprintf
    segger_rtt_printf.o(.ARM.exidx.text.SEGGER_RTT_printf) refers to segger_rtt_printf.o(.text.SEGGER_RTT_printf) for [Anonymous Symbol]
    filters.o(.text.FilterMedian_Init) refers to filters.o(.text.FilterMedian_Process) for FilterMedian_Process
    filters.o(.ARM.exidx.text.FilterMedian_Init) refers to filters.o(.text.FilterMedian_Init) for [Anonymous Symbol]
    filters.o(.text.FilterMedian_Process) refers to filters.o(.text.Filter_float_compare) for Filter_float_compare
    filters.o(.text.FilterMedian_Process) refers to qsortnoex.o(.text) for qsort
    filters.o(.ARM.exidx.text.FilterMedian_Process) refers to filters.o(.text.FilterMedian_Process) for [Anonymous Symbol]
    filters.o(.ARM.exidx.text.Filter_float_compare) refers to filters.o(.text.Filter_float_compare) for [Anonymous Symbol]
    filters.o(.text.FilterExp_Init) refers to filters.o(.text.FilterExp_Process) for FilterExp_Process
    filters.o(.ARM.exidx.text.FilterExp_Init) refers to filters.o(.text.FilterExp_Init) for [Anonymous Symbol]
    filters.o(.ARM.exidx.text.FilterExp_Process) refers to filters.o(.text.FilterExp_Process) for [Anonymous Symbol]
    filters.o(.text.FilterAverage_Init) refers to filters.o(.text.FilterAverage_Process) for FilterAverage_Process
    filters.o(.ARM.exidx.text.FilterAverage_Init) refers to filters.o(.text.FilterAverage_Init) for [Anonymous Symbol]
    filters.o(.ARM.exidx.text.FilterAverage_Process) refers to filters.o(.text.FilterAverage_Process) for [Anonymous Symbol]
    filters.o(.text.FilterPoly_Init) refers to rt_memcpy_w.o(.text) for __aeabi_memcpy4
    filters.o(.text.FilterPoly_Init) refers to filters.o(.text.FilterPoly_Process) for FilterPoly_Process
    filters.o(.ARM.exidx.text.FilterPoly_Init) refers to filters.o(.text.FilterPoly_Init) for [Anonymous Symbol]
    filters.o(.ARM.exidx.text.FilterPoly_Process) refers to filters.o(.text.FilterPoly_Process) for [Anonymous Symbol]
    filters.o(.text.FilterLUT_Init) refers to filters.o(.text.FilterLUT_Process) for FilterLUT_Process
    filters.o(.ARM.exidx.text.FilterLUT_Init) refers to filters.o(.text.FilterLUT_Init) for [Anonymous Symbol]
    filters.o(.ARM.exidx.text.FilterLUT_Process) refers to filters.o(.text.FilterLUT_Process) for [Anonymous Symbol]
    filters.o(.text.FilterRMS_Init) refers to rt_memclr_w.o(.text) for __aeabi_memclr4
    filters.o(.text.FilterRMS_Init) refers to filters.o(.text.FilterRMS_Process) for FilterRMS_Process
    filters.o(.ARM.exidx.text.FilterRMS_Init) refers to filters.o(.text.FilterRMS_Init) for [Anonymous Symbol]
    filters.o(.text.FilterRMS_Process) refers to filters.o(.text._sqrtf) for _sqrtf
    filters.o(.ARM.exidx.text.FilterRMS_Process) refers to filters.o(.text.FilterRMS_Process) for [Anonymous Symbol]
    filters.o(.ARM.exidx.text._sqrtf) refers to filters.o(.text._sqrtf) for [Anonymous Symbol]
    filters.o(.text.FilterMedianInt_Init) refers to filters.o(.text.FilterMedianInt_Process) for FilterMedianInt_Process
    filters.o(.ARM.exidx.text.FilterMedianInt_Init) refers to filters.o(.text.FilterMedianInt_Init) for [Anonymous Symbol]
    filters.o(.ARM.exidx.text.FilterMedianInt_Process) refers to filters.o(.text.FilterMedianInt_Process) for [Anonymous Symbol]
    filters.o(.text.FilterExpInt_Init) refers to filters.o(.text.FilterExpInt_Process) for FilterExpInt_Process
    filters.o(.ARM.exidx.text.FilterExpInt_Init) refers to filters.o(.text.FilterExpInt_Init) for [Anonymous Symbol]
    filters.o(.text.FilterExpInt_Process) refers to llsdiv.o(.text) for __aeabi_ldivmod
    filters.o(.ARM.exidx.text.FilterExpInt_Process) refers to filters.o(.text.FilterExpInt_Process) for [Anonymous Symbol]
    filters.o(.text.FilterAverageInt_Init) refers to filters.o(.text.FilterAverageInt_Process) for FilterAverageInt_Process
    filters.o(.ARM.exidx.text.FilterAverageInt_Init) refers to filters.o(.text.FilterAverageInt_Init) for [Anonymous Symbol]
    filters.o(.text.FilterAverageInt_Process) refers to llsdiv.o(.text) for __aeabi_ldivmod
    filters.o(.ARM.exidx.text.FilterAverageInt_Process) refers to filters.o(.text.FilterAverageInt_Process) for [Anonymous Symbol]
    filters.o(.text.FilterPolyInt_Init) refers to rt_memcpy_w.o(.text) for __aeabi_memcpy4
    filters.o(.text.FilterPolyInt_Init) refers to filters.o(.text.FilterPolyInt_Process) for FilterPolyInt_Process
    filters.o(.ARM.exidx.text.FilterPolyInt_Init) refers to filters.o(.text.FilterPolyInt_Init) for [Anonymous Symbol]
    filters.o(.text.FilterPolyInt_Process) refers to llsdiv.o(.text) for __aeabi_ldivmod
    filters.o(.ARM.exidx.text.FilterPolyInt_Process) refers to filters.o(.text.FilterPolyInt_Process) for [Anonymous Symbol]
    filters.o(.text.FilterLUTInt_Init) refers to filters.o(.text.FilterLUTInt_Process) for FilterLUTInt_Process
    filters.o(.ARM.exidx.text.FilterLUTInt_Init) refers to filters.o(.text.FilterLUTInt_Init) for [Anonymous Symbol]
    filters.o(.text.FilterLUTInt_Process) refers to llsdiv.o(.text) for __aeabi_ldivmod
    filters.o(.ARM.exidx.text.FilterLUTInt_Process) refers to filters.o(.text.FilterLUTInt_Process) for [Anonymous Symbol]
    filters.o(.text.FilterRMSInt_Init) refers to rt_memclr_w.o(.text) for __aeabi_memclr8
    filters.o(.text.FilterRMSInt_Init) refers to filters.o(.text.FilterRMSInt_Process) for FilterRMSInt_Process
    filters.o(.ARM.exidx.text.FilterRMSInt_Init) refers to filters.o(.text.FilterRMSInt_Init) for [Anonymous Symbol]
    filters.o(.text.FilterRMSInt_Process) refers to llsdiv.o(.text) for __aeabi_ldivmod
    filters.o(.text.FilterRMSInt_Process) refers to ffltll_clz.o(x$fpl$ffltll) for __aeabi_l2f
    filters.o(.text.FilterRMSInt_Process) refers to filters.o(.text._sqrtf) for _sqrtf
    filters.o(.ARM.exidx.text.FilterRMSInt_Process) refers to filters.o(.text.FilterRMSInt_Process) for [Anonymous Symbol]
    filters.o(.text.FilterBandPassDerivative_Init) refers to sinf.o(i.__hardfp_sinf) for __hardfp_sinf
    filters.o(.text.FilterBandPassDerivative_Init) refers to cosf.o(i.__hardfp_cosf) for __hardfp_cosf
    filters.o(.text.FilterBandPassDerivative_Init) refers to filters.o(.text.FilterBandPassDerivative_Process) for FilterBandPassDerivative_Process
    filters.o(.ARM.exidx.text.FilterBandPassDerivative_Init) refers to filters.o(.text.FilterBandPassDerivative_Init) for [Anonymous Symbol]
    filters.o(.ARM.exidx.text.FilterBandPassDerivative_Process) refers to filters.o(.text.FilterBandPassDerivative_Process) for [Anonymous Symbol]
    system_k1921vk035.o(.text.SystemCoreClockUpdate) refers to system_k1921vk035.o(.bss.SystemCoreClock) for SystemCoreClock
    system_k1921vk035.o(.ARM.exidx.text.SystemCoreClockUpdate) refers to system_k1921vk035.o(.text.SystemCoreClockUpdate) for [Anonymous Symbol]
    system_k1921vk035.o(.ARM.exidx.text.ClkInit) refers to system_k1921vk035.o(.text.ClkInit) for [Anonymous Symbol]
    system_k1921vk035.o(.ARM.exidx.text.FPUInit) refers to system_k1921vk035.o(.text.FPUInit) for [Anonymous Symbol]
    system_k1921vk035.o(.text.SystemInit) refers to system_k1921vk035.o(.text.ClkInit) for ClkInit
    system_k1921vk035.o(.text.SystemInit) refers to system_k1921vk035.o(.text.FPUInit) for FPUInit
    system_k1921vk035.o(.ARM.exidx.text.SystemInit) refers to system_k1921vk035.o(.text.SystemInit) for [Anonymous Symbol]
    startup_k1921vk035.o(STACK) refers (Special) to heapauxi.o(.text) for __use_two_region_memory
    startup_k1921vk035.o(HEAP) refers (Special) to heapauxi.o(.text) for __use_two_region_memory
    startup_k1921vk035.o(RESET) refers (Special) to heapauxi.o(.text) for __use_two_region_memory
    startup_k1921vk035.o(RESET) refers to startup_k1921vk035.o(STACK) for __initial_sp
    startup_k1921vk035.o(RESET) refers to startup_k1921vk035.o(.text) for Reset_Handler
    startup_k1921vk035.o(RESET) refers to vk035_it.o(.text.NMI_Handler) for NMI_Handler
    startup_k1921vk035.o(RESET) refers to vk035_it.o(.text.HardFault_Handler) for HardFault_Handler
    startup_k1921vk035.o(RESET) refers to vk035_it.o(.text.MemManage_Handler) for MemManage_Handler
    startup_k1921vk035.o(RESET) refers to vk035_it.o(.text.BusFault_Handler) for BusFault_Handler
    startup_k1921vk035.o(RESET) refers to vk035_it.o(.text.UsageFault_Handler) for UsageFault_Handler
    startup_k1921vk035.o(RESET) refers to vk035_it.o(.text.SVC_Handler) for SVC_Handler
    startup_k1921vk035.o(RESET) refers to vk035_it.o(.text.DebugMon_Handler) for DebugMon_Handler
    startup_k1921vk035.o(RESET) refers to vk035_it.o(.text.PendSV_Handler) for PendSV_Handler
    startup_k1921vk035.o(RESET) refers to vk035_it.o(.text.SysTick_Handler) for SysTick_Handler
    startup_k1921vk035.o(RESET) refers to vk035_it.o(.text.WDT_IRQHandler) for WDT_IRQHandler
    startup_k1921vk035.o(RESET) refers to vk035_it.o(.text.RCU_IRQHandler) for RCU_IRQHandler
    startup_k1921vk035.o(RESET) refers to vk035_it.o(.text.MFLASH_IRQHandler) for MFLASH_IRQHandler
    startup_k1921vk035.o(RESET) refers to vk035_it.o(.text.GPIOA_IRQHandler) for GPIOA_IRQHandler
    startup_k1921vk035.o(RESET) refers to vk035_it.o(.text.GPIOB_IRQHandler) for GPIOB_IRQHandler
    startup_k1921vk035.o(RESET) refers to vk035_it.o(.text.DMA_CH0_IRQHandler) for DMA_CH0_IRQHandler
    startup_k1921vk035.o(RESET) refers to vk035_it.o(.text.DMA_CH1_IRQHandler) for DMA_CH1_IRQHandler
    startup_k1921vk035.o(RESET) refers to vk035_it.o(.text.DMA_CH2_IRQHandler) for DMA_CH2_IRQHandler
    startup_k1921vk035.o(RESET) refers to vk035_it.o(.text.DMA_CH3_IRQHandler) for DMA_CH3_IRQHandler
    startup_k1921vk035.o(RESET) refers to vk035_it.o(.text.DMA_CH4_IRQHandler) for DMA_CH4_IRQHandler
    startup_k1921vk035.o(RESET) refers to vk035_it.o(.text.DMA_CH5_IRQHandler) for DMA_CH5_IRQHandler
    startup_k1921vk035.o(RESET) refers to vk035_it.o(.text.DMA_CH6_IRQHandler) for DMA_CH6_IRQHandler
    startup_k1921vk035.o(RESET) refers to vk035_it.o(.text.DMA_CH7_IRQHandler) for DMA_CH7_IRQHandler
    startup_k1921vk035.o(RESET) refers to vk035_it.o(.text.DMA_CH8_IRQHandler) for DMA_CH8_IRQHandler
    startup_k1921vk035.o(RESET) refers to vk035_it.o(.text.DMA_CH9_IRQHandler) for DMA_CH9_IRQHandler
    startup_k1921vk035.o(RESET) refers to vk035_it.o(.text.DMA_CH10_IRQHandler) for DMA_CH10_IRQHandler
    startup_k1921vk035.o(RESET) refers to vk035_it.o(.text.DMA_CH11_IRQHandler) for DMA_CH11_IRQHandler
    startup_k1921vk035.o(RESET) refers to vk035_it.o(.text.DMA_CH12_IRQHandler) for DMA_CH12_IRQHandler
    startup_k1921vk035.o(RESET) refers to vk035_it.o(.text.DMA_CH13_IRQHandler) for DMA_CH13_IRQHandler
    startup_k1921vk035.o(RESET) refers to vk035_it.o(.text.DMA_CH14_IRQHandler) for DMA_CH14_IRQHandler
    startup_k1921vk035.o(RESET) refers to vk035_it.o(.text.DMA_CH15_IRQHandler) for DMA_CH15_IRQHandler
    startup_k1921vk035.o(RESET) refers to vk035_it.o(.text.TMR0_IRQHandler) for TMR0_IRQHandler
    startup_k1921vk035.o(RESET) refers to vk035_it.o(.text.TMR1_IRQHandler) for TMR1_IRQHandler
    startup_k1921vk035.o(RESET) refers to vk035_it.o(.text.TMR2_IRQHandler) for TMR2_IRQHandler
    startup_k1921vk035.o(RESET) refers to vk035_it.o(.text.TMR3_IRQHandler) for TMR3_IRQHandler
    startup_k1921vk035.o(RESET) refers to vk035_it.o(.text.UART0_TD_IRQHandler) for UART0_TD_IRQHandler
    startup_k1921vk035.o(RESET) refers to vk035_it.o(.text.UART0_RX_IRQHandler) for UART0_RX_IRQHandler
    startup_k1921vk035.o(RESET) refers to vk035_it.o(.text.UART0_TX_IRQHandler) for UART0_TX_IRQHandler
    startup_k1921vk035.o(RESET) refers to vk035_it.o(.text.UART0_E_RT_IRQHandler) for UART0_E_RT_IRQHandler
    startup_k1921vk035.o(RESET) refers to vk035_it.o(.text.UART1_TD_IRQHandler) for UART1_TD_IRQHandler
    startup_k1921vk035.o(RESET) refers to vk035_it.o(.text.UART1_RX_IRQHandler) for UART1_RX_IRQHandler
    startup_k1921vk035.o(RESET) refers to vk035_it.o(.text.UART1_TX_IRQHandler) for UART1_TX_IRQHandler
    startup_k1921vk035.o(RESET) refers to vk035_it.o(.text.UART1_E_RT_IRQHandler) for UART1_E_RT_IRQHandler
    startup_k1921vk035.o(RESET) refers to vk035_it.o(.text.SPI_RO_RT_IRQHandler) for SPI_RO_RT_IRQHandler
    startup_k1921vk035.o(RESET) refers to vk035_it.o(.text.SPI_RX_IRQHandler) for SPI_RX_IRQHandler
    startup_k1921vk035.o(RESET) refers to vk035_it.o(.text.SPI_TX_IRQHandler) for SPI_TX_IRQHandler
    startup_k1921vk035.o(RESET) refers to vk035_it.o(.text.I2C_IRQHandler) for I2C_IRQHandler
    startup_k1921vk035.o(RESET) refers to vk035_it.o(.text.ECAP0_IRQHandler) for ECAP0_IRQHandler
    startup_k1921vk035.o(RESET) refers to vk035_it.o(.text.ECAP1_IRQHandler) for ECAP1_IRQHandler
    startup_k1921vk035.o(RESET) refers to vk035_it.o(.text.ECAP2_IRQHandler) for ECAP2_IRQHandler
    startup_k1921vk035.o(RESET) refers to vk035_it.o(.text.PWM0_IRQHandler) for PWM0_IRQHandler
    startup_k1921vk035.o(RESET) refers to vk035_it.o(.text.PWM0_HD_IRQHandler) for PWM0_HD_IRQHandler
    startup_k1921vk035.o(RESET) refers to vk035_it.o(.text.PWM0_TZ_IRQHandler) for PWM0_TZ_IRQHandler
    startup_k1921vk035.o(RESET) refers to vk035_it.o(.text.PWM1_IRQHandler) for PWM1_IRQHandler
    startup_k1921vk035.o(RESET) refers to vk035_it.o(.text.PWM1_HD_IRQHandler) for PWM1_HD_IRQHandler
    startup_k1921vk035.o(RESET) refers to vk035_it.o(.text.PWM1_TZ_IRQHandler) for PWM1_TZ_IRQHandler
    startup_k1921vk035.o(RESET) refers to vk035_it.o(.text.PWM2_IRQHandler) for PWM2_IRQHandler
    startup_k1921vk035.o(RESET) refers to vk035_it.o(.text.PWM2_HD_IRQHandler) for PWM2_HD_IRQHandler
    startup_k1921vk035.o(RESET) refers to vk035_it.o(.text.PWM2_TZ_IRQHandler) for PWM2_TZ_IRQHandler
    startup_k1921vk035.o(RESET) refers to vk035_it.o(.text.QEP_IRQHandler) for QEP_IRQHandler
    startup_k1921vk035.o(RESET) refers to vk035_it.o(.text.ADC_SEQ0_IRQHandler) for ADC_SEQ0_IRQHandler
    startup_k1921vk035.o(RESET) refers to vk035_it.o(.text.ADC_SEQ1_IRQHandler) for ADC_SEQ1_IRQHandler
    startup_k1921vk035.o(RESET) refers to vk035_it.o(.text.ADC_DC_IRQHandler) for ADC_DC_IRQHandler
    startup_k1921vk035.o(RESET) refers to vk035_it.o(.text.CAN0_IRQHandler) for CAN0_IRQHandler
    startup_k1921vk035.o(RESET) refers to vk035_it.o(.text.CAN1_IRQHandler) for CAN1_IRQHandler
    startup_k1921vk035.o(RESET) refers to vk035_it.o(.text.CAN2_IRQHandler) for CAN2_IRQHandler
    startup_k1921vk035.o(RESET) refers to vk035_it.o(.text.CAN3_IRQHandler) for CAN3_IRQHandler
    startup_k1921vk035.o(RESET) refers to vk035_it.o(.text.CAN4_IRQHandler) for CAN4_IRQHandler
    startup_k1921vk035.o(RESET) refers to vk035_it.o(.text.CAN5_IRQHandler) for CAN5_IRQHandler
    startup_k1921vk035.o(RESET) refers to vk035_it.o(.text.CAN6_IRQHandler) for CAN6_IRQHandler
    startup_k1921vk035.o(RESET) refers to vk035_it.o(.text.CAN7_IRQHandler) for CAN7_IRQHandler
    startup_k1921vk035.o(RESET) refers to vk035_it.o(.text.CAN8_IRQHandler) for CAN8_IRQHandler
    startup_k1921vk035.o(RESET) refers to vk035_it.o(.text.CAN9_IRQHandler) for CAN9_IRQHandler
    startup_k1921vk035.o(RESET) refers to vk035_it.o(.text.CAN10_IRQHandler) for CAN10_IRQHandler
    startup_k1921vk035.o(RESET) refers to vk035_it.o(.text.CAN11_IRQHandler) for CAN11_IRQHandler
    startup_k1921vk035.o(RESET) refers to vk035_it.o(.text.CAN12_IRQHandler) for CAN12_IRQHandler
    startup_k1921vk035.o(RESET) refers to vk035_it.o(.text.CAN13_IRQHandler) for CAN13_IRQHandler
    startup_k1921vk035.o(RESET) refers to vk035_it.o(.text.CAN14_IRQHandler) for CAN14_IRQHandler
    startup_k1921vk035.o(RESET) refers to vk035_it.o(.text.CAN15_IRQHandler) for CAN15_IRQHandler
    startup_k1921vk035.o(RESET) refers to vk035_it.o(.text.FPU_IRQHandler) for FPU_IRQHandler
    startup_k1921vk035.o(.text) refers (Special) to heapauxi.o(.text) for __use_two_region_memory
    startup_k1921vk035.o(.text) refers to system_k1921vk035.o(.text.SystemInit) for SystemInit
    startup_k1921vk035.o(.text) refers to __main.o(!!!main) for __main
    startup_k1921vk035.o(.text) refers to startup_k1921vk035.o(HEAP) for Heap_Mem
    startup_k1921vk035.o(.text) refers to startup_k1921vk035.o(STACK) for Stack_Mem
    plib035_adc.o(.text.ADC_DeInit) refers to plib035_adc.o(.text.RCU_ADCRstCmd) for RCU_ADCRstCmd
    plib035_adc.o(.ARM.exidx.text.ADC_DeInit) refers to plib035_adc.o(.text.ADC_DeInit) for [Anonymous Symbol]
    plib035_adc.o(.ARM.exidx.text.RCU_ADCRstCmd) refers to plib035_adc.o(.text.RCU_ADCRstCmd) for [Anonymous Symbol]
    plib035_adc.o(.text.ADC_SEQ_Init) refers to plib035_adc.o(.text.ADC_SEQ_StartEventConfig) for ADC_SEQ_StartEventConfig
    plib035_adc.o(.text.ADC_SEQ_Init) refers to plib035_adc.o(.text.ADC_SEQ_SwStartEnCmd) for ADC_SEQ_SwStartEnCmd
    plib035_adc.o(.text.ADC_SEQ_Init) refers to plib035_adc.o(.text.ADC_SEQ_ReqConfig) for ADC_SEQ_ReqConfig
    plib035_adc.o(.text.ADC_SEQ_Init) refers to plib035_adc.o(.text.ADC_SEQ_ReqMaxConfig) for ADC_SEQ_ReqMaxConfig
    plib035_adc.o(.text.ADC_SEQ_Init) refers to plib035_adc.o(.text.ADC_SEQ_ReqAverageConfig) for ADC_SEQ_ReqAverageConfig
    plib035_adc.o(.text.ADC_SEQ_Init) refers to plib035_adc.o(.text.ADC_SEQ_ReqAverageCmd) for ADC_SEQ_ReqAverageCmd
    plib035_adc.o(.text.ADC_SEQ_Init) refers to plib035_adc.o(.text.ADC_SEQ_RestartConfig) for ADC_SEQ_RestartConfig
    plib035_adc.o(.text.ADC_SEQ_Init) refers to plib035_adc.o(.text.ADC_SEQ_RestartAverageCmd) for ADC_SEQ_RestartAverageCmd
    plib035_adc.o(.text.ADC_SEQ_Init) refers to plib035_adc.o(.text.ADC_SEQ_SetRestartTimer) for ADC_SEQ_SetRestartTimer
    plib035_adc.o(.text.ADC_SEQ_Init) refers to plib035_adc.o(.text.ADC_SEQ_DCEnableCmd) for ADC_SEQ_DCEnableCmd
    plib035_adc.o(.text.ADC_SEQ_Init) refers to plib035_adc.o(.text.ADC_SEQ_DMAConfig) for ADC_SEQ_DMAConfig
    plib035_adc.o(.text.ADC_SEQ_Init) refers to plib035_adc.o(.text.ADC_SEQ_DMACmd) for ADC_SEQ_DMACmd
    plib035_adc.o(.ARM.exidx.text.ADC_SEQ_Init) refers to plib035_adc.o(.text.ADC_SEQ_Init) for [Anonymous Symbol]
    plib035_adc.o(.ARM.exidx.text.ADC_SEQ_StartEventConfig) refers to plib035_adc.o(.text.ADC_SEQ_StartEventConfig) for [Anonymous Symbol]
    plib035_adc.o(.ARM.exidx.text.ADC_SEQ_SwStartEnCmd) refers to plib035_adc.o(.text.ADC_SEQ_SwStartEnCmd) for [Anonymous Symbol]
    plib035_adc.o(.ARM.exidx.text.ADC_SEQ_ReqConfig) refers to plib035_adc.o(.text.ADC_SEQ_ReqConfig) for [Anonymous Symbol]
    plib035_adc.o(.ARM.exidx.text.ADC_SEQ_ReqMaxConfig) refers to plib035_adc.o(.text.ADC_SEQ_ReqMaxConfig) for [Anonymous Symbol]
    plib035_adc.o(.ARM.exidx.text.ADC_SEQ_ReqAverageConfig) refers to plib035_adc.o(.text.ADC_SEQ_ReqAverageConfig) for [Anonymous Symbol]
    plib035_adc.o(.ARM.exidx.text.ADC_SEQ_ReqAverageCmd) refers to plib035_adc.o(.text.ADC_SEQ_ReqAverageCmd) for [Anonymous Symbol]
    plib035_adc.o(.ARM.exidx.text.ADC_SEQ_RestartConfig) refers to plib035_adc.o(.text.ADC_SEQ_RestartConfig) for [Anonymous Symbol]
    plib035_adc.o(.ARM.exidx.text.ADC_SEQ_RestartAverageCmd) refers to plib035_adc.o(.text.ADC_SEQ_RestartAverageCmd) for [Anonymous Symbol]
    plib035_adc.o(.ARM.exidx.text.ADC_SEQ_SetRestartTimer) refers to plib035_adc.o(.text.ADC_SEQ_SetRestartTimer) for [Anonymous Symbol]
    plib035_adc.o(.ARM.exidx.text.ADC_SEQ_DCEnableCmd) refers to plib035_adc.o(.text.ADC_SEQ_DCEnableCmd) for [Anonymous Symbol]
    plib035_adc.o(.ARM.exidx.text.ADC_SEQ_DMAConfig) refers to plib035_adc.o(.text.ADC_SEQ_DMAConfig) for [Anonymous Symbol]
    plib035_adc.o(.ARM.exidx.text.ADC_SEQ_DMACmd) refers to plib035_adc.o(.text.ADC_SEQ_DMACmd) for [Anonymous Symbol]
    plib035_adc.o(.ARM.exidx.text.ADC_SEQ_StructInit) refers to plib035_adc.o(.text.ADC_SEQ_StructInit) for [Anonymous Symbol]
    plib035_adc.o(.text.ADC_DC_Init) refers to plib035_adc.o(.text.ADC_DC_OutputCmd) for ADC_DC_OutputCmd
    plib035_adc.o(.text.ADC_DC_Init) refers to plib035_adc.o(.text.ADC_DC_SetThresholdLow) for ADC_DC_SetThresholdLow
    plib035_adc.o(.text.ADC_DC_Init) refers to plib035_adc.o(.text.ADC_DC_SetThresholdHigh) for ADC_DC_SetThresholdHigh
    plib035_adc.o(.text.ADC_DC_Init) refers to plib035_adc.o(.text.ADC_DC_SourceConfig) for ADC_DC_SourceConfig
    plib035_adc.o(.text.ADC_DC_Init) refers to plib035_adc.o(.text.ADC_DC_ChannelConfig) for ADC_DC_ChannelConfig
    plib035_adc.o(.text.ADC_DC_Init) refers to plib035_adc.o(.text.ADC_DC_Config) for ADC_DC_Config
    plib035_adc.o(.ARM.exidx.text.ADC_DC_Init) refers to plib035_adc.o(.text.ADC_DC_Init) for [Anonymous Symbol]
    plib035_adc.o(.ARM.exidx.text.ADC_DC_OutputCmd) refers to plib035_adc.o(.text.ADC_DC_OutputCmd) for [Anonymous Symbol]
    plib035_adc.o(.ARM.exidx.text.ADC_DC_SetThresholdLow) refers to plib035_adc.o(.text.ADC_DC_SetThresholdLow) for [Anonymous Symbol]
    plib035_adc.o(.ARM.exidx.text.ADC_DC_SetThresholdHigh) refers to plib035_adc.o(.text.ADC_DC_SetThresholdHigh) for [Anonymous Symbol]
    plib035_adc.o(.ARM.exidx.text.ADC_DC_SourceConfig) refers to plib035_adc.o(.text.ADC_DC_SourceConfig) for [Anonymous Symbol]
    plib035_adc.o(.ARM.exidx.text.ADC_DC_ChannelConfig) refers to plib035_adc.o(.text.ADC_DC_ChannelConfig) for [Anonymous Symbol]
    plib035_adc.o(.ARM.exidx.text.ADC_DC_Config) refers to plib035_adc.o(.text.ADC_DC_Config) for [Anonymous Symbol]
    plib035_adc.o(.ARM.exidx.text.ADC_DC_StructInit) refers to plib035_adc.o(.text.ADC_DC_StructInit) for [Anonymous Symbol]
    plib035_dma.o(.ARM.exidx.text.DMA_ChannelDeInit) refers to plib035_dma.o(.text.DMA_ChannelDeInit) for [Anonymous Symbol]
    plib035_dma.o(.ARM.exidx.text.DMA_ChannelInit) refers to plib035_dma.o(.text.DMA_ChannelInit) for [Anonymous Symbol]
    plib035_dma.o(.ARM.exidx.text.DMA_ChannelStructInit) refers to plib035_dma.o(.text.DMA_ChannelStructInit) for [Anonymous Symbol]
    plib035_dma.o(.ARM.exidx.text.DMA_DeInit) refers to plib035_dma.o(.text.DMA_DeInit) for [Anonymous Symbol]
    plib035_dma.o(.text.DMA_Init) refers to plib035_dma.o(.text.DMA_ProtectConfig) for DMA_ProtectConfig
    plib035_dma.o(.text.DMA_Init) refers to plib035_dma.o(.text.DMA_UseBurstCmd) for DMA_UseBurstCmd
    plib035_dma.o(.text.DMA_Init) refers to plib035_dma.o(.text.DMA_AltCtrlCmd) for DMA_AltCtrlCmd
    plib035_dma.o(.text.DMA_Init) refers to plib035_dma.o(.text.DMA_HighPriorityCmd) for DMA_HighPriorityCmd
    plib035_dma.o(.text.DMA_Init) refers to plib035_dma.o(.text.DMA_ReqMaskCmd) for DMA_ReqMaskCmd
    plib035_dma.o(.text.DMA_Init) refers to plib035_dma.o(.text.DMA_ChannelEnableCmd) for DMA_ChannelEnableCmd
    plib035_dma.o(.ARM.exidx.text.DMA_Init) refers to plib035_dma.o(.text.DMA_Init) for [Anonymous Symbol]
    plib035_dma.o(.ARM.exidx.text.DMA_ProtectConfig) refers to plib035_dma.o(.text.DMA_ProtectConfig) for [Anonymous Symbol]
    plib035_dma.o(.ARM.exidx.text.DMA_UseBurstCmd) refers to plib035_dma.o(.text.DMA_UseBurstCmd) for [Anonymous Symbol]
    plib035_dma.o(.ARM.exidx.text.DMA_AltCtrlCmd) refers to plib035_dma.o(.text.DMA_AltCtrlCmd) for [Anonymous Symbol]
    plib035_dma.o(.ARM.exidx.text.DMA_HighPriorityCmd) refers to plib035_dma.o(.text.DMA_HighPriorityCmd) for [Anonymous Symbol]
    plib035_dma.o(.ARM.exidx.text.DMA_ReqMaskCmd) refers to plib035_dma.o(.text.DMA_ReqMaskCmd) for [Anonymous Symbol]
    plib035_dma.o(.ARM.exidx.text.DMA_ChannelEnableCmd) refers to plib035_dma.o(.text.DMA_ChannelEnableCmd) for [Anonymous Symbol]
    plib035_dma.o(.ARM.exidx.text.DMA_StructInit) refers to plib035_dma.o(.text.DMA_StructInit) for [Anonymous Symbol]
    plib035_ecap.o(.text.ECAP_DeInit) refers to plib035_ecap.o(.text.RCU_APBRstCmd) for RCU_APBRstCmd
    plib035_ecap.o(.ARM.exidx.text.ECAP_DeInit) refers to plib035_ecap.o(.text.ECAP_DeInit) for [Anonymous Symbol]
    plib035_ecap.o(.ARM.exidx.text.RCU_APBRstCmd) refers to plib035_ecap.o(.text.RCU_APBRstCmd) for [Anonymous Symbol]
    plib035_ecap.o(.text.ECAP_Init) refers to plib035_ecap.o(.text.ECAP_HaltConfig) for ECAP_HaltConfig
    plib035_ecap.o(.text.ECAP_Init) refers to plib035_ecap.o(.text.ECAP_SyncOutConfig) for ECAP_SyncOutConfig
    plib035_ecap.o(.text.ECAP_Init) refers to plib035_ecap.o(.text.ECAP_SyncCmd) for ECAP_SyncCmd
    plib035_ecap.o(.text.ECAP_Init) refers to plib035_ecap.o(.text.ECAP_ModeConfig) for ECAP_ModeConfig
    plib035_ecap.o(.ARM.exidx.text.ECAP_Init) refers to plib035_ecap.o(.text.ECAP_Init) for [Anonymous Symbol]
    plib035_ecap.o(.ARM.exidx.text.ECAP_HaltConfig) refers to plib035_ecap.o(.text.ECAP_HaltConfig) for [Anonymous Symbol]
    plib035_ecap.o(.ARM.exidx.text.ECAP_SyncOutConfig) refers to plib035_ecap.o(.text.ECAP_SyncOutConfig) for [Anonymous Symbol]
    plib035_ecap.o(.ARM.exidx.text.ECAP_SyncCmd) refers to plib035_ecap.o(.text.ECAP_SyncCmd) for [Anonymous Symbol]
    plib035_ecap.o(.ARM.exidx.text.ECAP_ModeConfig) refers to plib035_ecap.o(.text.ECAP_ModeConfig) for [Anonymous Symbol]
    plib035_ecap.o(.ARM.exidx.text.ECAP_StructInit) refers to plib035_ecap.o(.text.ECAP_StructInit) for [Anonymous Symbol]
    plib035_ecap.o(.text.ECAP_PWM_Init) refers to plib035_ecap.o(.text.ECAP_PWM_SetPeriod) for ECAP_PWM_SetPeriod
    plib035_ecap.o(.text.ECAP_PWM_Init) refers to plib035_ecap.o(.text.ECAP_PWM_SetCompare) for ECAP_PWM_SetCompare
    plib035_ecap.o(.text.ECAP_PWM_Init) refers to plib035_ecap.o(.text.ECAP_PWM_PolarityConfig) for ECAP_PWM_PolarityConfig
    plib035_ecap.o(.ARM.exidx.text.ECAP_PWM_Init) refers to plib035_ecap.o(.text.ECAP_PWM_Init) for [Anonymous Symbol]
    plib035_ecap.o(.ARM.exidx.text.ECAP_PWM_SetPeriod) refers to plib035_ecap.o(.text.ECAP_PWM_SetPeriod) for [Anonymous Symbol]
    plib035_ecap.o(.ARM.exidx.text.ECAP_PWM_SetCompare) refers to plib035_ecap.o(.text.ECAP_PWM_SetCompare) for [Anonymous Symbol]
    plib035_ecap.o(.ARM.exidx.text.ECAP_PWM_PolarityConfig) refers to plib035_ecap.o(.text.ECAP_PWM_PolarityConfig) for [Anonymous Symbol]
    plib035_ecap.o(.ARM.exidx.text.ECAP_PWM_StructInit) refers to plib035_ecap.o(.text.ECAP_PWM_StructInit) for [Anonymous Symbol]
    plib035_ecap.o(.text.ECAP_Capture_Init) refers to plib035_ecap.o(.text.ECAP_Capture_ModeConfig) for ECAP_Capture_ModeConfig
    plib035_ecap.o(.text.ECAP_Capture_Init) refers to plib035_ecap.o(.text.ECAP_Capture_StopConfig) for ECAP_Capture_StopConfig
    plib035_ecap.o(.text.ECAP_Capture_Init) refers to plib035_ecap.o(.text.ECAP_Capture_PrescaleConfig) for ECAP_Capture_PrescaleConfig
    plib035_ecap.o(.text.ECAP_Capture_Init) refers to plib035_ecap.o(.text.ECAP_Capture_PolarityEvt0Config) for ECAP_Capture_PolarityEvt0Config
    plib035_ecap.o(.text.ECAP_Capture_Init) refers to plib035_ecap.o(.text.ECAP_Capture_PolarityEvt1Config) for ECAP_Capture_PolarityEvt1Config
    plib035_ecap.o(.text.ECAP_Capture_Init) refers to plib035_ecap.o(.text.ECAP_Capture_PolarityEvt2Config) for ECAP_Capture_PolarityEvt2Config
    plib035_ecap.o(.text.ECAP_Capture_Init) refers to plib035_ecap.o(.text.ECAP_Capture_PolarityEvt3Config) for ECAP_Capture_PolarityEvt3Config
    plib035_ecap.o(.text.ECAP_Capture_Init) refers to plib035_ecap.o(.text.ECAP_Capture_RstEvt0Cmd) for ECAP_Capture_RstEvt0Cmd
    plib035_ecap.o(.text.ECAP_Capture_Init) refers to plib035_ecap.o(.text.ECAP_Capture_RstEvt1Cmd) for ECAP_Capture_RstEvt1Cmd
    plib035_ecap.o(.text.ECAP_Capture_Init) refers to plib035_ecap.o(.text.ECAP_Capture_RstEvt2Cmd) for ECAP_Capture_RstEvt2Cmd
    plib035_ecap.o(.text.ECAP_Capture_Init) refers to plib035_ecap.o(.text.ECAP_Capture_RstEvt3Cmd) for ECAP_Capture_RstEvt3Cmd
    plib035_ecap.o(.ARM.exidx.text.ECAP_Capture_Init) refers to plib035_ecap.o(.text.ECAP_Capture_Init) for [Anonymous Symbol]
    plib035_ecap.o(.ARM.exidx.text.ECAP_Capture_ModeConfig) refers to plib035_ecap.o(.text.ECAP_Capture_ModeConfig) for [Anonymous Symbol]
    plib035_ecap.o(.ARM.exidx.text.ECAP_Capture_StopConfig) refers to plib035_ecap.o(.text.ECAP_Capture_StopConfig) for [Anonymous Symbol]
    plib035_ecap.o(.ARM.exidx.text.ECAP_Capture_PrescaleConfig) refers to plib035_ecap.o(.text.ECAP_Capture_PrescaleConfig) for [Anonymous Symbol]
    plib035_ecap.o(.ARM.exidx.text.ECAP_Capture_PolarityEvt0Config) refers to plib035_ecap.o(.text.ECAP_Capture_PolarityEvt0Config) for [Anonymous Symbol]
    plib035_ecap.o(.ARM.exidx.text.ECAP_Capture_PolarityEvt1Config) refers to plib035_ecap.o(.text.ECAP_Capture_PolarityEvt1Config) for [Anonymous Symbol]
    plib035_ecap.o(.ARM.exidx.text.ECAP_Capture_PolarityEvt2Config) refers to plib035_ecap.o(.text.ECAP_Capture_PolarityEvt2Config) for [Anonymous Symbol]
    plib035_ecap.o(.ARM.exidx.text.ECAP_Capture_PolarityEvt3Config) refers to plib035_ecap.o(.text.ECAP_Capture_PolarityEvt3Config) for [Anonymous Symbol]
    plib035_ecap.o(.ARM.exidx.text.ECAP_Capture_RstEvt0Cmd) refers to plib035_ecap.o(.text.ECAP_Capture_RstEvt0Cmd) for [Anonymous Symbol]
    plib035_ecap.o(.ARM.exidx.text.ECAP_Capture_RstEvt1Cmd) refers to plib035_ecap.o(.text.ECAP_Capture_RstEvt1Cmd) for [Anonymous Symbol]
    plib035_ecap.o(.ARM.exidx.text.ECAP_Capture_RstEvt2Cmd) refers to plib035_ecap.o(.text.ECAP_Capture_RstEvt2Cmd) for [Anonymous Symbol]
    plib035_ecap.o(.ARM.exidx.text.ECAP_Capture_RstEvt3Cmd) refers to plib035_ecap.o(.text.ECAP_Capture_RstEvt3Cmd) for [Anonymous Symbol]
    plib035_ecap.o(.ARM.exidx.text.ECAP_Capture_StructInit) refers to plib035_ecap.o(.text.ECAP_Capture_StructInit) for [Anonymous Symbol]
    plib035_gpio.o(.text.GPIO_OutModeConfig) refers to plib035_gpio.o(.text.GPIO_ModeConfig) for GPIO_ModeConfig
    plib035_gpio.o(.ARM.exidx.text.GPIO_OutModeConfig) refers to plib035_gpio.o(.text.GPIO_OutModeConfig) for [Anonymous Symbol]
    plib035_gpio.o(.ARM.exidx.text.GPIO_ModeConfig) refers to plib035_gpio.o(.text.GPIO_ModeConfig) for [Anonymous Symbol]
    plib035_gpio.o(.text.GPIO_InModeConfig) refers to plib035_gpio.o(.text.GPIO_ModeConfig) for GPIO_ModeConfig
    plib035_gpio.o(.ARM.exidx.text.GPIO_InModeConfig) refers to plib035_gpio.o(.text.GPIO_InModeConfig) for [Anonymous Symbol]
    plib035_gpio.o(.text.GPIO_PullModeConfig) refers to plib035_gpio.o(.text.GPIO_ModeConfig) for GPIO_ModeConfig
    plib035_gpio.o(.ARM.exidx.text.GPIO_PullModeConfig) refers to plib035_gpio.o(.text.GPIO_PullModeConfig) for [Anonymous Symbol]
    plib035_gpio.o(.text.GPIO_DriveModeConfig) refers to plib035_gpio.o(.text.GPIO_ModeConfig) for GPIO_ModeConfig
    plib035_gpio.o(.ARM.exidx.text.GPIO_DriveModeConfig) refers to plib035_gpio.o(.text.GPIO_DriveModeConfig) for [Anonymous Symbol]
    plib035_gpio.o(.text.GPIO_DeInit) refers to plib035_gpio.o(.text.RCU_AHBRstCmd) for RCU_AHBRstCmd
    plib035_gpio.o(.ARM.exidx.text.GPIO_DeInit) refers to plib035_gpio.o(.text.GPIO_DeInit) for [Anonymous Symbol]
    plib035_gpio.o(.ARM.exidx.text.RCU_AHBRstCmd) refers to plib035_gpio.o(.text.RCU_AHBRstCmd) for [Anonymous Symbol]
    plib035_gpio.o(.text.GPIO_Init) refers to plib035_gpio.o(.text.GPIO_OutCmd) for GPIO_OutCmd
    plib035_gpio.o(.text.GPIO_Init) refers to plib035_gpio.o(.text.GPIO_AltFuncCmd) for GPIO_AltFuncCmd
    plib035_gpio.o(.text.GPIO_Init) refers to plib035_gpio.o(.text.GPIO_OutModeConfig) for GPIO_OutModeConfig
    plib035_gpio.o(.text.GPIO_Init) refers to plib035_gpio.o(.text.GPIO_InModeConfig) for GPIO_InModeConfig
    plib035_gpio.o(.text.GPIO_Init) refers to plib035_gpio.o(.text.GPIO_PullModeConfig) for GPIO_PullModeConfig
    plib035_gpio.o(.text.GPIO_Init) refers to plib035_gpio.o(.text.GPIO_DriveModeConfig) for GPIO_DriveModeConfig
    plib035_gpio.o(.text.GPIO_Init) refers to plib035_gpio.o(.text.GPIO_DigitalCmd) for GPIO_DigitalCmd
    plib035_gpio.o(.ARM.exidx.text.GPIO_Init) refers to plib035_gpio.o(.text.GPIO_Init) for [Anonymous Symbol]
    plib035_gpio.o(.ARM.exidx.text.GPIO_OutCmd) refers to plib035_gpio.o(.text.GPIO_OutCmd) for [Anonymous Symbol]
    plib035_gpio.o(.ARM.exidx.text.GPIO_AltFuncCmd) refers to plib035_gpio.o(.text.GPIO_AltFuncCmd) for [Anonymous Symbol]
    plib035_gpio.o(.ARM.exidx.text.GPIO_DigitalCmd) refers to plib035_gpio.o(.text.GPIO_DigitalCmd) for [Anonymous Symbol]
    plib035_gpio.o(.ARM.exidx.text.GPIO_StructInit) refers to plib035_gpio.o(.text.GPIO_StructInit) for [Anonymous Symbol]
    plib035_i2c.o(.text.I2C_FSFreqConfig) refers to plib035_i2c.o(.text.I2C_FSDivLowConfig) for I2C_FSDivLowConfig
    plib035_i2c.o(.text.I2C_FSFreqConfig) refers to plib035_i2c.o(.text.I2C_FSDivHighConfig) for I2C_FSDivHighConfig
    plib035_i2c.o(.ARM.exidx.text.I2C_FSFreqConfig) refers to plib035_i2c.o(.text.I2C_FSFreqConfig) for [Anonymous Symbol]
    plib035_i2c.o(.ARM.exidx.text.I2C_FSDivLowConfig) refers to plib035_i2c.o(.text.I2C_FSDivLowConfig) for [Anonymous Symbol]
    plib035_i2c.o(.ARM.exidx.text.I2C_FSDivHighConfig) refers to plib035_i2c.o(.text.I2C_FSDivHighConfig) for [Anonymous Symbol]
    plib035_i2c.o(.text.I2C_HSFreqConfig) refers to plib035_i2c.o(.text.I2C_HSDivLowConfig) for I2C_HSDivLowConfig
    plib035_i2c.o(.text.I2C_HSFreqConfig) refers to plib035_i2c.o(.text.I2C_HSDivHighConfig) for I2C_HSDivHighConfig
    plib035_i2c.o(.ARM.exidx.text.I2C_HSFreqConfig) refers to plib035_i2c.o(.text.I2C_HSFreqConfig) for [Anonymous Symbol]
    plib035_i2c.o(.ARM.exidx.text.I2C_HSDivLowConfig) refers to plib035_i2c.o(.text.I2C_HSDivLowConfig) for [Anonymous Symbol]
    plib035_i2c.o(.ARM.exidx.text.I2C_HSDivHighConfig) refers to plib035_i2c.o(.text.I2C_HSDivHighConfig) for [Anonymous Symbol]
    plib035_mflash.o(.text.MFLASH_ReadData) refers to plib035_mflash.o(.text.MFLASH_SetAddr) for MFLASH_SetAddr
    plib035_mflash.o(.text.MFLASH_ReadData) refers to plib035_mflash.o(.text.MFLASH_SetCmd) for MFLASH_SetCmd
    plib035_mflash.o(.text.MFLASH_ReadData) refers to plib035_mflash.o(.text.MFLASH_BusyStatus) for MFLASH_BusyStatus
    plib035_mflash.o(.text.MFLASH_ReadData) refers to plib035_mflash.o(.text.MFLASH_GetData) for MFLASH_GetData
    plib035_mflash.o(.ARM.exidx.text.MFLASH_ReadData) refers to plib035_mflash.o(.text.MFLASH_ReadData) for [Anonymous Symbol]
    plib035_mflash.o(.ARM.exidx.text.MFLASH_SetAddr) refers to plib035_mflash.o(.text.MFLASH_SetAddr) for [Anonymous Symbol]
    plib035_mflash.o(.ARM.exidx.text.MFLASH_SetCmd) refers to plib035_mflash.o(.text.MFLASH_SetCmd) for [Anonymous Symbol]
    plib035_mflash.o(.ARM.exidx.text.MFLASH_BusyStatus) refers to plib035_mflash.o(.text.MFLASH_BusyStatus) for [Anonymous Symbol]
    plib035_mflash.o(.ARM.exidx.text.MFLASH_GetData) refers to plib035_mflash.o(.text.MFLASH_GetData) for [Anonymous Symbol]
    plib035_mflash.o(.text.MFLASH_WriteData) refers to plib035_mflash.o(.text.MFLASH_SetAddr) for MFLASH_SetAddr
    plib035_mflash.o(.text.MFLASH_WriteData) refers to plib035_mflash.o(.text.MFLASH_SetData) for MFLASH_SetData
    plib035_mflash.o(.text.MFLASH_WriteData) refers to plib035_mflash.o(.text.MFLASH_SetCmd) for MFLASH_SetCmd
    plib035_mflash.o(.text.MFLASH_WriteData) refers to plib035_mflash.o(.text.MFLASH_BusyStatus) for MFLASH_BusyStatus
    plib035_mflash.o(.ARM.exidx.text.MFLASH_WriteData) refers to plib035_mflash.o(.text.MFLASH_WriteData) for [Anonymous Symbol]
    plib035_mflash.o(.ARM.exidx.text.MFLASH_SetData) refers to plib035_mflash.o(.text.MFLASH_SetData) for [Anonymous Symbol]
    plib035_mflash.o(.text.MFLASH_ErasePage) refers to plib035_mflash.o(.text.MFLASH_SetAddr) for MFLASH_SetAddr
    plib035_mflash.o(.text.MFLASH_ErasePage) refers to plib035_mflash.o(.text.MFLASH_SetCmd) for MFLASH_SetCmd
    plib035_mflash.o(.text.MFLASH_ErasePage) refers to plib035_mflash.o(.text.MFLASH_BusyStatus) for MFLASH_BusyStatus
    plib035_mflash.o(.ARM.exidx.text.MFLASH_ErasePage) refers to plib035_mflash.o(.text.MFLASH_ErasePage) for [Anonymous Symbol]
    plib035_mflash.o(.text.MFLASH_EraseFull) refers to plib035_mflash.o(.text.MFLASH_SetCmd) for MFLASH_SetCmd
    plib035_mflash.o(.text.MFLASH_EraseFull) refers to plib035_mflash.o(.text.MFLASH_BusyStatus) for MFLASH_BusyStatus
    plib035_mflash.o(.ARM.exidx.text.MFLASH_EraseFull) refers to plib035_mflash.o(.text.MFLASH_EraseFull) for [Anonymous Symbol]
    plib035_pwm.o(.text.PWM_DeInit) refers to plib035_pwm.o(.text.RCU_APBRstCmd) for RCU_APBRstCmd
    plib035_pwm.o(.ARM.exidx.text.PWM_DeInit) refers to plib035_pwm.o(.text.PWM_DeInit) for [Anonymous Symbol]
    plib035_pwm.o(.ARM.exidx.text.RCU_APBRstCmd) refers to plib035_pwm.o(.text.RCU_APBRstCmd) for [Anonymous Symbol]
    plib035_pwm.o(.text.PWM_TB_Init) refers to plib035_pwm.o(.text.PWM_TB_HaltConfig) for PWM_TB_HaltConfig
    plib035_pwm.o(.text.PWM_TB_Init) refers to plib035_pwm.o(.text.PWM_TB_PhaseSyncCmd) for PWM_TB_PhaseSyncCmd
    plib035_pwm.o(.text.PWM_TB_Init) refers to plib035_pwm.o(.text.PWM_TB_PhaseSyncDirConfig) for PWM_TB_PhaseSyncDirConfig
    plib035_pwm.o(.text.PWM_TB_Init) refers to plib035_pwm.o(.text.PWM_TB_ClkDivConfig) for PWM_TB_ClkDivConfig
    plib035_pwm.o(.text.PWM_TB_Init) refers to plib035_pwm.o(.text.PWM_TB_SyncOutConfig) for PWM_TB_SyncOutConfig
    plib035_pwm.o(.text.PWM_TB_Init) refers to plib035_pwm.o(.text.PWM_TB_PeriodDirectLoadCmd) for PWM_TB_PeriodDirectLoadCmd
    plib035_pwm.o(.text.PWM_TB_Init) refers to plib035_pwm.o(.text.PWM_TB_ModeConfig) for PWM_TB_ModeConfig
    plib035_pwm.o(.text.PWM_TB_Init) refers to plib035_pwm.o(.text.PWM_TB_SetPhase) for PWM_TB_SetPhase
    plib035_pwm.o(.text.PWM_TB_Init) refers to plib035_pwm.o(.text.PWM_TB_SetPeriod) for PWM_TB_SetPeriod
    plib035_pwm.o(.ARM.exidx.text.PWM_TB_Init) refers to plib035_pwm.o(.text.PWM_TB_Init) for [Anonymous Symbol]
    plib035_pwm.o(.ARM.exidx.text.PWM_TB_HaltConfig) refers to plib035_pwm.o(.text.PWM_TB_HaltConfig) for [Anonymous Symbol]
    plib035_pwm.o(.ARM.exidx.text.PWM_TB_PhaseSyncCmd) refers to plib035_pwm.o(.text.PWM_TB_PhaseSyncCmd) for [Anonymous Symbol]
    plib035_pwm.o(.ARM.exidx.text.PWM_TB_PhaseSyncDirConfig) refers to plib035_pwm.o(.text.PWM_TB_PhaseSyncDirConfig) for [Anonymous Symbol]
    plib035_pwm.o(.ARM.exidx.text.PWM_TB_ClkDivConfig) refers to plib035_pwm.o(.text.PWM_TB_ClkDivConfig) for [Anonymous Symbol]
    plib035_pwm.o(.ARM.exidx.text.PWM_TB_SyncOutConfig) refers to plib035_pwm.o(.text.PWM_TB_SyncOutConfig) for [Anonymous Symbol]
    plib035_pwm.o(.ARM.exidx.text.PWM_TB_PeriodDirectLoadCmd) refers to plib035_pwm.o(.text.PWM_TB_PeriodDirectLoadCmd) for [Anonymous Symbol]
    plib035_pwm.o(.ARM.exidx.text.PWM_TB_ModeConfig) refers to plib035_pwm.o(.text.PWM_TB_ModeConfig) for [Anonymous Symbol]
    plib035_pwm.o(.ARM.exidx.text.PWM_TB_SetPhase) refers to plib035_pwm.o(.text.PWM_TB_SetPhase) for [Anonymous Symbol]
    plib035_pwm.o(.ARM.exidx.text.PWM_TB_SetPeriod) refers to plib035_pwm.o(.text.PWM_TB_SetPeriod) for [Anonymous Symbol]
    plib035_pwm.o(.ARM.exidx.text.PWM_TB_StructInit) refers to plib035_pwm.o(.text.PWM_TB_StructInit) for [Anonymous Symbol]
    plib035_pwm.o(.text.PWM_AQ_Init) refers to plib035_pwm.o(.text.PWM_AQ_ActionAConfig) for PWM_AQ_ActionAConfig
    plib035_pwm.o(.text.PWM_AQ_Init) refers to plib035_pwm.o(.text.PWM_AQ_ActionBConfig) for PWM_AQ_ActionBConfig
    plib035_pwm.o(.ARM.exidx.text.PWM_AQ_Init) refers to plib035_pwm.o(.text.PWM_AQ_Init) for [Anonymous Symbol]
    plib035_pwm.o(.ARM.exidx.text.PWM_AQ_ActionAConfig) refers to plib035_pwm.o(.text.PWM_AQ_ActionAConfig) for [Anonymous Symbol]
    plib035_pwm.o(.ARM.exidx.text.PWM_AQ_ActionBConfig) refers to plib035_pwm.o(.text.PWM_AQ_ActionBConfig) for [Anonymous Symbol]
    plib035_pwm.o(.ARM.exidx.text.PWM_AQ_StructInit) refers to plib035_pwm.o(.text.PWM_AQ_StructInit) for [Anonymous Symbol]
    plib035_pwm.o(.text.PWM_CMP_Init) refers to plib035_pwm.o(.text.PWM_CMP_CmpALoadEventConfig) for PWM_CMP_CmpALoadEventConfig
    plib035_pwm.o(.text.PWM_CMP_Init) refers to plib035_pwm.o(.text.PWM_CMP_CmpADirectLoadCmd) for PWM_CMP_CmpADirectLoadCmd
    plib035_pwm.o(.text.PWM_CMP_Init) refers to plib035_pwm.o(.text.PWM_CMP_SetCmpA) for PWM_CMP_SetCmpA
    plib035_pwm.o(.text.PWM_CMP_Init) refers to plib035_pwm.o(.text.PWM_CMP_SetCmpB) for PWM_CMP_SetCmpB
    plib035_pwm.o(.ARM.exidx.text.PWM_CMP_Init) refers to plib035_pwm.o(.text.PWM_CMP_Init) for [Anonymous Symbol]
    plib035_pwm.o(.ARM.exidx.text.PWM_CMP_CmpALoadEventConfig) refers to plib035_pwm.o(.text.PWM_CMP_CmpALoadEventConfig) for [Anonymous Symbol]
    plib035_pwm.o(.ARM.exidx.text.PWM_CMP_CmpADirectLoadCmd) refers to plib035_pwm.o(.text.PWM_CMP_CmpADirectLoadCmd) for [Anonymous Symbol]
    plib035_pwm.o(.ARM.exidx.text.PWM_CMP_SetCmpA) refers to plib035_pwm.o(.text.PWM_CMP_SetCmpA) for [Anonymous Symbol]
    plib035_pwm.o(.ARM.exidx.text.PWM_CMP_SetCmpB) refers to plib035_pwm.o(.text.PWM_CMP_SetCmpB) for [Anonymous Symbol]
    plib035_pwm.o(.ARM.exidx.text.PWM_CMP_StructInit) refers to plib035_pwm.o(.text.PWM_CMP_StructInit) for [Anonymous Symbol]
    plib035_pwm.o(.text.PWM_HD_Init) refers to plib035_pwm.o(.text.PWM_HD_ActionAConfig) for PWM_HD_ActionAConfig
    plib035_pwm.o(.text.PWM_HD_Init) refers to plib035_pwm.o(.text.PWM_HD_ActionBConfig) for PWM_HD_ActionBConfig
    plib035_pwm.o(.text.PWM_HD_Init) refers to plib035_pwm.o(.text.PWM_HD_SourceCmd) for PWM_HD_SourceCmd
    plib035_pwm.o(.text.PWM_HD_Init) refers to plib035_pwm.o(.text.PWM_HD_CycleCmd) for PWM_HD_CycleCmd
    plib035_pwm.o(.text.PWM_HD_Init) refers to plib035_pwm.o(.text.PWM_HD_OneShotCmd) for PWM_HD_OneShotCmd
    plib035_pwm.o(.ARM.exidx.text.PWM_HD_Init) refers to plib035_pwm.o(.text.PWM_HD_Init) for [Anonymous Symbol]
    plib035_pwm.o(.ARM.exidx.text.PWM_HD_ActionAConfig) refers to plib035_pwm.o(.text.PWM_HD_ActionAConfig) for [Anonymous Symbol]
    plib035_pwm.o(.ARM.exidx.text.PWM_HD_ActionBConfig) refers to plib035_pwm.o(.text.PWM_HD_ActionBConfig) for [Anonymous Symbol]
    plib035_pwm.o(.ARM.exidx.text.PWM_HD_SourceCmd) refers to plib035_pwm.o(.text.PWM_HD_SourceCmd) for [Anonymous Symbol]
    plib035_pwm.o(.ARM.exidx.text.PWM_HD_CycleCmd) refers to plib035_pwm.o(.text.PWM_HD_CycleCmd) for [Anonymous Symbol]
    plib035_pwm.o(.ARM.exidx.text.PWM_HD_OneShotCmd) refers to plib035_pwm.o(.text.PWM_HD_OneShotCmd) for [Anonymous Symbol]
    plib035_pwm.o(.ARM.exidx.text.PWM_HD_StructInit) refers to plib035_pwm.o(.text.PWM_HD_StructInit) for [Anonymous Symbol]
    plib035_pwm.o(.text.PWM_DB_Init) refers to plib035_pwm.o(.text.PWM_DB_InConfig) for PWM_DB_InConfig
    plib035_pwm.o(.text.PWM_DB_Init) refers to plib035_pwm.o(.text.PWM_DB_OutConfig) for PWM_DB_OutConfig
    plib035_pwm.o(.text.PWM_DB_Init) refers to plib035_pwm.o(.text.PWM_DB_PolarityConfig) for PWM_DB_PolarityConfig
    plib035_pwm.o(.text.PWM_DB_Init) refers to plib035_pwm.o(.text.PWM_DB_SetRiseDelay) for PWM_DB_SetRiseDelay
    plib035_pwm.o(.text.PWM_DB_Init) refers to plib035_pwm.o(.text.PWM_DB_SetFallDelay) for PWM_DB_SetFallDelay
    plib035_pwm.o(.ARM.exidx.text.PWM_DB_Init) refers to plib035_pwm.o(.text.PWM_DB_Init) for [Anonymous Symbol]
    plib035_pwm.o(.ARM.exidx.text.PWM_DB_InConfig) refers to plib035_pwm.o(.text.PWM_DB_InConfig) for [Anonymous Symbol]
    plib035_pwm.o(.ARM.exidx.text.PWM_DB_OutConfig) refers to plib035_pwm.o(.text.PWM_DB_OutConfig) for [Anonymous Symbol]
    plib035_pwm.o(.ARM.exidx.text.PWM_DB_PolarityConfig) refers to plib035_pwm.o(.text.PWM_DB_PolarityConfig) for [Anonymous Symbol]
    plib035_pwm.o(.ARM.exidx.text.PWM_DB_SetRiseDelay) refers to plib035_pwm.o(.text.PWM_DB_SetRiseDelay) for [Anonymous Symbol]
    plib035_pwm.o(.ARM.exidx.text.PWM_DB_SetFallDelay) refers to plib035_pwm.o(.text.PWM_DB_SetFallDelay) for [Anonymous Symbol]
    plib035_pwm.o(.ARM.exidx.text.PWM_DB_StructInit) refers to plib035_pwm.o(.text.PWM_DB_StructInit) for [Anonymous Symbol]
    plib035_pwm.o(.text.PWM_TZ_Init) refers to plib035_pwm.o(.text.PWM_TZ_ActionAConfig) for PWM_TZ_ActionAConfig
    plib035_pwm.o(.text.PWM_TZ_Init) refers to plib035_pwm.o(.text.PWM_TZ_ActionBConfig) for PWM_TZ_ActionBConfig
    plib035_pwm.o(.text.PWM_TZ_Init) refers to plib035_pwm.o(.text.PWM_TZ_CycleCmd) for PWM_TZ_CycleCmd
    plib035_pwm.o(.text.PWM_TZ_Init) refers to plib035_pwm.o(.text.PWM_TZ_OneShotCmd) for PWM_TZ_OneShotCmd
    plib035_pwm.o(.ARM.exidx.text.PWM_TZ_Init) refers to plib035_pwm.o(.text.PWM_TZ_Init) for [Anonymous Symbol]
    plib035_pwm.o(.ARM.exidx.text.PWM_TZ_ActionAConfig) refers to plib035_pwm.o(.text.PWM_TZ_ActionAConfig) for [Anonymous Symbol]
    plib035_pwm.o(.ARM.exidx.text.PWM_TZ_ActionBConfig) refers to plib035_pwm.o(.text.PWM_TZ_ActionBConfig) for [Anonymous Symbol]
    plib035_pwm.o(.ARM.exidx.text.PWM_TZ_CycleCmd) refers to plib035_pwm.o(.text.PWM_TZ_CycleCmd) for [Anonymous Symbol]
    plib035_pwm.o(.ARM.exidx.text.PWM_TZ_OneShotCmd) refers to plib035_pwm.o(.text.PWM_TZ_OneShotCmd) for [Anonymous Symbol]
    plib035_pwm.o(.ARM.exidx.text.PWM_TZ_StructInit) refers to plib035_pwm.o(.text.PWM_TZ_StructInit) for [Anonymous Symbol]
    plib035_pwm.o(.text.PWM_ET_Init) refers to plib035_pwm.o(.text.PWM_ET_SOCAEventConfig) for PWM_ET_SOCAEventConfig
    plib035_pwm.o(.text.PWM_ET_Init) refers to plib035_pwm.o(.text.PWM_ET_SOCAPeriodConfig) for PWM_ET_SOCAPeriodConfig
    plib035_pwm.o(.text.PWM_ET_Init) refers to plib035_pwm.o(.text.PWM_ET_SOCACmd) for PWM_ET_SOCACmd
    plib035_pwm.o(.text.PWM_ET_Init) refers to plib035_pwm.o(.text.PWM_ET_SOCBEventConfig) for PWM_ET_SOCBEventConfig
    plib035_pwm.o(.text.PWM_ET_Init) refers to plib035_pwm.o(.text.PWM_ET_SOCBPeriodConfig) for PWM_ET_SOCBPeriodConfig
    plib035_pwm.o(.text.PWM_ET_Init) refers to plib035_pwm.o(.text.PWM_ET_SOCBCmd) for PWM_ET_SOCBCmd
    plib035_pwm.o(.text.PWM_ET_Init) refers to plib035_pwm.o(.text.PWM_ET_DRQAEventConfig) for PWM_ET_DRQAEventConfig
    plib035_pwm.o(.text.PWM_ET_Init) refers to plib035_pwm.o(.text.PWM_ET_DRQAPeriodConfig) for PWM_ET_DRQAPeriodConfig
    plib035_pwm.o(.text.PWM_ET_Init) refers to plib035_pwm.o(.text.PWM_ET_DRQACmd) for PWM_ET_DRQACmd
    plib035_pwm.o(.text.PWM_ET_Init) refers to plib035_pwm.o(.text.PWM_ET_DRQBEventConfig) for PWM_ET_DRQBEventConfig
    plib035_pwm.o(.text.PWM_ET_Init) refers to plib035_pwm.o(.text.PWM_ET_DRQBPeriodConfig) for PWM_ET_DRQBPeriodConfig
    plib035_pwm.o(.text.PWM_ET_Init) refers to plib035_pwm.o(.text.PWM_ET_DRQBCmd) for PWM_ET_DRQBCmd
    plib035_pwm.o(.ARM.exidx.text.PWM_ET_Init) refers to plib035_pwm.o(.text.PWM_ET_Init) for [Anonymous Symbol]
    plib035_pwm.o(.ARM.exidx.text.PWM_ET_SOCAEventConfig) refers to plib035_pwm.o(.text.PWM_ET_SOCAEventConfig) for [Anonymous Symbol]
    plib035_pwm.o(.ARM.exidx.text.PWM_ET_SOCAPeriodConfig) refers to plib035_pwm.o(.text.PWM_ET_SOCAPeriodConfig) for [Anonymous Symbol]
    plib035_pwm.o(.ARM.exidx.text.PWM_ET_SOCACmd) refers to plib035_pwm.o(.text.PWM_ET_SOCACmd) for [Anonymous Symbol]
    plib035_pwm.o(.ARM.exidx.text.PWM_ET_SOCBEventConfig) refers to plib035_pwm.o(.text.PWM_ET_SOCBEventConfig) for [Anonymous Symbol]
    plib035_pwm.o(.ARM.exidx.text.PWM_ET_SOCBPeriodConfig) refers to plib035_pwm.o(.text.PWM_ET_SOCBPeriodConfig) for [Anonymous Symbol]
    plib035_pwm.o(.ARM.exidx.text.PWM_ET_SOCBCmd) refers to plib035_pwm.o(.text.PWM_ET_SOCBCmd) for [Anonymous Symbol]
    plib035_pwm.o(.ARM.exidx.text.PWM_ET_DRQAEventConfig) refers to plib035_pwm.o(.text.PWM_ET_DRQAEventConfig) for [Anonymous Symbol]
    plib035_pwm.o(.ARM.exidx.text.PWM_ET_DRQAPeriodConfig) refers to plib035_pwm.o(.text.PWM_ET_DRQAPeriodConfig) for [Anonymous Symbol]
    plib035_pwm.o(.ARM.exidx.text.PWM_ET_DRQACmd) refers to plib035_pwm.o(.text.PWM_ET_DRQACmd) for [Anonymous Symbol]
    plib035_pwm.o(.ARM.exidx.text.PWM_ET_DRQBEventConfig) refers to plib035_pwm.o(.text.PWM_ET_DRQBEventConfig) for [Anonymous Symbol]
    plib035_pwm.o(.ARM.exidx.text.PWM_ET_DRQBPeriodConfig) refers to plib035_pwm.o(.text.PWM_ET_DRQBPeriodConfig) for [Anonymous Symbol]
    plib035_pwm.o(.ARM.exidx.text.PWM_ET_DRQBCmd) refers to plib035_pwm.o(.text.PWM_ET_DRQBCmd) for [Anonymous Symbol]
    plib035_pwm.o(.ARM.exidx.text.PWM_ET_StructInit) refers to plib035_pwm.o(.text.PWM_ET_StructInit) for [Anonymous Symbol]
    plib035_qep.o(.text.QEP_DeInit) refers to plib035_qep.o(.text.RCU_APBRstCmd) for RCU_APBRstCmd
    plib035_qep.o(.ARM.exidx.text.QEP_DeInit) refers to plib035_qep.o(.text.QEP_DeInit) for [Anonymous Symbol]
    plib035_qep.o(.ARM.exidx.text.RCU_APBRstCmd) refers to plib035_qep.o(.text.RCU_APBRstCmd) for [Anonymous Symbol]
    plib035_qep.o(.text.QEP_PC_Init) refers to plib035_qep.o(.text.QEP_PC_ModeConfig) for QEP_PC_ModeConfig
    plib035_qep.o(.text.QEP_PC_Init) refers to plib035_qep.o(.text.QEP_PC_CountRateConfig) for QEP_PC_CountRateConfig
    plib035_qep.o(.text.QEP_PC_Init) refers to plib035_qep.o(.text.QEP_PC_ResetEventConfig) for QEP_PC_ResetEventConfig
    plib035_qep.o(.text.QEP_PC_Init) refers to plib035_qep.o(.text.QEP_PC_InitEventSConfig) for QEP_PC_InitEventSConfig
    plib035_qep.o(.text.QEP_PC_Init) refers to plib035_qep.o(.text.QEP_PC_InitEventIConfig) for QEP_PC_InitEventIConfig
    plib035_qep.o(.text.QEP_PC_Init) refers to plib035_qep.o(.text.QEP_PC_LatchEventSConfig) for QEP_PC_LatchEventSConfig
    plib035_qep.o(.text.QEP_PC_Init) refers to plib035_qep.o(.text.QEP_PC_LatchEventIConfig) for QEP_PC_LatchEventIConfig
    plib035_qep.o(.text.QEP_PC_Init) refers to plib035_qep.o(.text.QEP_PC_SetCount) for QEP_PC_SetCount
    plib035_qep.o(.text.QEP_PC_Init) refers to plib035_qep.o(.text.QEP_PC_SetCountInit) for QEP_PC_SetCountInit
    plib035_qep.o(.text.QEP_PC_Init) refers to plib035_qep.o(.text.QEP_PC_SetCountMax) for QEP_PC_SetCountMax
    plib035_qep.o(.ARM.exidx.text.QEP_PC_Init) refers to plib035_qep.o(.text.QEP_PC_Init) for [Anonymous Symbol]
    plib035_qep.o(.ARM.exidx.text.QEP_PC_ModeConfig) refers to plib035_qep.o(.text.QEP_PC_ModeConfig) for [Anonymous Symbol]
    plib035_qep.o(.ARM.exidx.text.QEP_PC_CountRateConfig) refers to plib035_qep.o(.text.QEP_PC_CountRateConfig) for [Anonymous Symbol]
    plib035_qep.o(.ARM.exidx.text.QEP_PC_ResetEventConfig) refers to plib035_qep.o(.text.QEP_PC_ResetEventConfig) for [Anonymous Symbol]
    plib035_qep.o(.ARM.exidx.text.QEP_PC_InitEventSConfig) refers to plib035_qep.o(.text.QEP_PC_InitEventSConfig) for [Anonymous Symbol]
    plib035_qep.o(.ARM.exidx.text.QEP_PC_InitEventIConfig) refers to plib035_qep.o(.text.QEP_PC_InitEventIConfig) for [Anonymous Symbol]
    plib035_qep.o(.ARM.exidx.text.QEP_PC_LatchEventSConfig) refers to plib035_qep.o(.text.QEP_PC_LatchEventSConfig) for [Anonymous Symbol]
    plib035_qep.o(.ARM.exidx.text.QEP_PC_LatchEventIConfig) refers to plib035_qep.o(.text.QEP_PC_LatchEventIConfig) for [Anonymous Symbol]
    plib035_qep.o(.ARM.exidx.text.QEP_PC_SetCount) refers to plib035_qep.o(.text.QEP_PC_SetCount) for [Anonymous Symbol]
    plib035_qep.o(.ARM.exidx.text.QEP_PC_SetCountInit) refers to plib035_qep.o(.text.QEP_PC_SetCountInit) for [Anonymous Symbol]
    plib035_qep.o(.ARM.exidx.text.QEP_PC_SetCountMax) refers to plib035_qep.o(.text.QEP_PC_SetCountMax) for [Anonymous Symbol]
    plib035_qep.o(.ARM.exidx.text.QEP_PC_StructInit) refers to plib035_qep.o(.text.QEP_PC_StructInit) for [Anonymous Symbol]
    plib035_qep.o(.text.QEP_CMP_Init) refers to plib035_qep.o(.text.QEP_CMP_ShadowLoadCmd) for QEP_CMP_ShadowLoadCmd
    plib035_qep.o(.text.QEP_CMP_Init) refers to plib035_qep.o(.text.QEP_CMP_LoadEventConfig) for QEP_CMP_LoadEventConfig
    plib035_qep.o(.text.QEP_CMP_Init) refers to plib035_qep.o(.text.QEP_CMP_OutConfig) for QEP_CMP_OutConfig
    plib035_qep.o(.text.QEP_CMP_Init) refers to plib035_qep.o(.text.QEP_CMP_OutCmd) for QEP_CMP_OutCmd
    plib035_qep.o(.text.QEP_CMP_Init) refers to plib035_qep.o(.text.QEP_CMP_OutPolarityConfig) for QEP_CMP_OutPolarityConfig
    plib035_qep.o(.text.QEP_CMP_Init) refers to plib035_qep.o(.text.QEP_CMP_SetOutWidth) for QEP_CMP_SetOutWidth
    plib035_qep.o(.text.QEP_CMP_Init) refers to plib035_qep.o(.text.QEP_CMP_SetComp) for QEP_CMP_SetComp
    plib035_qep.o(.ARM.exidx.text.QEP_CMP_Init) refers to plib035_qep.o(.text.QEP_CMP_Init) for [Anonymous Symbol]
    plib035_qep.o(.ARM.exidx.text.QEP_CMP_ShadowLoadCmd) refers to plib035_qep.o(.text.QEP_CMP_ShadowLoadCmd) for [Anonymous Symbol]
    plib035_qep.o(.ARM.exidx.text.QEP_CMP_LoadEventConfig) refers to plib035_qep.o(.text.QEP_CMP_LoadEventConfig) for [Anonymous Symbol]
    plib035_qep.o(.ARM.exidx.text.QEP_CMP_OutConfig) refers to plib035_qep.o(.text.QEP_CMP_OutConfig) for [Anonymous Symbol]
    plib035_qep.o(.ARM.exidx.text.QEP_CMP_OutCmd) refers to plib035_qep.o(.text.QEP_CMP_OutCmd) for [Anonymous Symbol]
    plib035_qep.o(.ARM.exidx.text.QEP_CMP_OutPolarityConfig) refers to plib035_qep.o(.text.QEP_CMP_OutPolarityConfig) for [Anonymous Symbol]
    plib035_qep.o(.ARM.exidx.text.QEP_CMP_SetOutWidth) refers to plib035_qep.o(.text.QEP_CMP_SetOutWidth) for [Anonymous Symbol]
    plib035_qep.o(.ARM.exidx.text.QEP_CMP_SetComp) refers to plib035_qep.o(.text.QEP_CMP_SetComp) for [Anonymous Symbol]
    plib035_qep.o(.ARM.exidx.text.QEP_CMP_StructInit) refers to plib035_qep.o(.text.QEP_CMP_StructInit) for [Anonymous Symbol]
    plib035_qep.o(.text.QEP_CAP_Init) refers to plib035_qep.o(.text.QEP_CAP_DivShadowLoadCmd) for QEP_CAP_DivShadowLoadCmd
    plib035_qep.o(.text.QEP_CAP_Init) refers to plib035_qep.o(.text.QEP_CAP_ResetEventConfig) for QEP_CAP_ResetEventConfig
    plib035_qep.o(.text.QEP_CAP_Init) refers to plib035_qep.o(.text.QEP_CAP_DivConfig) for QEP_CAP_DivConfig
    plib035_qep.o(.text.QEP_CAP_Init) refers to plib035_qep.o(.text.QEP_CAP_LatchEventConfig) for QEP_CAP_LatchEventConfig
    plib035_qep.o(.text.QEP_CAP_Init) refers to plib035_qep.o(.text.QEP_CAP_SetCount) for QEP_CAP_SetCount
    plib035_qep.o(.text.QEP_CAP_Init) refers to plib035_qep.o(.text.QEP_CAP_SetPeriod) for QEP_CAP_SetPeriod
    plib035_qep.o(.ARM.exidx.text.QEP_CAP_Init) refers to plib035_qep.o(.text.QEP_CAP_Init) for [Anonymous Symbol]
    plib035_qep.o(.ARM.exidx.text.QEP_CAP_DivShadowLoadCmd) refers to plib035_qep.o(.text.QEP_CAP_DivShadowLoadCmd) for [Anonymous Symbol]
    plib035_qep.o(.ARM.exidx.text.QEP_CAP_ResetEventConfig) refers to plib035_qep.o(.text.QEP_CAP_ResetEventConfig) for [Anonymous Symbol]
    plib035_qep.o(.ARM.exidx.text.QEP_CAP_DivConfig) refers to plib035_qep.o(.text.QEP_CAP_DivConfig) for [Anonymous Symbol]
    plib035_qep.o(.ARM.exidx.text.QEP_CAP_LatchEventConfig) refers to plib035_qep.o(.text.QEP_CAP_LatchEventConfig) for [Anonymous Symbol]
    plib035_qep.o(.ARM.exidx.text.QEP_CAP_SetCount) refers to plib035_qep.o(.text.QEP_CAP_SetCount) for [Anonymous Symbol]
    plib035_qep.o(.ARM.exidx.text.QEP_CAP_SetPeriod) refers to plib035_qep.o(.text.QEP_CAP_SetPeriod) for [Anonymous Symbol]
    plib035_qep.o(.ARM.exidx.text.QEP_CAP_StructInit) refers to plib035_qep.o(.text.QEP_CAP_StructInit) for [Anonymous Symbol]
    plib035_rcu.o(.ARM.exidx.text.RCU_GetOSIClkFreq) refers to plib035_rcu.o(.text.RCU_GetOSIClkFreq) for [Anonymous Symbol]
    plib035_rcu.o(.ARM.exidx.text.RCU_GetOSEClkFreq) refers to plib035_rcu.o(.text.RCU_GetOSEClkFreq) for [Anonymous Symbol]
    plib035_rcu.o(.ARM.exidx.text.RCU_GetPLLClkFreq) refers to plib035_rcu.o(.text.RCU_GetPLLClkFreq) for [Anonymous Symbol]
    plib035_rcu.o(.text.RCU_GetPLLDivClkFreq) refers to plib035_rcu.o(.text.RCU_GetPLLClkFreq) for RCU_GetPLLClkFreq
    plib035_rcu.o(.ARM.exidx.text.RCU_GetPLLDivClkFreq) refers to plib035_rcu.o(.text.RCU_GetPLLDivClkFreq) for [Anonymous Symbol]
    plib035_rcu.o(.text.RCU_GetSysClkFreq) refers to plib035_rcu.o(.text.RCU_SysClkStatus) for RCU_SysClkStatus
    plib035_rcu.o(.text.RCU_GetSysClkFreq) refers to plib035_rcu.o(.text.getSysClkFreq) for getSysClkFreq
    plib035_rcu.o(.ARM.exidx.text.RCU_GetSysClkFreq) refers to plib035_rcu.o(.text.RCU_GetSysClkFreq) for [Anonymous Symbol]
    plib035_rcu.o(.ARM.exidx.text.RCU_SysClkStatus) refers to plib035_rcu.o(.text.RCU_SysClkStatus) for [Anonymous Symbol]
    plib035_rcu.o(.text.getSysClkFreq) refers to plib035_rcu.o(.text.RCU_GetOSIClkFreq) for RCU_GetOSIClkFreq
    plib035_rcu.o(.text.getSysClkFreq) refers to plib035_rcu.o(.text.RCU_GetOSEClkFreq) for RCU_GetOSEClkFreq
    plib035_rcu.o(.text.getSysClkFreq) refers to plib035_rcu.o(.text.RCU_GetPLLClkFreq) for RCU_GetPLLClkFreq
    plib035_rcu.o(.text.getSysClkFreq) refers to plib035_rcu.o(.text.RCU_GetPLLDivClkFreq) for RCU_GetPLLDivClkFreq
    plib035_rcu.o(.ARM.exidx.text.getSysClkFreq) refers to plib035_rcu.o(.text.getSysClkFreq) for [Anonymous Symbol]
    plib035_rcu.o(.text.RCU_GetUARTClkFreq) refers to plib035_rcu.o(.text.getPeriphClkFreq) for getPeriphClkFreq
    plib035_rcu.o(.ARM.exidx.text.RCU_GetUARTClkFreq) refers to plib035_rcu.o(.text.RCU_GetUARTClkFreq) for [Anonymous Symbol]
    plib035_rcu.o(.text.getPeriphClkFreq) refers to plib035_rcu.o(.text.RCU_GetOSEClkFreq) for RCU_GetOSEClkFreq
    plib035_rcu.o(.text.getPeriphClkFreq) refers to plib035_rcu.o(.text.RCU_GetPLLClkFreq) for RCU_GetPLLClkFreq
    plib035_rcu.o(.text.getPeriphClkFreq) refers to plib035_rcu.o(.text.RCU_GetPLLDivClkFreq) for RCU_GetPLLDivClkFreq
    plib035_rcu.o(.text.getPeriphClkFreq) refers to plib035_rcu.o(.text.RCU_GetOSIClkFreq) for RCU_GetOSIClkFreq
    plib035_rcu.o(.ARM.exidx.text.getPeriphClkFreq) refers to plib035_rcu.o(.text.getPeriphClkFreq) for [Anonymous Symbol]
    plib035_rcu.o(.text.RCU_GetSPIClkFreq) refers to plib035_rcu.o(.text.getPeriphClkFreq) for getPeriphClkFreq
    plib035_rcu.o(.ARM.exidx.text.RCU_GetSPIClkFreq) refers to plib035_rcu.o(.text.RCU_GetSPIClkFreq) for [Anonymous Symbol]
    plib035_rcu.o(.text.RCU_GetADCClkFreq) refers to plib035_rcu.o(.text.getPeriphClkFreq) for getPeriphClkFreq
    plib035_rcu.o(.ARM.exidx.text.RCU_GetADCClkFreq) refers to plib035_rcu.o(.text.RCU_GetADCClkFreq) for [Anonymous Symbol]
    plib035_rcu.o(.text.RCU_GetWDTClkFreq) refers to plib035_rcu.o(.text.getSysPeriphClkFreq) for getSysPeriphClkFreq
    plib035_rcu.o(.ARM.exidx.text.RCU_GetWDTClkFreq) refers to plib035_rcu.o(.text.RCU_GetWDTClkFreq) for [Anonymous Symbol]
    plib035_rcu.o(.text.getSysPeriphClkFreq) refers to plib035_rcu.o(.text.RCU_GetOSEClkFreq) for RCU_GetOSEClkFreq
    plib035_rcu.o(.text.getSysPeriphClkFreq) refers to plib035_rcu.o(.text.RCU_GetPLLClkFreq) for RCU_GetPLLClkFreq
    plib035_rcu.o(.text.getSysPeriphClkFreq) refers to plib035_rcu.o(.text.RCU_GetPLLDivClkFreq) for RCU_GetPLLDivClkFreq
    plib035_rcu.o(.text.getSysPeriphClkFreq) refers to plib035_rcu.o(.text.RCU_GetOSIClkFreq) for RCU_GetOSIClkFreq
    plib035_rcu.o(.ARM.exidx.text.getSysPeriphClkFreq) refers to plib035_rcu.o(.text.getSysPeriphClkFreq) for [Anonymous Symbol]
    plib035_rcu.o(.text.RCU_GetTraceClkFreq) refers to plib035_rcu.o(.text.getSysPeriphClkFreq) for getSysPeriphClkFreq
    plib035_rcu.o(.ARM.exidx.text.RCU_GetTraceClkFreq) refers to plib035_rcu.o(.text.RCU_GetTraceClkFreq) for [Anonymous Symbol]
    plib035_rcu.o(.text.RCU_GetClkOutFreq) refers to plib035_rcu.o(.text.getSysPeriphClkFreq) for getSysPeriphClkFreq
    plib035_rcu.o(.ARM.exidx.text.RCU_GetClkOutFreq) refers to plib035_rcu.o(.text.RCU_GetClkOutFreq) for [Anonymous Symbol]
    plib035_rcu.o(.text.RCU_PLL_AutoConfig) refers to plib035_rcu.o(.text.RCU_PLL_StructInit) for RCU_PLL_StructInit
    plib035_rcu.o(.text.RCU_PLL_AutoConfig) refers to plib035_rcu.o(.text.RCU_PLL_Init) for RCU_PLL_Init
    plib035_rcu.o(.text.RCU_PLL_AutoConfig) refers to plib035_rcu.o(.text.MFLASH_LatencyConfig) for MFLASH_LatencyConfig
    plib035_rcu.o(.text.RCU_PLL_AutoConfig) refers to plib035_rcu.o(.text.RCU_SysClkChangeCmd) for RCU_SysClkChangeCmd
    plib035_rcu.o(.ARM.exidx.text.RCU_PLL_AutoConfig) refers to plib035_rcu.o(.text.RCU_PLL_AutoConfig) for [Anonymous Symbol]
    plib035_rcu.o(.ARM.exidx.text.RCU_PLL_StructInit) refers to plib035_rcu.o(.text.RCU_PLL_StructInit) for [Anonymous Symbol]
    plib035_rcu.o(.text.RCU_PLL_Init) refers to plib035_rcu.o(.text.RCU_PLL_OutCmd) for RCU_PLL_OutCmd
    plib035_rcu.o(.text.RCU_PLL_Init) refers to plib035_rcu.o(.text.RCU_PLL_LockStatus) for RCU_PLL_LockStatus
    plib035_rcu.o(.ARM.exidx.text.RCU_PLL_Init) refers to plib035_rcu.o(.text.RCU_PLL_Init) for [Anonymous Symbol]
    plib035_rcu.o(.ARM.exidx.text.MFLASH_LatencyConfig) refers to plib035_rcu.o(.text.MFLASH_LatencyConfig) for [Anonymous Symbol]
    plib035_rcu.o(.text.RCU_SysClkChangeCmd) refers to plib035_rcu.o(.text.RCU_SysClkConfig) for RCU_SysClkConfig
    plib035_rcu.o(.text.RCU_SysClkChangeCmd) refers to plib035_rcu.o(.text.RCU_BusyStatus) for RCU_BusyStatus
    plib035_rcu.o(.text.RCU_SysClkChangeCmd) refers to plib035_rcu.o(.text.RCU_SysClkStatus) for RCU_SysClkStatus
    plib035_rcu.o(.ARM.exidx.text.RCU_SysClkChangeCmd) refers to plib035_rcu.o(.text.RCU_SysClkChangeCmd) for [Anonymous Symbol]
    plib035_rcu.o(.ARM.exidx.text.RCU_PLL_OutCmd) refers to plib035_rcu.o(.text.RCU_PLL_OutCmd) for [Anonymous Symbol]
    plib035_rcu.o(.ARM.exidx.text.RCU_PLL_LockStatus) refers to plib035_rcu.o(.text.RCU_PLL_LockStatus) for [Anonymous Symbol]
    plib035_rcu.o(.text.RCU_PLL_DeInit) refers to plib035_rcu.o(.text.RCU_PLL_OutCmd) for RCU_PLL_OutCmd
    plib035_rcu.o(.ARM.exidx.text.RCU_PLL_DeInit) refers to plib035_rcu.o(.text.RCU_PLL_DeInit) for [Anonymous Symbol]
    plib035_rcu.o(.ARM.exidx.text.RCU_SysClkConfig) refers to plib035_rcu.o(.text.RCU_SysClkConfig) for [Anonymous Symbol]
    plib035_rcu.o(.ARM.exidx.text.RCU_BusyStatus) refers to plib035_rcu.o(.text.RCU_BusyStatus) for [Anonymous Symbol]
    plib035_spi.o(.text.SPI_DeInit) refers to plib035_spi.o(.text.RCU_SPIRstCmd) for RCU_SPIRstCmd
    plib035_spi.o(.ARM.exidx.text.SPI_DeInit) refers to plib035_spi.o(.text.SPI_DeInit) for [Anonymous Symbol]
    plib035_spi.o(.ARM.exidx.text.RCU_SPIRstCmd) refers to plib035_spi.o(.text.RCU_SPIRstCmd) for [Anonymous Symbol]
    plib035_spi.o(.text.SPI_Init) refers to plib035_spi.o(.text.SPI_SCKDivConfig) for SPI_SCKDivConfig
    plib035_spi.o(.text.SPI_Init) refers to plib035_spi.o(.text.SPI_DataWidthConfig) for SPI_DataWidthConfig
    plib035_spi.o(.text.SPI_Init) refers to plib035_spi.o(.text.SPI_FrameFormatConfig) for SPI_FrameFormatConfig
    plib035_spi.o(.text.SPI_Init) refers to plib035_spi.o(.text.SPI_ModeConfig) for SPI_ModeConfig
    plib035_spi.o(.ARM.exidx.text.SPI_Init) refers to plib035_spi.o(.text.SPI_Init) for [Anonymous Symbol]
    plib035_spi.o(.ARM.exidx.text.SPI_SCKDivConfig) refers to plib035_spi.o(.text.SPI_SCKDivConfig) for [Anonymous Symbol]
    plib035_spi.o(.ARM.exidx.text.SPI_DataWidthConfig) refers to plib035_spi.o(.text.SPI_DataWidthConfig) for [Anonymous Symbol]
    plib035_spi.o(.ARM.exidx.text.SPI_FrameFormatConfig) refers to plib035_spi.o(.text.SPI_FrameFormatConfig) for [Anonymous Symbol]
    plib035_spi.o(.ARM.exidx.text.SPI_ModeConfig) refers to plib035_spi.o(.text.SPI_ModeConfig) for [Anonymous Symbol]
    plib035_spi.o(.ARM.exidx.text.SPI_StructInit) refers to plib035_spi.o(.text.SPI_StructInit) for [Anonymous Symbol]
    plib035_tmr.o(.text.TMR_PeriodConfig) refers to plib035_tmr.o(.text.TMR_SetLoad) for TMR_SetLoad
    plib035_tmr.o(.ARM.exidx.text.TMR_PeriodConfig) refers to plib035_tmr.o(.text.TMR_PeriodConfig) for [Anonymous Symbol]
    plib035_tmr.o(.ARM.exidx.text.TMR_SetLoad) refers to plib035_tmr.o(.text.TMR_SetLoad) for [Anonymous Symbol]
    plib035_tmr.o(.text.TMR_FreqConfig) refers to plib035_tmr.o(.text.TMR_SetLoad) for TMR_SetLoad
    plib035_tmr.o(.ARM.exidx.text.TMR_FreqConfig) refers to plib035_tmr.o(.text.TMR_FreqConfig) for [Anonymous Symbol]
    plib035_uart.o(.text.UART_AutoBaudConfig) refers to plib035_rcu.o(.text.RCU_GetUARTClkFreq) for RCU_GetUARTClkFreq
    plib035_uart.o(.text.UART_AutoBaudConfig) refers to plib035_uart.o(.text.UART_BaudDivConfig) for UART_BaudDivConfig
    plib035_uart.o(.ARM.exidx.text.UART_AutoBaudConfig) refers to plib035_uart.o(.text.UART_AutoBaudConfig) for [Anonymous Symbol]
    plib035_uart.o(.ARM.exidx.text.UART_BaudDivConfig) refers to plib035_uart.o(.text.UART_BaudDivConfig) for [Anonymous Symbol]
    plib035_uart.o(.text.UART_DeInit) refers to plib035_uart.o(.text.RCU_UARTRstCmd) for RCU_UARTRstCmd
    plib035_uart.o(.ARM.exidx.text.UART_DeInit) refers to plib035_uart.o(.text.UART_DeInit) for [Anonymous Symbol]
    plib035_uart.o(.ARM.exidx.text.RCU_UARTRstCmd) refers to plib035_uart.o(.text.RCU_UARTRstCmd) for [Anonymous Symbol]
    plib035_uart.o(.text.UART_Init) refers to plib035_uart.o(.text.UART_AutoBaudConfig) for UART_AutoBaudConfig
    plib035_uart.o(.text.UART_Init) refers to plib035_uart.o(.text.UART_DataWidthConfig) for UART_DataWidthConfig
    plib035_uart.o(.text.UART_Init) refers to plib035_uart.o(.text.UART_StopBitConfig) for UART_StopBitConfig
    plib035_uart.o(.text.UART_Init) refers to plib035_uart.o(.text.UART_ParityBitConfig) for UART_ParityBitConfig
    plib035_uart.o(.text.UART_Init) refers to plib035_uart.o(.text.UART_FIFOCmd) for UART_FIFOCmd
    plib035_uart.o(.text.UART_Init) refers to plib035_uart.o(.text.UART_TxCmd) for UART_TxCmd
    plib035_uart.o(.text.UART_Init) refers to plib035_uart.o(.text.UART_RxCmd) for UART_RxCmd
    plib035_uart.o(.ARM.exidx.text.UART_Init) refers to plib035_uart.o(.text.UART_Init) for [Anonymous Symbol]
    plib035_uart.o(.ARM.exidx.text.UART_DataWidthConfig) refers to plib035_uart.o(.text.UART_DataWidthConfig) for [Anonymous Symbol]
    plib035_uart.o(.ARM.exidx.text.UART_StopBitConfig) refers to plib035_uart.o(.text.UART_StopBitConfig) for [Anonymous Symbol]
    plib035_uart.o(.ARM.exidx.text.UART_ParityBitConfig) refers to plib035_uart.o(.text.UART_ParityBitConfig) for [Anonymous Symbol]
    plib035_uart.o(.ARM.exidx.text.UART_FIFOCmd) refers to plib035_uart.o(.text.UART_FIFOCmd) for [Anonymous Symbol]
    plib035_uart.o(.ARM.exidx.text.UART_TxCmd) refers to plib035_uart.o(.text.UART_TxCmd) for [Anonymous Symbol]
    plib035_uart.o(.ARM.exidx.text.UART_RxCmd) refers to plib035_uart.o(.text.UART_RxCmd) for [Anonymous Symbol]
    plib035_uart.o(.ARM.exidx.text.UART_StructInit) refers to plib035_uart.o(.text.UART_StructInit) for [Anonymous Symbol]
    retarget_conf.o(.ARM.exidx.text.retarget_init) refers to retarget_conf.o(.text.retarget_init) for [Anonymous Symbol]
    retarget_conf.o(.ARM.exidx.text.retarget_get_char) refers to retarget_conf.o(.text.retarget_get_char) for [Anonymous Symbol]
    retarget_conf.o(.ARM.exidx.text.retarget_put_char) refers to retarget_conf.o(.text.retarget_put_char) for [Anonymous Symbol]
    llsdiv.o(.text) refers to lludivv7m.o(.text) for __aeabi_uldivmod
    rt_memcpy_v6.o(.text) refers to rt_memcpy_w.o(.text) for __aeabi_memcpy4
    __main.o(!!!main) refers to __rtentry.o(.ARM.Collect$$rtentry$$00000000) for __rt_entry
    ffltll_clz.o(x$fpl$ffltll) refers (Special) to usenofp.o(x$fpl$usenofp) for __I$use$fp
    cosf.o(i.__hardfp_cosf) refers (Special) to usenofp.o(x$fpl$usenofp) for __I$use$fp
    cosf.o(i.__hardfp_cosf) refers to rredf.o(i.__mathlib_rredf2) for __mathlib_rredf2
    cosf.o(i.__hardfp_cosf) refers to _rserrno.o(.text) for __set_errno
    cosf.o(i.__hardfp_cosf) refers to funder.o(i.__mathlib_flt_invalid) for __mathlib_flt_invalid
    cosf.o(i.__hardfp_cosf) refers to funder.o(i.__mathlib_flt_infnan) for __mathlib_flt_infnan
    cosf.o(i.__softfp_cosf) refers (Special) to usenofp.o(x$fpl$usenofp) for __I$use$fp
    cosf.o(i.__softfp_cosf) refers to cosf.o(i.__hardfp_cosf) for __hardfp_cosf
    cosf.o(i.cosf) refers (Special) to usenofp.o(x$fpl$usenofp) for __I$use$fp
    cosf.o(i.cosf) refers to cosf.o(i.__hardfp_cosf) for __hardfp_cosf
    sinf.o(i.__hardfp_sinf) refers (Special) to usenofp.o(x$fpl$usenofp) for __I$use$fp
    sinf.o(i.__hardfp_sinf) refers to rredf.o(i.__mathlib_rredf2) for __mathlib_rredf2
    sinf.o(i.__hardfp_sinf) refers to fpclassifyf.o(i.__ARM_fpclassifyf) for __ARM_fpclassifyf
    sinf.o(i.__hardfp_sinf) refers to funder.o(i.__mathlib_flt_underflow) for __mathlib_flt_underflow
    sinf.o(i.__hardfp_sinf) refers to _rserrno.o(.text) for __set_errno
    sinf.o(i.__hardfp_sinf) refers to funder.o(i.__mathlib_flt_invalid) for __mathlib_flt_invalid
    sinf.o(i.__hardfp_sinf) refers to funder.o(i.__mathlib_flt_infnan) for __mathlib_flt_infnan
    sinf.o(i.__softfp_sinf) refers (Special) to usenofp.o(x$fpl$usenofp) for __I$use$fp
    sinf.o(i.__softfp_sinf) refers to sinf.o(i.__hardfp_sinf) for __hardfp_sinf
    sinf.o(i.sinf) refers (Special) to usenofp.o(x$fpl$usenofp) for __I$use$fp
    sinf.o(i.sinf) refers to sinf.o(i.__hardfp_sinf) for __hardfp_sinf
    __rtentry.o(.ARM.Collect$$rtentry$$00000000) refers (Special) to __rtentry2.o(.ARM.Collect$$rtentry$$0000000A) for __rt_entry_li
    __rtentry.o(.ARM.Collect$$rtentry$$00000000) refers (Special) to __rtentry2.o(.ARM.Collect$$rtentry$$0000000D) for __rt_entry_main
    __rtentry.o(.ARM.Collect$$rtentry$$00000000) refers (Special) to __rtentry2.o(.ARM.Collect$$rtentry$$0000000C) for __rt_entry_postli_1
    __rtentry.o(.ARM.Collect$$rtentry$$00000000) refers (Special) to __rtentry2.o(.ARM.Collect$$rtentry$$00000009) for __rt_entry_postsh_1
    __rtentry.o(.ARM.Collect$$rtentry$$00000000) refers (Special) to __rtentry2.o(.ARM.Collect$$rtentry$$00000002) for __rt_entry_presh_1
    __rtentry.o(.ARM.Collect$$rtentry$$00000000) refers (Special) to __rtentry4.o(.ARM.Collect$$rtentry$$00000004) for __rt_entry_sh
    aeabi_ldiv0_sigfpe.o(.text) refers to rt_div0.o(.text) for __rt_div0
    _rserrno.o(.text) refers to rt_errno_addr_intlibspace.o(.text) for __aeabi_errno_addr
    fpclassifyf.o(i.__ARM_fpclassifyf) refers (Special) to usenofp.o(x$fpl$usenofp) for __I$use$fp
    rredf.o(i.__mathlib_rredf2) refers (Special) to usenofp.o(x$fpl$usenofp) for __I$use$fp
    rredf.o(i.__mathlib_rredf2) refers to rredf.o(.constdata) for .constdata
    rredf.o(.constdata) refers (Special) to usenofp.o(x$fpl$usenofp) for __I$use$fp
    __rtentry2.o(.ARM.Collect$$rtentry$$00000008) refers to boardinit2.o(.text) for _platform_post_stackheap_init
    __rtentry2.o(.ARM.Collect$$rtentry$$0000000A) refers to libinit.o(.ARM.Collect$$libinit$$00000000) for __rt_lib_init
    __rtentry2.o(.ARM.Collect$$rtentry$$0000000B) refers to boardinit3.o(.text) for _platform_post_lib_init
    __rtentry2.o(.ARM.Collect$$rtentry$$0000000D) refers to main.o(.text.main) for main
    __rtentry2.o(.ARM.Collect$$rtentry$$0000000D) refers to exit.o(.text) for exit
    __rtentry2.o(.ARM.exidx) refers to __rtentry2.o(.ARM.Collect$$rtentry$$00000001) for .ARM.Collect$$rtentry$$00000001
    __rtentry2.o(.ARM.exidx) refers to __rtentry2.o(.ARM.Collect$$rtentry$$00000008) for .ARM.Collect$$rtentry$$00000008
    __rtentry2.o(.ARM.exidx) refers to __rtentry2.o(.ARM.Collect$$rtentry$$0000000A) for .ARM.Collect$$rtentry$$0000000A
    __rtentry2.o(.ARM.exidx) refers to __rtentry2.o(.ARM.Collect$$rtentry$$0000000B) for .ARM.Collect$$rtentry$$0000000B
    __rtentry2.o(.ARM.exidx) refers to __rtentry2.o(.ARM.Collect$$rtentry$$0000000D) for .ARM.Collect$$rtentry$$0000000D
    __rtentry4.o(.ARM.Collect$$rtentry$$00000004) refers to sys_stackheap_outer.o(.text) for __user_setup_stackheap
    __rtentry4.o(.ARM.exidx) refers to __rtentry4.o(.ARM.Collect$$rtentry$$00000004) for .ARM.Collect$$rtentry$$00000004
    rt_div0.o(.text) refers to defsig_fpe_outer.o(.text) for __rt_SIGFPE
    rt_errno_addr.o(.text) refers to rt_errno_addr.o(.bss) for __aeabi_errno_addr_data
    rt_errno_addr_intlibspace.o(.text) refers to libspace.o(.bss) for __libspace_start
    libspace.o(.text) refers to libspace.o(.bss) for __libspace_start
    sys_stackheap_outer.o(.text) refers to libspace.o(.text) for __user_perproc_libspace
    sys_stackheap_outer.o(.text) refers to startup_k1921vk035.o(.text) for __user_initial_stackheap
    exit.o(.text) refers to rtexit.o(.ARM.Collect$$rtexit$$00000000) for __rt_exit
    defsig_fpe_outer.o(.text) refers to defsig_fpe_inner.o(.text) for __rt_SIGFPE_inner
    defsig_fpe_outer.o(.text) refers to defsig_exit.o(.text) for __sig_exit
    defsig_fpe_formal.o(.text) refers to rt_raise.o(.text) for __rt_raise
    libinit.o(.ARM.Collect$$libinit$$00000000) refers (Special) to libinit2.o(.ARM.Collect$$libinit$$00000030) for __rt_lib_init_alloca_1
    libinit.o(.ARM.Collect$$libinit$$00000000) refers (Special) to libinit2.o(.ARM.Collect$$libinit$$0000002E) for __rt_lib_init_argv_1
    libinit.o(.ARM.Collect$$libinit$$00000000) refers (Special) to libinit2.o(.ARM.Collect$$libinit$$0000001D) for __rt_lib_init_atexit_1
    libinit.o(.ARM.Collect$$libinit$$00000000) refers (Special) to libinit2.o(.ARM.Collect$$libinit$$00000023) for __rt_lib_init_clock_1
    libinit.o(.ARM.Collect$$libinit$$00000000) refers (Special) to libinit2.o(.ARM.Collect$$libinit$$00000034) for __rt_lib_init_cpp_1
    libinit.o(.ARM.Collect$$libinit$$00000000) refers (Special) to libinit2.o(.ARM.Collect$$libinit$$00000032) for __rt_lib_init_exceptions_1
    libinit.o(.ARM.Collect$$libinit$$00000000) refers (Special) to libinit2.o(.ARM.Collect$$libinit$$00000001) for __rt_lib_init_fp_1
    libinit.o(.ARM.Collect$$libinit$$00000000) refers (Special) to libinit2.o(.ARM.Collect$$libinit$$00000021) for __rt_lib_init_fp_trap_1
    libinit.o(.ARM.Collect$$libinit$$00000000) refers (Special) to libinit2.o(.ARM.Collect$$libinit$$00000025) for __rt_lib_init_getenv_1
    libinit.o(.ARM.Collect$$libinit$$00000000) refers (Special) to libinit2.o(.ARM.Collect$$libinit$$0000000C) for __rt_lib_init_heap_1
    libinit.o(.ARM.Collect$$libinit$$00000000) refers (Special) to libinit2.o(.ARM.Collect$$libinit$$00000013) for __rt_lib_init_lc_collate_1
    libinit.o(.ARM.Collect$$libinit$$00000000) refers (Special) to libinit2.o(.ARM.Collect$$libinit$$00000015) for __rt_lib_init_lc_ctype_1
    libinit.o(.ARM.Collect$$libinit$$00000000) refers (Special) to libinit2.o(.ARM.Collect$$libinit$$00000017) for __rt_lib_init_lc_monetary_1
    libinit.o(.ARM.Collect$$libinit$$00000000) refers (Special) to libinit2.o(.ARM.Collect$$libinit$$00000019) for __rt_lib_init_lc_numeric_1
    libinit.o(.ARM.Collect$$libinit$$00000000) refers (Special) to libinit2.o(.ARM.Collect$$libinit$$0000001B) for __rt_lib_init_lc_time_1
    libinit.o(.ARM.Collect$$libinit$$00000000) refers (Special) to libinit2.o(.ARM.Collect$$libinit$$00000006) for __rt_lib_init_preinit_1
    libinit.o(.ARM.Collect$$libinit$$00000000) refers (Special) to libinit2.o(.ARM.Collect$$libinit$$00000010) for __rt_lib_init_rand_1
    libinit.o(.ARM.Collect$$libinit$$00000000) refers (Special) to libinit2.o(.ARM.Collect$$libinit$$00000004) for __rt_lib_init_relocate_pie_1
    libinit.o(.ARM.Collect$$libinit$$00000000) refers (Special) to libinit2.o(.ARM.Collect$$libinit$$00000035) for __rt_lib_init_return
    libinit.o(.ARM.Collect$$libinit$$00000000) refers (Special) to libinit2.o(.ARM.Collect$$libinit$$0000001F) for __rt_lib_init_signal_1
    libinit.o(.ARM.Collect$$libinit$$00000000) refers (Special) to libinit2.o(.ARM.Collect$$libinit$$00000027) for __rt_lib_init_stdio_1
    libinit.o(.ARM.Collect$$libinit$$00000000) refers (Special) to libinit2.o(.ARM.Collect$$libinit$$0000000E) for __rt_lib_init_user_alloc_1
    rtexit.o(.ARM.Collect$$rtexit$$00000000) refers (Special) to rtexit2.o(.ARM.Collect$$rtexit$$00000004) for __rt_exit_exit
    rtexit.o(.ARM.Collect$$rtexit$$00000000) refers (Special) to rtexit2.o(.ARM.Collect$$rtexit$$00000003) for __rt_exit_ls
    rtexit.o(.ARM.Collect$$rtexit$$00000000) refers (Special) to rtexit2.o(.ARM.Collect$$rtexit$$00000002) for __rt_exit_prels_1
    rtexit.o(.ARM.exidx) refers (Special) to rtexit2.o(.ARM.Collect$$rtexit$$00000004) for __rt_exit_exit
    rtexit.o(.ARM.exidx) refers (Special) to rtexit2.o(.ARM.Collect$$rtexit$$00000003) for __rt_exit_ls
    rtexit.o(.ARM.exidx) refers (Special) to rtexit2.o(.ARM.Collect$$rtexit$$00000002) for __rt_exit_prels_1
    rtexit.o(.ARM.exidx) refers to rtexit.o(.ARM.Collect$$rtexit$$00000000) for .ARM.Collect$$rtexit$$00000000
    rt_raise.o(.text) refers to __raise.o(.text) for __raise
    rt_raise.o(.text) refers to sys_exit.o(.text) for _sys_exit
    defsig_exit.o(.text) refers to sys_exit.o(.text) for _sys_exit
    defsig_fpe_inner.o(.text) refers to defsig_general.o(.text) for __default_signal_display
    libinit2.o(.ARM.Collect$$libinit$$00000001) refers to fpinit.o(x$fpl$fpinit) for _fp_init
    libinit2.o(.ARM.Collect$$libinit$$00000012) refers to libinit2.o(.ARM.Collect$$libinit$$00000011) for .ARM.Collect$$libinit$$00000011
    libinit2.o(.ARM.Collect$$libinit$$00000014) refers to libinit2.o(.ARM.Collect$$libinit$$00000011) for .ARM.Collect$$libinit$$00000011
    libinit2.o(.ARM.Collect$$libinit$$00000016) refers to libinit2.o(.ARM.Collect$$libinit$$00000011) for .ARM.Collect$$libinit$$00000011
    libinit2.o(.ARM.Collect$$libinit$$00000018) refers to libinit2.o(.ARM.Collect$$libinit$$00000011) for .ARM.Collect$$libinit$$00000011
    libinit2.o(.ARM.Collect$$libinit$$0000001A) refers to libinit2.o(.ARM.Collect$$libinit$$00000011) for .ARM.Collect$$libinit$$00000011
    libinit2.o(.ARM.Collect$$libinit$$00000028) refers to argv_veneer.o(.emb_text) for __ARM_argv_veneer
    libinit2.o(.ARM.Collect$$libinit$$00000029) refers to argv_veneer.o(.emb_text) for __ARM_argv_veneer
    sys_exit.o(.text) refers (Special) to use_no_semi.o(.text) for __I$use$semihosting
    sys_exit.o(.text) refers (Special) to indicate_semi.o(.text) for __semihosting_library_function
    sys_exit_hlt.o(.text) refers (Special) to use_no_semi.o(.text) for __I$use$semihosting
    sys_exit_hlt.o(.text) refers (Special) to indicate_semi.o(.text) for __semihosting_library_function
    rtexit2.o(.ARM.Collect$$rtexit$$00000003) refers to libshutdown.o(.ARM.Collect$$libshutdown$$00000000) for __rt_lib_shutdown
    rtexit2.o(.ARM.Collect$$rtexit$$00000004) refers to sys_exit.o(.text) for _sys_exit
    rtexit2.o(.ARM.exidx) refers to rtexit2.o(.ARM.Collect$$rtexit$$00000001) for .ARM.Collect$$rtexit$$00000001
    rtexit2.o(.ARM.exidx) refers to rtexit2.o(.ARM.Collect$$rtexit$$00000003) for .ARM.Collect$$rtexit$$00000003
    rtexit2.o(.ARM.exidx) refers to rtexit2.o(.ARM.Collect$$rtexit$$00000004) for .ARM.Collect$$rtexit$$00000004
    __raise.o(.text) refers to defsig.o(CL$$defsig) for __default_signal_handler
    defsig_general.o(.text) refers to sys_wrch.o(.text) for _ttywrch
    argv_veneer.o(.emb_text) refers to no_argv.o(.text) for __ARM_get_argv
    sys_wrch.o(.text) refers (Special) to use_no_semi.o(.text) for __I$use$semihosting
    sys_wrch.o(.text) refers (Special) to indicate_semi.o(.text) for __semihosting_library_function
    sys_wrch_hlt.o(.text) refers (Special) to use_no_semi.o(.text) for __I$use$semihosting
    sys_wrch_hlt.o(.text) refers (Special) to indicate_semi.o(.text) for __semihosting_library_function
    defsig.o(CL$$defsig) refers to defsig_fpe_inner.o(.text) for __rt_SIGFPE_inner
    defsig.o(CL$$defsig) refers to defsig_rtmem_inner.o(.text) for __rt_SIGRTMEM_inner
    _get_argv_nomalloc.o(.text) refers (Special) to hrguard.o(.text) for __heap_region$guard
    _get_argv_nomalloc.o(.text) refers to defsig_rtmem_outer.o(.text) for __rt_SIGRTMEM
    _get_argv_nomalloc.o(.text) refers to sys_command.o(.text) for _sys_command_string
    libshutdown.o(.ARM.Collect$$libshutdown$$00000000) refers (Special) to libshutdown2.o(.ARM.Collect$$libshutdown$$00000002) for __rt_lib_shutdown_cpp_1
    libshutdown.o(.ARM.Collect$$libshutdown$$00000000) refers (Special) to libshutdown2.o(.ARM.Collect$$libshutdown$$00000007) for __rt_lib_shutdown_fp_trap_1
    libshutdown.o(.ARM.Collect$$libshutdown$$00000000) refers (Special) to libshutdown2.o(.ARM.Collect$$libshutdown$$0000000F) for __rt_lib_shutdown_heap_1
    libshutdown.o(.ARM.Collect$$libshutdown$$00000000) refers (Special) to libshutdown2.o(.ARM.Collect$$libshutdown$$00000010) for __rt_lib_shutdown_return
    libshutdown.o(.ARM.Collect$$libshutdown$$00000000) refers (Special) to libshutdown2.o(.ARM.Collect$$libshutdown$$0000000A) for __rt_lib_shutdown_signal_1
    libshutdown.o(.ARM.Collect$$libshutdown$$00000000) refers (Special) to libshutdown2.o(.ARM.Collect$$libshutdown$$00000004) for __rt_lib_shutdown_stdio_1
    libshutdown.o(.ARM.Collect$$libshutdown$$00000000) refers (Special) to libshutdown2.o(.ARM.Collect$$libshutdown$$0000000C) for __rt_lib_shutdown_user_alloc_1
    sys_command.o(.text) refers (Special) to use_no_semi.o(.text) for __I$use$semihosting
    sys_command.o(.text) refers (Special) to indicate_semi.o(.text) for __semihosting_library_function
    sys_command_hlt.o(.text) refers (Special) to use_no_semi.o(.text) for __I$use$semihosting
    sys_command_hlt.o(.text) refers (Special) to indicate_semi.o(.text) for __semihosting_library_function
    defsig_abrt_inner.o(.text) refers to defsig_general.o(.text) for __default_signal_display
    defsig_rtred_inner.o(.text) refers to defsig_general.o(.text) for __default_signal_display
    defsig_rtmem_inner.o(.text) refers to defsig_general.o(.text) for __default_signal_display
    defsig_rtmem_outer.o(.text) refers to defsig_rtmem_inner.o(.text) for __rt_SIGRTMEM_inner
    defsig_rtmem_outer.o(.text) refers to defsig_exit.o(.text) for __sig_exit
    defsig_rtmem_formal.o(.text) refers to rt_raise.o(.text) for __rt_raise
    defsig_stak_inner.o(.text) refers to defsig_general.o(.text) for __default_signal_display
    defsig_pvfn_inner.o(.text) refers to defsig_general.o(.text) for __default_signal_display
    defsig_cppl_inner.o(.text) refers to defsig_general.o(.text) for __default_signal_display
    defsig_segv_inner.o(.text) refers to defsig_general.o(.text) for __default_signal_display
    defsig_other.o(.text) refers to defsig_general.o(.text) for __default_signal_display


==============================================================================

Removing Unused input sections from the image.

    Removing main.o(.text), (0 bytes).
    Removing main.o(.ARM.exidx.text.periph_init), (8 bytes).
    Removing main.o(.ARM.exidx.text.restart_receive), (8 bytes).
    Removing main.o(.ARM.exidx.text.heartbit), (8 bytes).
    Removing main.o(.ARM.exidx.text.main), (8 bytes).
    Removing main.o(.ARM.exidx.text.GPIO_ToggleBits), (8 bytes).
    Removing main.o(.ARM.exidx.text.Error_Handler), (8 bytes).
    Removing main.o(.ARM.use_no_argv), (4 bytes).
    Removing gpio.o(.text), (0 bytes).
    Removing gpio.o(.ARM.exidx.text.gpio_init), (8 bytes).
    Removing gpio.o(.ARM.exidx.text.RCU_AHBClkCmd), (8 bytes).
    Removing gpio.o(.ARM.exidx.text.RCU_AHBRstCmd), (8 bytes).
    Removing gpio.o(.ARM.exidx.text.gpio_get_init), (8 bytes).
    Removing tmr.o(.text), (0 bytes).
    Removing tmr.o(.ARM.exidx.text.tmr_init_first), (8 bytes).
    Removing tmr.o(.ARM.exidx.text.RCU_APBClkCmd), (8 bytes).
    Removing tmr.o(.ARM.exidx.text.RCU_APBRstCmd), (8 bytes).
    Removing tmr.o(.ARM.exidx.text.tmr_init), (8 bytes).
    Removing tmr.o(.ARM.exidx.text.__NVIC_EnableIRQ), (8 bytes).
    Removing tmr.o(.ARM.exidx.text.TMR_Init), (8 bytes).
    Removing tmr.o(.ARM.exidx.text.tmr_set_callback), (8 bytes).
    Removing tmr.o(.ARM.exidx.text.tmr_start), (8 bytes).
    Removing tmr.o(.ARM.exidx.text.TMR_Cmd), (8 bytes).
    Removing tmr.o(.text.tmr_stop), (50 bytes).
    Removing tmr.o(.ARM.exidx.text.tmr_stop), (8 bytes).
    Removing tmr.o(.ARM.exidx.text.tmr_delay), (8 bytes).
    Removing tmr.o(.ARM.exidx.text.tmr_delay_start), (8 bytes).
    Removing tmr.o(.ARM.exidx.text.tmr_delay_done), (8 bytes).
    Removing tmr.o(.ARM.exidx.text.tmr_handler), (8 bytes).
    Removing tmr.o(.ARM.exidx.text.TMR_ITStatus), (8 bytes).
    Removing tmr.o(.ARM.exidx.text.TMR_ITStatusClear), (8 bytes).
    Removing tmr.o(.ARM.exidx.text.TMR_SetLoad), (8 bytes).
    Removing tmr.o(.ARM.exidx.text.TMR_ITCmd), (8 bytes).
    Removing tmr.o(.ARM.exidx.text.TMR_DMAReqCmd), (8 bytes).
    Removing tmr.o(.ARM.exidx.text.TMR_ADCSOCCmd), (8 bytes).
    Removing tmr.o(.ARM.exidx.text.TMR_ExtInputConfig), (8 bytes).
    Removing uart.o(.text), (0 bytes).
    Removing uart.o(.ARM.exidx.text.uart_init_first), (8 bytes).
    Removing uart.o(.ARM.exidx.text.uart1_gpio_init), (8 bytes).
    Removing uart.o(.ARM.exidx.text.RCU_UARTClkConfig), (8 bytes).
    Removing uart.o(.ARM.exidx.text.RCU_UARTClkCmd), (8 bytes).
    Removing uart.o(.ARM.exidx.text.__NVIC_EnableIRQ), (8 bytes).
    Removing uart.o(.ARM.exidx.text.uart_init), (8 bytes).
    Removing uart.o(.ARM.exidx.text.uart_start), (8 bytes).
    Removing uart.o(.ARM.exidx.text.UART_ITFIFOLevelRxConfig), (8 bytes).
    Removing uart.o(.ARM.exidx.text.UART_ITFIFOLevelTxConfig), (8 bytes).
    Removing uart.o(.ARM.exidx.text.UART_Cmd), (8 bytes).
    Removing uart.o(.ARM.exidx.text.uart_transmit), (8 bytes).
    Removing uart.o(.ARM.exidx.text.__uart_fifo_transmit), (8 bytes).
    Removing uart.o(.text.uart_receive), (146 bytes).
    Removing uart.o(.ARM.exidx.text.uart_receive), (8 bytes).
    Removing uart.o(.ARM.exidx.text.uart_transmit_it), (8 bytes).
    Removing uart.o(.ARM.exidx.text.UART_ITCmd), (8 bytes).
    Removing uart.o(.ARM.exidx.text.uart_receive_it), (8 bytes).
    Removing uart.o(.ARM.exidx.text.uart_handler), (8 bytes).
    Removing uart.o(.ARM.exidx.text.UART_ErrorStatusClear), (8 bytes).
    Removing uart.o(.ARM.exidx.text.UART_ITStatusClear), (8 bytes).
    Removing uart.o(.ARM.exidx.text.__uart_fifo_receive), (8 bytes).
    Removing uart.o(.ARM.exidx.text.uart_set_callback), (8 bytes).
    Removing uart.o(.text.uart0_gpio_init), (2 bytes).
    Removing uart.o(.ARM.exidx.text.uart0_gpio_init), (8 bytes).
    Removing uart.o(.text.uart0_gpio_deinit), (2 bytes).
    Removing uart.o(.ARM.exidx.text.uart0_gpio_deinit), (8 bytes).
    Removing uart.o(.text.uart1_gpio_deinit), (114 bytes).
    Removing uart.o(.ARM.exidx.text.uart1_gpio_deinit), (8 bytes).
    Removing uart.o(.ARM.exidx.text.UART_FlagStatus), (8 bytes).
    Removing uart.o(.ARM.exidx.text.UART_RecieveData), (8 bytes).
    Removing uart.o(.ARM.exidx.text.UART_SendData), (8 bytes).
    Removing sysclk.o(.text), (0 bytes).
    Removing sysclk.o(.ARM.exidx.text.sysclk_init), (8 bytes).
    Removing sysclk.o(.ARM.exidx.text.RCU_ClkOutConfig), (8 bytes).
    Removing sysclk.o(.ARM.exidx.text.RCU_ClkOutCmd), (8 bytes).
    Removing sysclk.o(.ARM.exidx.text.SysTick_Config), (8 bytes).
    Removing sysclk.o(.ARM.exidx.text.millis), (8 bytes).
    Removing sysclk.o(.ARM.exidx.text.millis_inc), (8 bytes).
    Removing sysclk.o(.text.micros), (4 bytes).
    Removing sysclk.o(.ARM.exidx.text.micros), (8 bytes).
    Removing sysclk.o(.text.micros_inc), (16 bytes).
    Removing sysclk.o(.ARM.exidx.text.micros_inc), (8 bytes).
    Removing sysclk.o(.ARM.exidx.text.__NVIC_SetPriority), (8 bytes).
    Removing vk035_it.o(.text), (0 bytes).
    Removing vk035_it.o(.ARM.exidx.text.WDT_IRQHandler), (8 bytes).
    Removing vk035_it.o(.ARM.exidx.text.RCU_IRQHandler), (8 bytes).
    Removing vk035_it.o(.ARM.exidx.text.MFLASH_IRQHandler), (8 bytes).
    Removing vk035_it.o(.ARM.exidx.text.GPIOA_IRQHandler), (8 bytes).
    Removing vk035_it.o(.ARM.exidx.text.GPIOB_IRQHandler), (8 bytes).
    Removing vk035_it.o(.ARM.exidx.text.TMR0_IRQHandler), (8 bytes).
    Removing vk035_it.o(.ARM.exidx.text.TMR1_IRQHandler), (8 bytes).
    Removing vk035_it.o(.ARM.exidx.text.TMR2_IRQHandler), (8 bytes).
    Removing vk035_it.o(.ARM.exidx.text.TMR3_IRQHandler), (8 bytes).
    Removing vk035_it.o(.ARM.exidx.text.UART0_TD_IRQHandler), (8 bytes).
    Removing vk035_it.o(.ARM.exidx.text.UART0_RX_IRQHandler), (8 bytes).
    Removing vk035_it.o(.ARM.exidx.text.UART0_TX_IRQHandler), (8 bytes).
    Removing vk035_it.o(.ARM.exidx.text.UART0_E_RT_IRQHandler), (8 bytes).
    Removing vk035_it.o(.ARM.exidx.text.UART1_TD_IRQHandler), (8 bytes).
    Removing vk035_it.o(.ARM.exidx.text.UART1_RX_IRQHandler), (8 bytes).
    Removing vk035_it.o(.ARM.exidx.text.UART1_TX_IRQHandler), (8 bytes).
    Removing vk035_it.o(.ARM.exidx.text.UART1_E_RT_IRQHandler), (8 bytes).
    Removing vk035_it.o(.ARM.exidx.text.SPI_RO_RT_IRQHandler), (8 bytes).
    Removing vk035_it.o(.ARM.exidx.text.SPI_RX_IRQHandler), (8 bytes).
    Removing vk035_it.o(.ARM.exidx.text.SPI_TX_IRQHandler), (8 bytes).
    Removing vk035_it.o(.ARM.exidx.text.I2C_IRQHandler), (8 bytes).
    Removing vk035_it.o(.ARM.exidx.text.ECAP0_IRQHandler), (8 bytes).
    Removing vk035_it.o(.ARM.exidx.text.ECAP1_IRQHandler), (8 bytes).
    Removing vk035_it.o(.ARM.exidx.text.ECAP2_IRQHandler), (8 bytes).
    Removing vk035_it.o(.ARM.exidx.text.PWM0_IRQHandler), (8 bytes).
    Removing vk035_it.o(.ARM.exidx.text.PWM0_HD_IRQHandler), (8 bytes).
    Removing vk035_it.o(.ARM.exidx.text.PWM0_TZ_IRQHandler), (8 bytes).
    Removing vk035_it.o(.ARM.exidx.text.PWM1_IRQHandler), (8 bytes).
    Removing vk035_it.o(.ARM.exidx.text.PWM1_HD_IRQHandler), (8 bytes).
    Removing vk035_it.o(.ARM.exidx.text.PWM1_TZ_IRQHandler), (8 bytes).
    Removing vk035_it.o(.ARM.exidx.text.PWM2_IRQHandler), (8 bytes).
    Removing vk035_it.o(.ARM.exidx.text.PWM2_HD_IRQHandler), (8 bytes).
    Removing vk035_it.o(.ARM.exidx.text.PWM2_TZ_IRQHandler), (8 bytes).
    Removing vk035_it.o(.ARM.exidx.text.QEP_IRQHandler), (8 bytes).
    Removing vk035_it.o(.ARM.exidx.text.ADC_SEQ0_IRQHandler), (8 bytes).
    Removing vk035_it.o(.ARM.exidx.text.ADC_SEQ1_IRQHandler), (8 bytes).
    Removing vk035_it.o(.ARM.exidx.text.ADC_DC_IRQHandler), (8 bytes).
    Removing vk035_it.o(.ARM.exidx.text.CAN0_IRQHandler), (8 bytes).
    Removing vk035_it.o(.ARM.exidx.text.CAN1_IRQHandler), (8 bytes).
    Removing vk035_it.o(.ARM.exidx.text.CAN2_IRQHandler), (8 bytes).
    Removing vk035_it.o(.ARM.exidx.text.CAN3_IRQHandler), (8 bytes).
    Removing vk035_it.o(.ARM.exidx.text.CAN4_IRQHandler), (8 bytes).
    Removing vk035_it.o(.ARM.exidx.text.CAN5_IRQHandler), (8 bytes).
    Removing vk035_it.o(.ARM.exidx.text.CAN6_IRQHandler), (8 bytes).
    Removing vk035_it.o(.ARM.exidx.text.CAN7_IRQHandler), (8 bytes).
    Removing vk035_it.o(.ARM.exidx.text.CAN8_IRQHandler), (8 bytes).
    Removing vk035_it.o(.ARM.exidx.text.CAN9_IRQHandler), (8 bytes).
    Removing vk035_it.o(.ARM.exidx.text.CAN10_IRQHandler), (8 bytes).
    Removing vk035_it.o(.ARM.exidx.text.CAN11_IRQHandler), (8 bytes).
    Removing vk035_it.o(.ARM.exidx.text.CAN12_IRQHandler), (8 bytes).
    Removing vk035_it.o(.ARM.exidx.text.CAN13_IRQHandler), (8 bytes).
    Removing vk035_it.o(.ARM.exidx.text.CAN14_IRQHandler), (8 bytes).
    Removing vk035_it.o(.ARM.exidx.text.CAN15_IRQHandler), (8 bytes).
    Removing vk035_it.o(.ARM.exidx.text.FPU_IRQHandler), (8 bytes).
    Removing vk035_it.o(.ARM.exidx.text.DMA_CH0_IRQHandler), (8 bytes).
    Removing vk035_it.o(.ARM.exidx.text.DMA_CH1_IRQHandler), (8 bytes).
    Removing vk035_it.o(.ARM.exidx.text.DMA_CH2_IRQHandler), (8 bytes).
    Removing vk035_it.o(.ARM.exidx.text.DMA_CH3_IRQHandler), (8 bytes).
    Removing vk035_it.o(.ARM.exidx.text.DMA_CH4_IRQHandler), (8 bytes).
    Removing vk035_it.o(.ARM.exidx.text.DMA_CH5_IRQHandler), (8 bytes).
    Removing vk035_it.o(.ARM.exidx.text.DMA_CH6_IRQHandler), (8 bytes).
    Removing vk035_it.o(.ARM.exidx.text.DMA_CH7_IRQHandler), (8 bytes).
    Removing vk035_it.o(.ARM.exidx.text.DMA_CH8_IRQHandler), (8 bytes).
    Removing vk035_it.o(.ARM.exidx.text.DMA_CH9_IRQHandler), (8 bytes).
    Removing vk035_it.o(.ARM.exidx.text.DMA_CH10_IRQHandler), (8 bytes).
    Removing vk035_it.o(.ARM.exidx.text.DMA_CH11_IRQHandler), (8 bytes).
    Removing vk035_it.o(.ARM.exidx.text.DMA_CH12_IRQHandler), (8 bytes).
    Removing vk035_it.o(.ARM.exidx.text.DMA_CH13_IRQHandler), (8 bytes).
    Removing vk035_it.o(.ARM.exidx.text.DMA_CH14_IRQHandler), (8 bytes).
    Removing vk035_it.o(.ARM.exidx.text.DMA_CH15_IRQHandler), (8 bytes).
    Removing vk035_it.o(.ARM.exidx.text.NMI_Handler), (8 bytes).
    Removing vk035_it.o(.ARM.exidx.text.HardFault_Handler), (8 bytes).
    Removing vk035_it.o(.ARM.exidx.text.MemManage_Handler), (8 bytes).
    Removing vk035_it.o(.ARM.exidx.text.BusFault_Handler), (8 bytes).
    Removing vk035_it.o(.ARM.exidx.text.UsageFault_Handler), (8 bytes).
    Removing vk035_it.o(.ARM.exidx.text.SVC_Handler), (8 bytes).
    Removing vk035_it.o(.ARM.exidx.text.DebugMon_Handler), (8 bytes).
    Removing vk035_it.o(.ARM.exidx.text.PendSV_Handler), (8 bytes).
    Removing vk035_it.o(.ARM.exidx.text.SysTick_Handler), (8 bytes).
    Removing segger_rtt.o(.text), (0 bytes).
    Removing segger_rtt.o(.text.SEGGER_RTT_ReadUpBufferNoLock), (314 bytes).
    Removing segger_rtt.o(.ARM.exidx.text.SEGGER_RTT_ReadUpBufferNoLock), (8 bytes).
    Removing segger_rtt.o(.text._DoInit), (166 bytes).
    Removing segger_rtt.o(.ARM.exidx.text._DoInit), (8 bytes).
    Removing segger_rtt.o(.text.SEGGER_RTT_ReadNoLock), (314 bytes).
    Removing segger_rtt.o(.ARM.exidx.text.SEGGER_RTT_ReadNoLock), (8 bytes).
    Removing segger_rtt.o(.text.SEGGER_RTT_ReadUpBuffer), (48 bytes).
    Removing segger_rtt.o(.ARM.exidx.text.SEGGER_RTT_ReadUpBuffer), (8 bytes).
    Removing segger_rtt.o(.text.SEGGER_RTT_Read), (48 bytes).
    Removing segger_rtt.o(.ARM.exidx.text.SEGGER_RTT_Read), (8 bytes).
    Removing segger_rtt.o(.text.SEGGER_RTT_WriteWithOverwriteNoLock), (290 bytes).
    Removing segger_rtt.o(.ARM.exidx.text.SEGGER_RTT_WriteWithOverwriteNoLock), (8 bytes).
    Removing segger_rtt.o(.text.SEGGER_RTT_WriteDownBufferNoLock), (176 bytes).
    Removing segger_rtt.o(.ARM.exidx.text.SEGGER_RTT_WriteDownBufferNoLock), (8 bytes).
    Removing segger_rtt.o(.text._GetAvailWriteSpace), (62 bytes).
    Removing segger_rtt.o(.ARM.exidx.text._GetAvailWriteSpace), (8 bytes).
    Removing segger_rtt.o(.text._WriteNoCheck), (140 bytes).
    Removing segger_rtt.o(.ARM.exidx.text._WriteNoCheck), (8 bytes).
    Removing segger_rtt.o(.text._WriteBlocking), (228 bytes).
    Removing segger_rtt.o(.ARM.exidx.text._WriteBlocking), (8 bytes).
    Removing segger_rtt.o(.text.SEGGER_RTT_WriteNoLock), (176 bytes).
    Removing segger_rtt.o(.ARM.exidx.text.SEGGER_RTT_WriteNoLock), (8 bytes).
    Removing segger_rtt.o(.text.SEGGER_RTT_WriteDownBuffer), (78 bytes).
    Removing segger_rtt.o(.ARM.exidx.text.SEGGER_RTT_WriteDownBuffer), (8 bytes).
    Removing segger_rtt.o(.text.SEGGER_RTT_Write), (78 bytes).
    Removing segger_rtt.o(.ARM.exidx.text.SEGGER_RTT_Write), (8 bytes).
    Removing segger_rtt.o(.text.SEGGER_RTT_WriteString), (30 bytes).
    Removing segger_rtt.o(.ARM.exidx.text.SEGGER_RTT_WriteString), (8 bytes).
    Removing segger_rtt.o(.text.SEGGER_RTT_PutCharSkipNoLock), (114 bytes).
    Removing segger_rtt.o(.ARM.exidx.text.SEGGER_RTT_PutCharSkipNoLock), (8 bytes).
    Removing segger_rtt.o(.text.SEGGER_RTT_PutCharSkip), (166 bytes).
    Removing segger_rtt.o(.ARM.exidx.text.SEGGER_RTT_PutCharSkip), (8 bytes).
    Removing segger_rtt.o(.text.SEGGER_RTT_PutChar), (194 bytes).
    Removing segger_rtt.o(.ARM.exidx.text.SEGGER_RTT_PutChar), (8 bytes).
    Removing segger_rtt.o(.text.SEGGER_RTT_GetKey), (48 bytes).
    Removing segger_rtt.o(.ARM.exidx.text.SEGGER_RTT_GetKey), (8 bytes).
    Removing segger_rtt.o(.text.SEGGER_RTT_WaitKey), (28 bytes).
    Removing segger_rtt.o(.ARM.exidx.text.SEGGER_RTT_WaitKey), (8 bytes).
    Removing segger_rtt.o(.text.SEGGER_RTT_HasKey), (82 bytes).
    Removing segger_rtt.o(.ARM.exidx.text.SEGGER_RTT_HasKey), (8 bytes).
    Removing segger_rtt.o(.text.SEGGER_RTT_HasData), (44 bytes).
    Removing segger_rtt.o(.ARM.exidx.text.SEGGER_RTT_HasData), (8 bytes).
    Removing segger_rtt.o(.text.SEGGER_RTT_HasDataUp), (44 bytes).
    Removing segger_rtt.o(.ARM.exidx.text.SEGGER_RTT_HasDataUp), (8 bytes).
    Removing segger_rtt.o(.text.SEGGER_RTT_AllocDownBuffer), (244 bytes).
    Removing segger_rtt.o(.ARM.exidx.text.SEGGER_RTT_AllocDownBuffer), (8 bytes).
    Removing segger_rtt.o(.text.SEGGER_RTT_AllocUpBuffer), (244 bytes).
    Removing segger_rtt.o(.ARM.exidx.text.SEGGER_RTT_AllocUpBuffer), (8 bytes).
    Removing segger_rtt.o(.text.SEGGER_RTT_ConfigUpBuffer), (162 bytes).
    Removing segger_rtt.o(.ARM.exidx.text.SEGGER_RTT_ConfigUpBuffer), (8 bytes).
    Removing segger_rtt.o(.text.SEGGER_RTT_ConfigDownBuffer), (166 bytes).
    Removing segger_rtt.o(.ARM.exidx.text.SEGGER_RTT_ConfigDownBuffer), (8 bytes).
    Removing segger_rtt.o(.text.SEGGER_RTT_SetNameUpBuffer), (118 bytes).
    Removing segger_rtt.o(.ARM.exidx.text.SEGGER_RTT_SetNameUpBuffer), (8 bytes).
    Removing segger_rtt.o(.text.SEGGER_RTT_SetNameDownBuffer), (118 bytes).
    Removing segger_rtt.o(.ARM.exidx.text.SEGGER_RTT_SetNameDownBuffer), (8 bytes).
    Removing segger_rtt.o(.text.SEGGER_RTT_SetFlagsUpBuffer), (118 bytes).
    Removing segger_rtt.o(.ARM.exidx.text.SEGGER_RTT_SetFlagsUpBuffer), (8 bytes).
    Removing segger_rtt.o(.text.SEGGER_RTT_SetFlagsDownBuffer), (118 bytes).
    Removing segger_rtt.o(.ARM.exidx.text.SEGGER_RTT_SetFlagsDownBuffer), (8 bytes).
    Removing segger_rtt.o(.text.SEGGER_RTT_Init), (8 bytes).
    Removing segger_rtt.o(.ARM.exidx.text.SEGGER_RTT_Init), (8 bytes).
    Removing segger_rtt.o(.text.SEGGER_RTT_SetTerminal), (220 bytes).
    Removing segger_rtt.o(.ARM.exidx.text.SEGGER_RTT_SetTerminal), (8 bytes).
    Removing segger_rtt.o(.text.SEGGER_RTT_TerminalOut), (348 bytes).
    Removing segger_rtt.o(.ARM.exidx.text.SEGGER_RTT_TerminalOut), (8 bytes).
    Removing segger_rtt.o(.text._PostTerminalSwitch), (50 bytes).
    Removing segger_rtt.o(.ARM.exidx.text._PostTerminalSwitch), (8 bytes).
    Removing segger_rtt.o(.text.SEGGER_RTT_GetAvailWriteSpace), (38 bytes).
    Removing segger_rtt.o(.ARM.exidx.text.SEGGER_RTT_GetAvailWriteSpace), (8 bytes).
    Removing segger_rtt.o(.text.SEGGER_RTT_GetBytesInBuffer), (98 bytes).
    Removing segger_rtt.o(.ARM.exidx.text.SEGGER_RTT_GetBytesInBuffer), (8 bytes).
    Removing segger_rtt.o(.bss._SEGGER_RTT), (168 bytes).
    Removing segger_rtt.o(.rodata._aTerminalId), (16 bytes).
    Removing segger_rtt.o(.bss._ActiveTerminal), (1 bytes).
    Removing segger_rtt.o(.rodata._DoInit._aInitStr), (17 bytes).
    Removing segger_rtt.o(.rodata.str1.1), (9 bytes).
    Removing segger_rtt.o(.bss._acUpBuffer), (4096 bytes).
    Removing segger_rtt.o(.bss._acDownBuffer), (16 bytes).
    Removing segger_rtt_printf.o(.text), (0 bytes).
    Removing segger_rtt_printf.o(.text.SEGGER_RTT_vprintf), (848 bytes).
    Removing segger_rtt_printf.o(.ARM.exidx.text.SEGGER_RTT_vprintf), (8 bytes).
    Removing segger_rtt_printf.o(.text._StoreChar), (118 bytes).
    Removing segger_rtt_printf.o(.ARM.exidx.text._StoreChar), (8 bytes).
    Removing segger_rtt_printf.o(.text._PrintInt), (460 bytes).
    Removing segger_rtt_printf.o(.ARM.exidx.text._PrintInt), (8 bytes).
    Removing segger_rtt_printf.o(.text._PrintUnsigned), (428 bytes).
    Removing segger_rtt_printf.o(.ARM.exidx.text._PrintUnsigned), (8 bytes).
    Removing segger_rtt_printf.o(.text.SEGGER_RTT_printf), (42 bytes).
    Removing segger_rtt_printf.o(.ARM.exidx.text.SEGGER_RTT_printf), (8 bytes).
    Removing segger_rtt_printf.o(.rodata.str1.1), (7 bytes).
    Removing segger_rtt_printf.o(.rodata._PrintUnsigned._aV2C), (16 bytes).
    Removing filters.o(.text), (0 bytes).
    Removing filters.o(.text.FilterMedian_Init), (160 bytes).
    Removing filters.o(.ARM.exidx.text.FilterMedian_Init), (8 bytes).
    Removing filters.o(.text.FilterMedian_Process), (178 bytes).
    Removing filters.o(.ARM.exidx.text.FilterMedian_Process), (8 bytes).
    Removing filters.o(.text.Filter_float_compare), (84 bytes).
    Removing filters.o(.ARM.exidx.text.Filter_float_compare), (8 bytes).
    Removing filters.o(.text.FilterExp_Init), (88 bytes).
    Removing filters.o(.ARM.exidx.text.FilterExp_Init), (8 bytes).
    Removing filters.o(.text.FilterExp_Process), (114 bytes).
    Removing filters.o(.ARM.exidx.text.FilterExp_Process), (8 bytes).
    Removing filters.o(.text.FilterAverage_Init), (126 bytes).
    Removing filters.o(.ARM.exidx.text.FilterAverage_Init), (8 bytes).
    Removing filters.o(.text.FilterAverage_Process), (146 bytes).
    Removing filters.o(.ARM.exidx.text.FilterAverage_Process), (8 bytes).
    Removing filters.o(.text.FilterPoly_Init), (130 bytes).
    Removing filters.o(.ARM.exidx.text.FilterPoly_Init), (8 bytes).
    Removing filters.o(.text.FilterPoly_Process), (154 bytes).
    Removing filters.o(.ARM.exidx.text.FilterPoly_Process), (8 bytes).
    Removing filters.o(.text.FilterLUT_Init), (138 bytes).
    Removing filters.o(.ARM.exidx.text.FilterLUT_Init), (8 bytes).
    Removing filters.o(.text.FilterLUT_Process), (412 bytes).
    Removing filters.o(.ARM.exidx.text.FilterLUT_Process), (8 bytes).
    Removing filters.o(.text.FilterRMS_Init), (148 bytes).
    Removing filters.o(.ARM.exidx.text.FilterRMS_Init), (8 bytes).
    Removing filters.o(.text.FilterRMS_Process), (296 bytes).
    Removing filters.o(.ARM.exidx.text.FilterRMS_Process), (8 bytes).
    Removing filters.o(.text._sqrtf), (30 bytes).
    Removing filters.o(.ARM.exidx.text._sqrtf), (8 bytes).
    Removing filters.o(.text.FilterMedianInt_Init), (170 bytes).
    Removing filters.o(.ARM.exidx.text.FilterMedianInt_Init), (8 bytes).
    Removing filters.o(.text.FilterMedianInt_Process), (480 bytes).
    Removing filters.o(.ARM.exidx.text.FilterMedianInt_Process), (8 bytes).
    Removing filters.o(.text.FilterExpInt_Init), (94 bytes).
    Removing filters.o(.ARM.exidx.text.FilterExpInt_Init), (8 bytes).
    Removing filters.o(.text.FilterExpInt_Process), (118 bytes).
    Removing filters.o(.ARM.exidx.text.FilterExpInt_Process), (8 bytes).
    Removing filters.o(.text.FilterAverageInt_Init), (128 bytes).
    Removing filters.o(.ARM.exidx.text.FilterAverageInt_Init), (8 bytes).
    Removing filters.o(.text.FilterAverageInt_Process), (138 bytes).
    Removing filters.o(.ARM.exidx.text.FilterAverageInt_Process), (8 bytes).
    Removing filters.o(.text.FilterPolyInt_Init), (138 bytes).
    Removing filters.o(.ARM.exidx.text.FilterPolyInt_Init), (8 bytes).
    Removing filters.o(.text.FilterPolyInt_Process), (202 bytes).
    Removing filters.o(.ARM.exidx.text.FilterPolyInt_Process), (8 bytes).
    Removing filters.o(.text.FilterLUTInt_Init), (138 bytes).
    Removing filters.o(.ARM.exidx.text.FilterLUTInt_Init), (8 bytes).
    Removing filters.o(.text.FilterLUTInt_Process), (428 bytes).
    Removing filters.o(.ARM.exidx.text.FilterLUTInt_Process), (8 bytes).
    Removing filters.o(.text.FilterRMSInt_Init), (152 bytes).
    Removing filters.o(.ARM.exidx.text.FilterRMSInt_Init), (8 bytes).
    Removing filters.o(.text.FilterRMSInt_Process), (348 bytes).
    Removing filters.o(.ARM.exidx.text.FilterRMSInt_Process), (8 bytes).
    Removing filters.o(.text.FilterBandPassDerivative_Init), (432 bytes).
    Removing filters.o(.ARM.exidx.text.FilterBandPassDerivative_Init), (8 bytes).
    Removing filters.o(.text.FilterBandPassDerivative_Process), (174 bytes).
    Removing filters.o(.ARM.exidx.text.FilterBandPassDerivative_Process), (8 bytes).
    Removing system_k1921vk035.o(.text), (0 bytes).
    Removing system_k1921vk035.o(.ARM.exidx.text.SystemCoreClockUpdate), (8 bytes).
    Removing system_k1921vk035.o(.ARM.exidx.text.ClkInit), (8 bytes).
    Removing system_k1921vk035.o(.ARM.exidx.text.FPUInit), (8 bytes).
    Removing system_k1921vk035.o(.ARM.exidx.text.SystemInit), (8 bytes).
    Removing plib035_adc.o(.text), (0 bytes).
    Removing plib035_adc.o(.text.ADC_DeInit), (16 bytes).
    Removing plib035_adc.o(.ARM.exidx.text.ADC_DeInit), (8 bytes).
    Removing plib035_adc.o(.text.RCU_ADCRstCmd), (38 bytes).
    Removing plib035_adc.o(.ARM.exidx.text.RCU_ADCRstCmd), (8 bytes).
    Removing plib035_adc.o(.text.ADC_SEQ_Init), (218 bytes).
    Removing plib035_adc.o(.ARM.exidx.text.ADC_SEQ_Init), (8 bytes).
    Removing plib035_adc.o(.text.ADC_SEQ_StartEventConfig), (44 bytes).
    Removing plib035_adc.o(.ARM.exidx.text.ADC_SEQ_StartEventConfig), (8 bytes).
    Removing plib035_adc.o(.text.ADC_SEQ_SwStartEnCmd), (42 bytes).
    Removing plib035_adc.o(.ARM.exidx.text.ADC_SEQ_SwStartEnCmd), (8 bytes).
    Removing plib035_adc.o(.text.ADC_SEQ_ReqConfig), (68 bytes).
    Removing plib035_adc.o(.ARM.exidx.text.ADC_SEQ_ReqConfig), (8 bytes).
    Removing plib035_adc.o(.text.ADC_SEQ_ReqMaxConfig), (40 bytes).
    Removing plib035_adc.o(.ARM.exidx.text.ADC_SEQ_ReqMaxConfig), (8 bytes).
    Removing plib035_adc.o(.text.ADC_SEQ_ReqAverageConfig), (48 bytes).
    Removing plib035_adc.o(.ARM.exidx.text.ADC_SEQ_ReqAverageConfig), (8 bytes).
    Removing plib035_adc.o(.text.ADC_SEQ_ReqAverageCmd), (48 bytes).
    Removing plib035_adc.o(.ARM.exidx.text.ADC_SEQ_ReqAverageCmd), (8 bytes).
    Removing plib035_adc.o(.text.ADC_SEQ_RestartConfig), (36 bytes).
    Removing plib035_adc.o(.ARM.exidx.text.ADC_SEQ_RestartConfig), (8 bytes).
    Removing plib035_adc.o(.text.ADC_SEQ_RestartAverageCmd), (48 bytes).
    Removing plib035_adc.o(.ARM.exidx.text.ADC_SEQ_RestartAverageCmd), (8 bytes).
    Removing plib035_adc.o(.text.ADC_SEQ_SetRestartTimer), (36 bytes).
    Removing plib035_adc.o(.ARM.exidx.text.ADC_SEQ_SetRestartTimer), (8 bytes).
    Removing plib035_adc.o(.text.ADC_SEQ_DCEnableCmd), (64 bytes).
    Removing plib035_adc.o(.ARM.exidx.text.ADC_SEQ_DCEnableCmd), (8 bytes).
    Removing plib035_adc.o(.text.ADC_SEQ_DMAConfig), (48 bytes).
    Removing plib035_adc.o(.ARM.exidx.text.ADC_SEQ_DMAConfig), (8 bytes).
    Removing plib035_adc.o(.text.ADC_SEQ_DMACmd), (40 bytes).
    Removing plib035_adc.o(.ARM.exidx.text.ADC_SEQ_DMACmd), (8 bytes).
    Removing plib035_adc.o(.text.ADC_SEQ_StructInit), (122 bytes).
    Removing plib035_adc.o(.ARM.exidx.text.ADC_SEQ_StructInit), (8 bytes).
    Removing plib035_adc.o(.text.ADC_DC_Init), (88 bytes).
    Removing plib035_adc.o(.ARM.exidx.text.ADC_DC_Init), (8 bytes).
    Removing plib035_adc.o(.text.ADC_DC_OutputCmd), (54 bytes).
    Removing plib035_adc.o(.ARM.exidx.text.ADC_DC_OutputCmd), (8 bytes).
    Removing plib035_adc.o(.text.ADC_DC_SetThresholdLow), (42 bytes).
    Removing plib035_adc.o(.ARM.exidx.text.ADC_DC_SetThresholdLow), (8 bytes).
    Removing plib035_adc.o(.text.ADC_DC_SetThresholdHigh), (50 bytes).
    Removing plib035_adc.o(.ARM.exidx.text.ADC_DC_SetThresholdHigh), (8 bytes).
    Removing plib035_adc.o(.text.ADC_DC_SourceConfig), (54 bytes).
    Removing plib035_adc.o(.ARM.exidx.text.ADC_DC_SourceConfig), (8 bytes).
    Removing plib035_adc.o(.text.ADC_DC_ChannelConfig), (54 bytes).
    Removing plib035_adc.o(.ARM.exidx.text.ADC_DC_ChannelConfig), (8 bytes).
    Removing plib035_adc.o(.text.ADC_DC_Config), (70 bytes).
    Removing plib035_adc.o(.ARM.exidx.text.ADC_DC_Config), (8 bytes).
    Removing plib035_adc.o(.text.ADC_DC_StructInit), (38 bytes).
    Removing plib035_adc.o(.ARM.exidx.text.ADC_DC_StructInit), (8 bytes).
    Removing plib035_can.o(.text), (0 bytes).
    Removing plib035_dma.o(.text), (0 bytes).
    Removing plib035_dma.o(.text.DMA_ChannelDeInit), (22 bytes).
    Removing plib035_dma.o(.ARM.exidx.text.DMA_ChannelDeInit), (8 bytes).
    Removing plib035_dma.o(.text.DMA_ChannelInit), (326 bytes).
    Removing plib035_dma.o(.ARM.exidx.text.DMA_ChannelInit), (8 bytes).
    Removing plib035_dma.o(.text.DMA_ChannelStructInit), (78 bytes).
    Removing plib035_dma.o(.ARM.exidx.text.DMA_ChannelStructInit), (8 bytes).
    Removing plib035_dma.o(.text.DMA_DeInit), (78 bytes).
    Removing plib035_dma.o(.ARM.exidx.text.DMA_DeInit), (8 bytes).
    Removing plib035_dma.o(.text.DMA_Init), (68 bytes).
    Removing plib035_dma.o(.ARM.exidx.text.DMA_Init), (8 bytes).
    Removing plib035_dma.o(.text.DMA_ProtectConfig), (46 bytes).
    Removing plib035_dma.o(.ARM.exidx.text.DMA_ProtectConfig), (8 bytes).
    Removing plib035_dma.o(.text.DMA_UseBurstCmd), (50 bytes).
    Removing plib035_dma.o(.ARM.exidx.text.DMA_UseBurstCmd), (8 bytes).
    Removing plib035_dma.o(.text.DMA_AltCtrlCmd), (50 bytes).
    Removing plib035_dma.o(.ARM.exidx.text.DMA_AltCtrlCmd), (8 bytes).
    Removing plib035_dma.o(.text.DMA_HighPriorityCmd), (50 bytes).
    Removing plib035_dma.o(.ARM.exidx.text.DMA_HighPriorityCmd), (8 bytes).
    Removing plib035_dma.o(.text.DMA_ReqMaskCmd), (50 bytes).
    Removing plib035_dma.o(.ARM.exidx.text.DMA_ReqMaskCmd), (8 bytes).
    Removing plib035_dma.o(.text.DMA_ChannelEnableCmd), (50 bytes).
    Removing plib035_dma.o(.ARM.exidx.text.DMA_ChannelEnableCmd), (8 bytes).
    Removing plib035_dma.o(.text.DMA_StructInit), (50 bytes).
    Removing plib035_dma.o(.ARM.exidx.text.DMA_StructInit), (8 bytes).
    Removing plib035_ecap.o(.text), (0 bytes).
    Removing plib035_ecap.o(.text.ECAP_DeInit), (84 bytes).
    Removing plib035_ecap.o(.ARM.exidx.text.ECAP_DeInit), (8 bytes).
    Removing plib035_ecap.o(.text.RCU_APBRstCmd), (64 bytes).
    Removing plib035_ecap.o(.ARM.exidx.text.RCU_APBRstCmd), (8 bytes).
    Removing plib035_ecap.o(.text.ECAP_Init), (52 bytes).
    Removing plib035_ecap.o(.ARM.exidx.text.ECAP_Init), (8 bytes).
    Removing plib035_ecap.o(.text.ECAP_HaltConfig), (34 bytes).
    Removing plib035_ecap.o(.ARM.exidx.text.ECAP_HaltConfig), (8 bytes).
    Removing plib035_ecap.o(.text.ECAP_SyncOutConfig), (34 bytes).
    Removing plib035_ecap.o(.ARM.exidx.text.ECAP_SyncOutConfig), (8 bytes).
    Removing plib035_ecap.o(.text.ECAP_SyncCmd), (34 bytes).
    Removing plib035_ecap.o(.ARM.exidx.text.ECAP_SyncCmd), (8 bytes).
    Removing plib035_ecap.o(.text.ECAP_ModeConfig), (34 bytes).
    Removing plib035_ecap.o(.ARM.exidx.text.ECAP_ModeConfig), (8 bytes).
    Removing plib035_ecap.o(.text.ECAP_StructInit), (26 bytes).
    Removing plib035_ecap.o(.ARM.exidx.text.ECAP_StructInit), (8 bytes).
    Removing plib035_ecap.o(.text.ECAP_PWM_Init), (42 bytes).
    Removing plib035_ecap.o(.ARM.exidx.text.ECAP_PWM_Init), (8 bytes).
    Removing plib035_ecap.o(.text.ECAP_PWM_SetPeriod), (16 bytes).
    Removing plib035_ecap.o(.ARM.exidx.text.ECAP_PWM_SetPeriod), (8 bytes).
    Removing plib035_ecap.o(.text.ECAP_PWM_SetCompare), (16 bytes).
    Removing plib035_ecap.o(.ARM.exidx.text.ECAP_PWM_SetCompare), (8 bytes).
    Removing plib035_ecap.o(.text.ECAP_PWM_PolarityConfig), (34 bytes).
    Removing plib035_ecap.o(.ARM.exidx.text.ECAP_PWM_PolarityConfig), (8 bytes).
    Removing plib035_ecap.o(.text.ECAP_PWM_StructInit), (30 bytes).
    Removing plib035_ecap.o(.ARM.exidx.text.ECAP_PWM_StructInit), (8 bytes).
    Removing plib035_ecap.o(.text.ECAP_Capture_Init), (122 bytes).
    Removing plib035_ecap.o(.ARM.exidx.text.ECAP_Capture_Init), (8 bytes).
    Removing plib035_ecap.o(.text.ECAP_Capture_ModeConfig), (26 bytes).
    Removing plib035_ecap.o(.ARM.exidx.text.ECAP_Capture_ModeConfig), (8 bytes).
    Removing plib035_ecap.o(.text.ECAP_Capture_StopConfig), (30 bytes).
    Removing plib035_ecap.o(.ARM.exidx.text.ECAP_Capture_StopConfig), (8 bytes).
    Removing plib035_ecap.o(.text.ECAP_Capture_PrescaleConfig), (30 bytes).
    Removing plib035_ecap.o(.ARM.exidx.text.ECAP_Capture_PrescaleConfig), (8 bytes).
    Removing plib035_ecap.o(.text.ECAP_Capture_PolarityEvt0Config), (26 bytes).
    Removing plib035_ecap.o(.ARM.exidx.text.ECAP_Capture_PolarityEvt0Config), (8 bytes).
    Removing plib035_ecap.o(.text.ECAP_Capture_PolarityEvt1Config), (34 bytes).
    Removing plib035_ecap.o(.ARM.exidx.text.ECAP_Capture_PolarityEvt1Config), (8 bytes).
    Removing plib035_ecap.o(.text.ECAP_Capture_PolarityEvt2Config), (34 bytes).
    Removing plib035_ecap.o(.ARM.exidx.text.ECAP_Capture_PolarityEvt2Config), (8 bytes).
    Removing plib035_ecap.o(.text.ECAP_Capture_PolarityEvt3Config), (34 bytes).
    Removing plib035_ecap.o(.ARM.exidx.text.ECAP_Capture_PolarityEvt3Config), (8 bytes).
    Removing plib035_ecap.o(.text.ECAP_Capture_RstEvt0Cmd), (34 bytes).
    Removing plib035_ecap.o(.ARM.exidx.text.ECAP_Capture_RstEvt0Cmd), (8 bytes).
    Removing plib035_ecap.o(.text.ECAP_Capture_RstEvt1Cmd), (34 bytes).
    Removing plib035_ecap.o(.ARM.exidx.text.ECAP_Capture_RstEvt1Cmd), (8 bytes).
    Removing plib035_ecap.o(.text.ECAP_Capture_RstEvt2Cmd), (34 bytes).
    Removing plib035_ecap.o(.ARM.exidx.text.ECAP_Capture_RstEvt2Cmd), (8 bytes).
    Removing plib035_ecap.o(.text.ECAP_Capture_RstEvt3Cmd), (34 bytes).
    Removing plib035_ecap.o(.ARM.exidx.text.ECAP_Capture_RstEvt3Cmd), (8 bytes).
    Removing plib035_ecap.o(.text.ECAP_Capture_StructInit), (56 bytes).
    Removing plib035_ecap.o(.ARM.exidx.text.ECAP_Capture_StructInit), (8 bytes).
    Removing plib035_gpio.o(.text), (0 bytes).
    Removing plib035_gpio.o(.ARM.exidx.text.GPIO_OutModeConfig), (8 bytes).
    Removing plib035_gpio.o(.ARM.exidx.text.GPIO_ModeConfig), (8 bytes).
    Removing plib035_gpio.o(.ARM.exidx.text.GPIO_InModeConfig), (8 bytes).
    Removing plib035_gpio.o(.ARM.exidx.text.GPIO_PullModeConfig), (8 bytes).
    Removing plib035_gpio.o(.ARM.exidx.text.GPIO_DriveModeConfig), (8 bytes).
    Removing plib035_gpio.o(.ARM.exidx.text.GPIO_DeInit), (8 bytes).
    Removing plib035_gpio.o(.ARM.exidx.text.RCU_AHBRstCmd), (8 bytes).
    Removing plib035_gpio.o(.ARM.exidx.text.GPIO_Init), (8 bytes).
    Removing plib035_gpio.o(.ARM.exidx.text.GPIO_OutCmd), (8 bytes).
    Removing plib035_gpio.o(.ARM.exidx.text.GPIO_AltFuncCmd), (8 bytes).
    Removing plib035_gpio.o(.ARM.exidx.text.GPIO_DigitalCmd), (8 bytes).
    Removing plib035_gpio.o(.ARM.exidx.text.GPIO_StructInit), (8 bytes).
    Removing plib035_i2c.o(.text), (0 bytes).
    Removing plib035_i2c.o(.text.I2C_FSFreqConfig), (42 bytes).
    Removing plib035_i2c.o(.ARM.exidx.text.I2C_FSFreqConfig), (8 bytes).
    Removing plib035_i2c.o(.text.I2C_FSDivLowConfig), (32 bytes).
    Removing plib035_i2c.o(.ARM.exidx.text.I2C_FSDivLowConfig), (8 bytes).
    Removing plib035_i2c.o(.text.I2C_FSDivHighConfig), (24 bytes).
    Removing plib035_i2c.o(.ARM.exidx.text.I2C_FSDivHighConfig), (8 bytes).
    Removing plib035_i2c.o(.text.I2C_HSFreqConfig), (44 bytes).
    Removing plib035_i2c.o(.ARM.exidx.text.I2C_HSFreqConfig), (8 bytes).
    Removing plib035_i2c.o(.text.I2C_HSDivLowConfig), (32 bytes).
    Removing plib035_i2c.o(.ARM.exidx.text.I2C_HSDivLowConfig), (8 bytes).
    Removing plib035_i2c.o(.text.I2C_HSDivHighConfig), (24 bytes).
    Removing plib035_i2c.o(.ARM.exidx.text.I2C_HSDivHighConfig), (8 bytes).
    Removing plib035_mflash.o(.text), (0 bytes).
    Removing plib035_mflash.o(.text.MFLASH_ReadData), (104 bytes).
    Removing plib035_mflash.o(.ARM.exidx.text.MFLASH_ReadData), (8 bytes).
    Removing plib035_mflash.o(.text.MFLASH_SetAddr), (18 bytes).
    Removing plib035_mflash.o(.ARM.exidx.text.MFLASH_SetAddr), (8 bytes).
    Removing plib035_mflash.o(.text.MFLASH_SetCmd), (40 bytes).
    Removing plib035_mflash.o(.ARM.exidx.text.MFLASH_SetCmd), (8 bytes).
    Removing plib035_mflash.o(.text.MFLASH_BusyStatus), (14 bytes).
    Removing plib035_mflash.o(.ARM.exidx.text.MFLASH_BusyStatus), (8 bytes).
    Removing plib035_mflash.o(.text.MFLASH_GetData), (20 bytes).
    Removing plib035_mflash.o(.ARM.exidx.text.MFLASH_GetData), (8 bytes).
    Removing plib035_mflash.o(.text.MFLASH_WriteData), (102 bytes).
    Removing plib035_mflash.o(.ARM.exidx.text.MFLASH_WriteData), (8 bytes).
    Removing plib035_mflash.o(.text.MFLASH_SetData), (24 bytes).
    Removing plib035_mflash.o(.ARM.exidx.text.MFLASH_SetData), (8 bytes).
    Removing plib035_mflash.o(.text.MFLASH_ErasePage), (64 bytes).
    Removing plib035_mflash.o(.ARM.exidx.text.MFLASH_ErasePage), (8 bytes).
    Removing plib035_mflash.o(.text.MFLASH_EraseFull), (44 bytes).
    Removing plib035_mflash.o(.ARM.exidx.text.MFLASH_EraseFull), (8 bytes).
    Removing plib035_pmu.o(.text), (0 bytes).
    Removing plib035_pwm.o(.text), (0 bytes).
    Removing plib035_pwm.o(.text.PWM_DeInit), (78 bytes).
    Removing plib035_pwm.o(.ARM.exidx.text.PWM_DeInit), (8 bytes).
    Removing plib035_pwm.o(.text.RCU_APBRstCmd), (64 bytes).
    Removing plib035_pwm.o(.ARM.exidx.text.RCU_APBRstCmd), (8 bytes).
    Removing plib035_pwm.o(.text.PWM_TB_Init), (104 bytes).
    Removing plib035_pwm.o(.ARM.exidx.text.PWM_TB_Init), (8 bytes).
    Removing plib035_pwm.o(.text.PWM_TB_HaltConfig), (34 bytes).
    Removing plib035_pwm.o(.ARM.exidx.text.PWM_TB_HaltConfig), (8 bytes).
    Removing plib035_pwm.o(.text.PWM_TB_PhaseSyncCmd), (34 bytes).
    Removing plib035_pwm.o(.ARM.exidx.text.PWM_TB_PhaseSyncCmd), (8 bytes).
    Removing plib035_pwm.o(.text.PWM_TB_PhaseSyncDirConfig), (34 bytes).
    Removing plib035_pwm.o(.ARM.exidx.text.PWM_TB_PhaseSyncDirConfig), (8 bytes).
    Removing plib035_pwm.o(.text.PWM_TB_ClkDivConfig), (44 bytes).
    Removing plib035_pwm.o(.ARM.exidx.text.PWM_TB_ClkDivConfig), (8 bytes).
    Removing plib035_pwm.o(.text.PWM_TB_SyncOutConfig), (34 bytes).
    Removing plib035_pwm.o(.ARM.exidx.text.PWM_TB_SyncOutConfig), (8 bytes).
    Removing plib035_pwm.o(.text.PWM_TB_PeriodDirectLoadCmd), (34 bytes).
    Removing plib035_pwm.o(.ARM.exidx.text.PWM_TB_PeriodDirectLoadCmd), (8 bytes).
    Removing plib035_pwm.o(.text.PWM_TB_ModeConfig), (26 bytes).
    Removing plib035_pwm.o(.ARM.exidx.text.PWM_TB_ModeConfig), (8 bytes).
    Removing plib035_pwm.o(.text.PWM_TB_SetPhase), (16 bytes).
    Removing plib035_pwm.o(.ARM.exidx.text.PWM_TB_SetPhase), (8 bytes).
    Removing plib035_pwm.o(.text.PWM_TB_SetPeriod), (16 bytes).
    Removing plib035_pwm.o(.ARM.exidx.text.PWM_TB_SetPeriod), (8 bytes).
    Removing plib035_pwm.o(.text.PWM_TB_StructInit), (50 bytes).
    Removing plib035_pwm.o(.ARM.exidx.text.PWM_TB_StructInit), (8 bytes).
    Removing plib035_pwm.o(.text.PWM_AQ_Init), (168 bytes).
    Removing plib035_pwm.o(.ARM.exidx.text.PWM_AQ_Init), (8 bytes).
    Removing plib035_pwm.o(.text.PWM_AQ_ActionAConfig), (42 bytes).
    Removing plib035_pwm.o(.ARM.exidx.text.PWM_AQ_ActionAConfig), (8 bytes).
    Removing plib035_pwm.o(.text.PWM_AQ_ActionBConfig), (42 bytes).
    Removing plib035_pwm.o(.ARM.exidx.text.PWM_AQ_ActionBConfig), (8 bytes).
    Removing plib035_pwm.o(.text.PWM_AQ_StructInit), (58 bytes).
    Removing plib035_pwm.o(.ARM.exidx.text.PWM_AQ_StructInit), (8 bytes).
    Removing plib035_pwm.o(.text.PWM_CMP_Init), (72 bytes).
    Removing plib035_pwm.o(.ARM.exidx.text.PWM_CMP_Init), (8 bytes).
    Removing plib035_pwm.o(.text.PWM_CMP_CmpALoadEventConfig), (26 bytes).
    Removing plib035_pwm.o(.ARM.exidx.text.PWM_CMP_CmpALoadEventConfig), (8 bytes).
    Removing plib035_pwm.o(.text.PWM_CMP_CmpADirectLoadCmd), (34 bytes).
    Removing plib035_pwm.o(.ARM.exidx.text.PWM_CMP_CmpADirectLoadCmd), (8 bytes).
    Removing plib035_pwm.o(.text.PWM_CMP_SetCmpA), (22 bytes).
    Removing plib035_pwm.o(.ARM.exidx.text.PWM_CMP_SetCmpA), (8 bytes).
    Removing plib035_pwm.o(.text.PWM_CMP_SetCmpB), (22 bytes).
    Removing plib035_pwm.o(.ARM.exidx.text.PWM_CMP_SetCmpB), (8 bytes).
    Removing plib035_pwm.o(.text.PWM_CMP_StructInit), (34 bytes).
    Removing plib035_pwm.o(.ARM.exidx.text.PWM_CMP_StructInit), (8 bytes).
    Removing plib035_pwm.o(.text.PWM_HD_Init), (64 bytes).
    Removing plib035_pwm.o(.ARM.exidx.text.PWM_HD_Init), (8 bytes).
    Removing plib035_pwm.o(.text.PWM_HD_ActionAConfig), (30 bytes).
    Removing plib035_pwm.o(.ARM.exidx.text.PWM_HD_ActionAConfig), (8 bytes).
    Removing plib035_pwm.o(.text.PWM_HD_ActionBConfig), (38 bytes).
    Removing plib035_pwm.o(.ARM.exidx.text.PWM_HD_ActionBConfig), (8 bytes).
    Removing plib035_pwm.o(.text.PWM_HD_SourceCmd), (58 bytes).
    Removing plib035_pwm.o(.ARM.exidx.text.PWM_HD_SourceCmd), (8 bytes).
    Removing plib035_pwm.o(.text.PWM_HD_CycleCmd), (38 bytes).
    Removing plib035_pwm.o(.ARM.exidx.text.PWM_HD_CycleCmd), (8 bytes).
    Removing plib035_pwm.o(.text.PWM_HD_OneShotCmd), (34 bytes).
    Removing plib035_pwm.o(.ARM.exidx.text.PWM_HD_OneShotCmd), (8 bytes).
    Removing plib035_pwm.o(.text.PWM_HD_StructInit), (32 bytes).
    Removing plib035_pwm.o(.ARM.exidx.text.PWM_HD_StructInit), (8 bytes).
    Removing plib035_pwm.o(.text.PWM_DB_Init), (62 bytes).
    Removing plib035_pwm.o(.ARM.exidx.text.PWM_DB_Init), (8 bytes).
    Removing plib035_pwm.o(.text.PWM_DB_InConfig), (34 bytes).
    Removing plib035_pwm.o(.ARM.exidx.text.PWM_DB_InConfig), (8 bytes).
    Removing plib035_pwm.o(.text.PWM_DB_OutConfig), (26 bytes).
    Removing plib035_pwm.o(.ARM.exidx.text.PWM_DB_OutConfig), (8 bytes).
    Removing plib035_pwm.o(.text.PWM_DB_PolarityConfig), (34 bytes).
    Removing plib035_pwm.o(.ARM.exidx.text.PWM_DB_PolarityConfig), (8 bytes).
    Removing plib035_pwm.o(.text.PWM_DB_SetRiseDelay), (16 bytes).
    Removing plib035_pwm.o(.ARM.exidx.text.PWM_DB_SetRiseDelay), (8 bytes).
    Removing plib035_pwm.o(.text.PWM_DB_SetFallDelay), (16 bytes).
    Removing plib035_pwm.o(.ARM.exidx.text.PWM_DB_SetFallDelay), (8 bytes).
    Removing plib035_pwm.o(.text.PWM_DB_StructInit), (30 bytes).
    Removing plib035_pwm.o(.ARM.exidx.text.PWM_DB_StructInit), (8 bytes).
    Removing plib035_pwm.o(.text.PWM_TZ_Init), (52 bytes).
    Removing plib035_pwm.o(.ARM.exidx.text.PWM_TZ_Init), (8 bytes).
    Removing plib035_pwm.o(.text.PWM_TZ_ActionAConfig), (26 bytes).
    Removing plib035_pwm.o(.ARM.exidx.text.PWM_TZ_ActionAConfig), (8 bytes).
    Removing plib035_pwm.o(.text.PWM_TZ_ActionBConfig), (34 bytes).
    Removing plib035_pwm.o(.ARM.exidx.text.PWM_TZ_ActionBConfig), (8 bytes).
    Removing plib035_pwm.o(.text.PWM_TZ_CycleCmd), (26 bytes).
    Removing plib035_pwm.o(.ARM.exidx.text.PWM_TZ_CycleCmd), (8 bytes).
    Removing plib035_pwm.o(.text.PWM_TZ_OneShotCmd), (34 bytes).
    Removing plib035_pwm.o(.ARM.exidx.text.PWM_TZ_OneShotCmd), (8 bytes).
    Removing plib035_pwm.o(.text.PWM_TZ_StructInit), (26 bytes).
    Removing plib035_pwm.o(.ARM.exidx.text.PWM_TZ_StructInit), (8 bytes).
    Removing plib035_pwm.o(.text.PWM_ET_Init), (132 bytes).
    Removing plib035_pwm.o(.ARM.exidx.text.PWM_ET_Init), (8 bytes).
    Removing plib035_pwm.o(.text.PWM_ET_SOCAEventConfig), (34 bytes).
    Removing plib035_pwm.o(.ARM.exidx.text.PWM_ET_SOCAEventConfig), (8 bytes).
    Removing plib035_pwm.o(.text.PWM_ET_SOCAPeriodConfig), (30 bytes).
    Removing plib035_pwm.o(.ARM.exidx.text.PWM_ET_SOCAPeriodConfig), (8 bytes).
    Removing plib035_pwm.o(.text.PWM_ET_SOCACmd), (34 bytes).
    Removing plib035_pwm.o(.ARM.exidx.text.PWM_ET_SOCACmd), (8 bytes).
    Removing plib035_pwm.o(.text.PWM_ET_SOCBEventConfig), (34 bytes).
    Removing plib035_pwm.o(.ARM.exidx.text.PWM_ET_SOCBEventConfig), (8 bytes).
    Removing plib035_pwm.o(.text.PWM_ET_SOCBPeriodConfig), (30 bytes).
    Removing plib035_pwm.o(.ARM.exidx.text.PWM_ET_SOCBPeriodConfig), (8 bytes).
    Removing plib035_pwm.o(.text.PWM_ET_SOCBCmd), (34 bytes).
    Removing plib035_pwm.o(.ARM.exidx.text.PWM_ET_SOCBCmd), (8 bytes).
    Removing plib035_pwm.o(.text.PWM_ET_DRQAEventConfig), (34 bytes).
    Removing plib035_pwm.o(.ARM.exidx.text.PWM_ET_DRQAEventConfig), (8 bytes).
    Removing plib035_pwm.o(.text.PWM_ET_DRQAPeriodConfig), (30 bytes).
    Removing plib035_pwm.o(.ARM.exidx.text.PWM_ET_DRQAPeriodConfig), (8 bytes).
    Removing plib035_pwm.o(.text.PWM_ET_DRQACmd), (34 bytes).
    Removing plib035_pwm.o(.ARM.exidx.text.PWM_ET_DRQACmd), (8 bytes).
    Removing plib035_pwm.o(.text.PWM_ET_DRQBEventConfig), (34 bytes).
    Removing plib035_pwm.o(.ARM.exidx.text.PWM_ET_DRQBEventConfig), (8 bytes).
    Removing plib035_pwm.o(.text.PWM_ET_DRQBPeriodConfig), (30 bytes).
    Removing plib035_pwm.o(.ARM.exidx.text.PWM_ET_DRQBPeriodConfig), (8 bytes).
    Removing plib035_pwm.o(.text.PWM_ET_DRQBCmd), (34 bytes).
    Removing plib035_pwm.o(.ARM.exidx.text.PWM_ET_DRQBCmd), (8 bytes).
    Removing plib035_pwm.o(.text.PWM_ET_StructInit), (60 bytes).
    Removing plib035_pwm.o(.ARM.exidx.text.PWM_ET_StructInit), (8 bytes).
    Removing plib035_qep.o(.text), (0 bytes).
    Removing plib035_qep.o(.text.QEP_DeInit), (28 bytes).
    Removing plib035_qep.o(.ARM.exidx.text.QEP_DeInit), (8 bytes).
    Removing plib035_qep.o(.text.RCU_APBRstCmd), (64 bytes).
    Removing plib035_qep.o(.ARM.exidx.text.RCU_APBRstCmd), (8 bytes).
    Removing plib035_qep.o(.text.QEP_PC_Init), (90 bytes).
    Removing plib035_qep.o(.ARM.exidx.text.QEP_PC_Init), (8 bytes).
    Removing plib035_qep.o(.text.QEP_PC_ModeConfig), (38 bytes).
    Removing plib035_qep.o(.ARM.exidx.text.QEP_PC_ModeConfig), (8 bytes).
    Removing plib035_qep.o(.text.QEP_PC_CountRateConfig), (38 bytes).
    Removing plib035_qep.o(.ARM.exidx.text.QEP_PC_CountRateConfig), (8 bytes).
    Removing plib035_qep.o(.text.QEP_PC_ResetEventConfig), (38 bytes).
    Removing plib035_qep.o(.ARM.exidx.text.QEP_PC_ResetEventConfig), (8 bytes).
    Removing plib035_qep.o(.text.QEP_PC_InitEventSConfig), (38 bytes).
    Removing plib035_qep.o(.ARM.exidx.text.QEP_PC_InitEventSConfig), (8 bytes).
    Removing plib035_qep.o(.text.QEP_PC_InitEventIConfig), (38 bytes).
    Removing plib035_qep.o(.ARM.exidx.text.QEP_PC_InitEventIConfig), (8 bytes).
    Removing plib035_qep.o(.text.QEP_PC_LatchEventSConfig), (38 bytes).
    Removing plib035_qep.o(.ARM.exidx.text.QEP_PC_LatchEventSConfig), (8 bytes).
    Removing plib035_qep.o(.text.QEP_PC_LatchEventIConfig), (38 bytes).
    Removing plib035_qep.o(.ARM.exidx.text.QEP_PC_LatchEventIConfig), (8 bytes).
    Removing plib035_qep.o(.text.QEP_PC_SetCount), (20 bytes).
    Removing plib035_qep.o(.ARM.exidx.text.QEP_PC_SetCount), (8 bytes).
    Removing plib035_qep.o(.text.QEP_PC_SetCountInit), (20 bytes).
    Removing plib035_qep.o(.ARM.exidx.text.QEP_PC_SetCountInit), (8 bytes).
    Removing plib035_qep.o(.text.QEP_PC_SetCountMax), (20 bytes).
    Removing plib035_qep.o(.ARM.exidx.text.QEP_PC_SetCountMax), (8 bytes).
    Removing plib035_qep.o(.text.QEP_PC_StructInit), (50 bytes).
    Removing plib035_qep.o(.ARM.exidx.text.QEP_PC_StructInit), (8 bytes).
    Removing plib035_qep.o(.text.QEP_CMP_Init), (66 bytes).
    Removing plib035_qep.o(.ARM.exidx.text.QEP_CMP_Init), (8 bytes).
    Removing plib035_qep.o(.text.QEP_CMP_ShadowLoadCmd), (38 bytes).
    Removing plib035_qep.o(.ARM.exidx.text.QEP_CMP_ShadowLoadCmd), (8 bytes).
    Removing plib035_qep.o(.text.QEP_CMP_LoadEventConfig), (38 bytes).
    Removing plib035_qep.o(.ARM.exidx.text.QEP_CMP_LoadEventConfig), (8 bytes).
    Removing plib035_qep.o(.text.QEP_CMP_OutConfig), (38 bytes).
    Removing plib035_qep.o(.ARM.exidx.text.QEP_CMP_OutConfig), (8 bytes).
    Removing plib035_qep.o(.text.QEP_CMP_OutCmd), (38 bytes).
    Removing plib035_qep.o(.ARM.exidx.text.QEP_CMP_OutCmd), (8 bytes).
    Removing plib035_qep.o(.text.QEP_CMP_OutPolarityConfig), (38 bytes).
    Removing plib035_qep.o(.ARM.exidx.text.QEP_CMP_OutPolarityConfig), (8 bytes).
    Removing plib035_qep.o(.text.QEP_CMP_SetOutWidth), (26 bytes).
    Removing plib035_qep.o(.ARM.exidx.text.QEP_CMP_SetOutWidth), (8 bytes).
    Removing plib035_qep.o(.text.QEP_CMP_SetComp), (20 bytes).
    Removing plib035_qep.o(.ARM.exidx.text.QEP_CMP_SetComp), (8 bytes).
    Removing plib035_qep.o(.text.QEP_CMP_StructInit), (38 bytes).
    Removing plib035_qep.o(.ARM.exidx.text.QEP_CMP_StructInit), (8 bytes).
    Removing plib035_qep.o(.text.QEP_CAP_Init), (60 bytes).
    Removing plib035_qep.o(.ARM.exidx.text.QEP_CAP_Init), (8 bytes).
    Removing plib035_qep.o(.text.QEP_CAP_DivShadowLoadCmd), (38 bytes).
    Removing plib035_qep.o(.ARM.exidx.text.QEP_CAP_DivShadowLoadCmd), (8 bytes).
    Removing plib035_qep.o(.text.QEP_CAP_ResetEventConfig), (38 bytes).
    Removing plib035_qep.o(.ARM.exidx.text.QEP_CAP_ResetEventConfig), (8 bytes).
    Removing plib035_qep.o(.text.QEP_CAP_DivConfig), (44 bytes).
    Removing plib035_qep.o(.ARM.exidx.text.QEP_CAP_DivConfig), (8 bytes).
    Removing plib035_qep.o(.text.QEP_CAP_LatchEventConfig), (38 bytes).
    Removing plib035_qep.o(.ARM.exidx.text.QEP_CAP_LatchEventConfig), (8 bytes).
    Removing plib035_qep.o(.text.QEP_CAP_SetCount), (20 bytes).
    Removing plib035_qep.o(.ARM.exidx.text.QEP_CAP_SetCount), (8 bytes).
    Removing plib035_qep.o(.text.QEP_CAP_SetPeriod), (20 bytes).
    Removing plib035_qep.o(.ARM.exidx.text.QEP_CAP_SetPeriod), (8 bytes).
    Removing plib035_qep.o(.text.QEP_CAP_StructInit), (38 bytes).
    Removing plib035_qep.o(.ARM.exidx.text.QEP_CAP_StructInit), (8 bytes).
    Removing plib035_rcu.o(.text), (0 bytes).
    Removing plib035_rcu.o(.ARM.exidx.text.RCU_GetOSIClkFreq), (8 bytes).
    Removing plib035_rcu.o(.ARM.exidx.text.RCU_GetOSEClkFreq), (8 bytes).
    Removing plib035_rcu.o(.ARM.exidx.text.RCU_GetPLLClkFreq), (8 bytes).
    Removing plib035_rcu.o(.ARM.exidx.text.RCU_GetPLLDivClkFreq), (8 bytes).
    Removing plib035_rcu.o(.text.RCU_GetSysClkFreq), (24 bytes).
    Removing plib035_rcu.o(.ARM.exidx.text.RCU_GetSysClkFreq), (8 bytes).
    Removing plib035_rcu.o(.ARM.exidx.text.RCU_SysClkStatus), (8 bytes).
    Removing plib035_rcu.o(.text.getSysClkFreq), (72 bytes).
    Removing plib035_rcu.o(.ARM.exidx.text.getSysClkFreq), (8 bytes).
    Removing plib035_rcu.o(.ARM.exidx.text.RCU_GetUARTClkFreq), (8 bytes).
    Removing plib035_rcu.o(.ARM.exidx.text.getPeriphClkFreq), (8 bytes).
    Removing plib035_rcu.o(.text.RCU_GetSPIClkFreq), (80 bytes).
    Removing plib035_rcu.o(.ARM.exidx.text.RCU_GetSPIClkFreq), (8 bytes).
    Removing plib035_rcu.o(.text.RCU_GetADCClkFreq), (80 bytes).
    Removing plib035_rcu.o(.ARM.exidx.text.RCU_GetADCClkFreq), (8 bytes).
    Removing plib035_rcu.o(.text.RCU_GetWDTClkFreq), (80 bytes).
    Removing plib035_rcu.o(.ARM.exidx.text.RCU_GetWDTClkFreq), (8 bytes).
    Removing plib035_rcu.o(.text.getSysPeriphClkFreq), (72 bytes).
    Removing plib035_rcu.o(.ARM.exidx.text.getSysPeriphClkFreq), (8 bytes).
    Removing plib035_rcu.o(.text.RCU_GetTraceClkFreq), (80 bytes).
    Removing plib035_rcu.o(.ARM.exidx.text.RCU_GetTraceClkFreq), (8 bytes).
    Removing plib035_rcu.o(.text.RCU_GetClkOutFreq), (80 bytes).
    Removing plib035_rcu.o(.ARM.exidx.text.RCU_GetClkOutFreq), (8 bytes).
    Removing plib035_rcu.o(.ARM.exidx.text.RCU_PLL_AutoConfig), (8 bytes).
    Removing plib035_rcu.o(.ARM.exidx.text.RCU_PLL_StructInit), (8 bytes).
    Removing plib035_rcu.o(.ARM.exidx.text.RCU_PLL_Init), (8 bytes).
    Removing plib035_rcu.o(.ARM.exidx.text.MFLASH_LatencyConfig), (8 bytes).
    Removing plib035_rcu.o(.ARM.exidx.text.RCU_SysClkChangeCmd), (8 bytes).
    Removing plib035_rcu.o(.ARM.exidx.text.RCU_PLL_OutCmd), (8 bytes).
    Removing plib035_rcu.o(.ARM.exidx.text.RCU_PLL_LockStatus), (8 bytes).
    Removing plib035_rcu.o(.text.RCU_PLL_DeInit), (38 bytes).
    Removing plib035_rcu.o(.ARM.exidx.text.RCU_PLL_DeInit), (8 bytes).
    Removing plib035_rcu.o(.ARM.exidx.text.RCU_SysClkConfig), (8 bytes).
    Removing plib035_rcu.o(.ARM.exidx.text.RCU_BusyStatus), (8 bytes).
    Removing plib035_spi.o(.text), (0 bytes).
    Removing plib035_spi.o(.text.SPI_DeInit), (16 bytes).
    Removing plib035_spi.o(.ARM.exidx.text.SPI_DeInit), (8 bytes).
    Removing plib035_spi.o(.text.RCU_SPIRstCmd), (38 bytes).
    Removing plib035_spi.o(.ARM.exidx.text.RCU_SPIRstCmd), (8 bytes).
    Removing plib035_spi.o(.text.SPI_Init), (44 bytes).
    Removing plib035_spi.o(.ARM.exidx.text.SPI_Init), (8 bytes).
    Removing plib035_spi.o(.text.SPI_SCKDivConfig), (46 bytes).
    Removing plib035_spi.o(.ARM.exidx.text.SPI_SCKDivConfig), (8 bytes).
    Removing plib035_spi.o(.text.SPI_DataWidthConfig), (30 bytes).
    Removing plib035_spi.o(.ARM.exidx.text.SPI_DataWidthConfig), (8 bytes).
    Removing plib035_spi.o(.text.SPI_FrameFormatConfig), (38 bytes).
    Removing plib035_spi.o(.ARM.exidx.text.SPI_FrameFormatConfig), (8 bytes).
    Removing plib035_spi.o(.text.SPI_ModeConfig), (38 bytes).
    Removing plib035_spi.o(.ARM.exidx.text.SPI_ModeConfig), (8 bytes).
    Removing plib035_spi.o(.text.SPI_StructInit), (34 bytes).
    Removing plib035_spi.o(.ARM.exidx.text.SPI_StructInit), (8 bytes).
    Removing plib035_tmr.o(.text), (0 bytes).
    Removing plib035_tmr.o(.ARM.exidx.text.TMR_PeriodConfig), (8 bytes).
    Removing plib035_tmr.o(.ARM.exidx.text.TMR_SetLoad), (8 bytes).
    Removing plib035_tmr.o(.ARM.exidx.text.TMR_FreqConfig), (8 bytes).
    Removing plib035_uart.o(.text), (0 bytes).
    Removing plib035_uart.o(.ARM.exidx.text.UART_AutoBaudConfig), (8 bytes).
    Removing plib035_uart.o(.ARM.exidx.text.UART_BaudDivConfig), (8 bytes).
    Removing plib035_uart.o(.ARM.exidx.text.UART_DeInit), (8 bytes).
    Removing plib035_uart.o(.ARM.exidx.text.RCU_UARTRstCmd), (8 bytes).
    Removing plib035_uart.o(.ARM.exidx.text.UART_Init), (8 bytes).
    Removing plib035_uart.o(.ARM.exidx.text.UART_DataWidthConfig), (8 bytes).
    Removing plib035_uart.o(.ARM.exidx.text.UART_StopBitConfig), (8 bytes).
    Removing plib035_uart.o(.ARM.exidx.text.UART_ParityBitConfig), (8 bytes).
    Removing plib035_uart.o(.ARM.exidx.text.UART_FIFOCmd), (8 bytes).
    Removing plib035_uart.o(.ARM.exidx.text.UART_TxCmd), (8 bytes).
    Removing plib035_uart.o(.ARM.exidx.text.UART_RxCmd), (8 bytes).
    Removing plib035_uart.o(.text.UART_StructInit), (44 bytes).
    Removing plib035_uart.o(.ARM.exidx.text.UART_StructInit), (8 bytes).
    Removing plib035_wdt.o(.text), (0 bytes).
    Removing retarget.o(.text), (0 bytes).
    Removing retarget_conf.o(.text), (0 bytes).
    Removing retarget_conf.o(.text.retarget_init), (2 bytes).
    Removing retarget_conf.o(.ARM.exidx.text.retarget_init), (8 bytes).
    Removing retarget_conf.o(.text.retarget_get_char), (4 bytes).
    Removing retarget_conf.o(.ARM.exidx.text.retarget_get_char), (8 bytes).
    Removing retarget_conf.o(.text.retarget_put_char), (10 bytes).
    Removing retarget_conf.o(.ARM.exidx.text.retarget_put_char), (8 bytes).

746 unused section(s) (total 28924 bytes) removed from the image.

==============================================================================

Image Symbol Table

    Local Symbols

    Symbol Name                              Value     Ov Type        Size  Object(Section)

    ../clib/angel/boardlib.s                 0x00000000   Number         0  boardinit1.o ABSOLUTE
    ../clib/angel/boardlib.s                 0x00000000   Number         0  boardinit2.o ABSOLUTE
    ../clib/angel/boardlib.s                 0x00000000   Number         0  boardinit3.o ABSOLUTE
    ../clib/angel/boardlib.s                 0x00000000   Number         0  boardshut.o ABSOLUTE
    ../clib/angel/dczerorl2.s                0x00000000   Number         0  __dczerorl2.o ABSOLUTE
    ../clib/angel/handlers.s                 0x00000000   Number         0  __scatter_zi.o ABSOLUTE
    ../clib/angel/kernel.s                   0x00000000   Number         0  __rtentry.o ABSOLUTE
    ../clib/angel/kernel.s                   0x00000000   Number         0  __rtentry2.o ABSOLUTE
    ../clib/angel/kernel.s                   0x00000000   Number         0  __rtentry4.o ABSOLUTE
    ../clib/angel/kernel.s                   0x00000000   Number         0  rtexit.o ABSOLUTE
    ../clib/angel/kernel.s                   0x00000000   Number         0  rtexit2.o ABSOLUTE
    ../clib/angel/rt.s                       0x00000000   Number         0  aeabi_ldiv0.o ABSOLUTE
    ../clib/angel/rt.s                       0x00000000   Number         0  aeabi_ldiv0_sigfpe.o ABSOLUTE
    ../clib/angel/rt.s                       0x00000000   Number         0  rt_div0.o ABSOLUTE
    ../clib/angel/rt.s                       0x00000000   Number         0  rt_errno_addr.o ABSOLUTE
    ../clib/angel/rt.s                       0x00000000   Number         0  rt_errno_addr_intlibspace.o ABSOLUTE
    ../clib/angel/rt.s                       0x00000000   Number         0  rt_raise.o ABSOLUTE
    ../clib/angel/scatter.s                  0x00000000   Number         0  __scatter.o ABSOLUTE
    ../clib/angel/startup.s                  0x00000000   Number         0  __main.o ABSOLUTE
    ../clib/angel/sys.s                      0x00000000   Number         0  libspace.o ABSOLUTE
    ../clib/angel/sys.s                      0x00000000   Number         0  sys_stackheap_outer.o ABSOLUTE
    ../clib/angel/sys.s                      0x00000000   Number         0  use_no_semi.o ABSOLUTE
    ../clib/angel/sys.s                      0x00000000   Number         0  indicate_semi.o ABSOLUTE
    ../clib/angel/sysapp.c                   0x00000000   Number         0  sys_exit.o ABSOLUTE
    ../clib/angel/sysapp.c                   0x00000000   Number         0  sys_exit_hlt.o ABSOLUTE
    ../clib/angel/sysapp.c                   0x00000000   Number         0  sys_wrch.o ABSOLUTE
    ../clib/angel/sysapp.c                   0x00000000   Number         0  sys_wrch_hlt.o ABSOLUTE
    ../clib/angel/sysapp.c                   0x00000000   Number         0  sys_command.o ABSOLUTE
    ../clib/angel/sysapp.c                   0x00000000   Number         0  sys_command_hlt.o ABSOLUTE
    ../clib/armsys.c                         0x00000000   Number         0  argv_veneer.o ABSOLUTE
    ../clib/armsys.c                         0x00000000   Number         0  argv_veneer.o ABSOLUTE
    ../clib/armsys.c                         0x00000000   Number         0  _get_argv_nomalloc.o ABSOLUTE
    ../clib/armsys.c                         0x00000000   Number         0  no_argv.o ABSOLUTE
    ../clib/fenv.c                           0x00000000   Number         0  _rserrno.o ABSOLUTE
    ../clib/heapalloc.c                      0x00000000   Number         0  hrguard.o ABSOLUTE
    ../clib/heapaux.c                        0x00000000   Number         0  heapauxi.o ABSOLUTE
    ../clib/libinit.s                        0x00000000   Number         0  libinit.o ABSOLUTE
    ../clib/libinit.s                        0x00000000   Number         0  libinit2.o ABSOLUTE
    ../clib/libinit.s                        0x00000000   Number         0  libshutdown.o ABSOLUTE
    ../clib/libinit.s                        0x00000000   Number         0  libshutdown2.o ABSOLUTE
    ../clib/longlong.s                       0x00000000   Number         0  llsdiv.o ABSOLUTE
    ../clib/longlong.s                       0x00000000   Number         0  lludivv7m.o ABSOLUTE
    ../clib/memcpset.s                       0x00000000   Number         0  rt_memcpy_v6.o ABSOLUTE
    ../clib/memcpset.s                       0x00000000   Number         0  rt_memcpy_w.o ABSOLUTE
    ../clib/memcpset.s                       0x00000000   Number         0  rt_memclr_w.o ABSOLUTE
    ../clib/signal.c                         0x00000000   Number         0  defsig_fpe_outer.o ABSOLUTE
    ../clib/signal.c                         0x00000000   Number         0  defsig_fpe_formal.o ABSOLUTE
    ../clib/signal.c                         0x00000000   Number         0  defsig_exit.o ABSOLUTE
    ../clib/signal.c                         0x00000000   Number         0  defsig_fpe_inner.o ABSOLUTE
    ../clib/signal.c                         0x00000000   Number         0  __raise.o ABSOLUTE
    ../clib/signal.c                         0x00000000   Number         0  defsig_general.o ABSOLUTE
    ../clib/signal.c                         0x00000000   Number         0  defsig_abrt_inner.o ABSOLUTE
    ../clib/signal.c                         0x00000000   Number         0  defsig_rtred_inner.o ABSOLUTE
    ../clib/signal.c                         0x00000000   Number         0  defsig_rtmem_inner.o ABSOLUTE
    ../clib/signal.c                         0x00000000   Number         0  defsig_rtmem_outer.o ABSOLUTE
    ../clib/signal.c                         0x00000000   Number         0  defsig_rtmem_formal.o ABSOLUTE
    ../clib/signal.c                         0x00000000   Number         0  defsig_stak_inner.o ABSOLUTE
    ../clib/signal.c                         0x00000000   Number         0  defsig_pvfn_inner.o ABSOLUTE
    ../clib/signal.c                         0x00000000   Number         0  defsig_cppl_inner.o ABSOLUTE
    ../clib/signal.c                         0x00000000   Number         0  defsig_segv_inner.o ABSOLUTE
    ../clib/signal.c                         0x00000000   Number         0  defsig_other.o ABSOLUTE
    ../clib/signal.s                         0x00000000   Number         0  defsig.o ABSOLUTE
    ../clib/stdlib.c                         0x00000000   Number         0  qsortnoex.o ABSOLUTE
    ../clib/stdlib.c                         0x00000000   Number         0  exit.o ABSOLUTE
    ../clib/string.c                         0x00000000   Number         0  strlen.o ABSOLUTE
    ../fplib/ffltll.s                        0x00000000   Number         0  ffltll_clz.o ABSOLUTE
    ../fplib/fpinit.s                        0x00000000   Number         0  fpinit.o ABSOLUTE
    ../fplib/usenofp.s                       0x00000000   Number         0  usenofp.o ABSOLUTE
    ../mathlib/cosf.c                        0x00000000   Number         0  cosf.o ABSOLUTE
    ../mathlib/fpclassifyf.c                 0x00000000   Number         0  fpclassifyf.o ABSOLUTE
    ../mathlib/funder.c                      0x00000000   Number         0  funder.o ABSOLUTE
    ../mathlib/rredf.c                       0x00000000   Number         0  rredf.o ABSOLUTE
    ../mathlib/sinf.c                        0x00000000   Number         0  sinf.o ABSOLUTE
    SEGGER_RTT.c                             0x00000000   Number         0  segger_rtt.o ABSOLUTE
    SEGGER_RTT_printf.c                      0x00000000   Number         0  segger_rtt_printf.o ABSOLUTE
    dc.s                                     0x00000000   Number         0  dc.o ABSOLUTE
    filters.c                                0x00000000   Number         0  filters.o ABSOLUTE
    gpio.c                                   0x00000000   Number         0  gpio.o ABSOLUTE
    main.c                                   0x00000000   Number         0  main.o ABSOLUTE
    platform\Device\NIIET\K1921VK035\Source\ARM\startup_K1921VK035.s 0x00000000   Number         0  startup_k1921vk035.o ABSOLUTE
    plib035_adc.c                            0x00000000   Number         0  plib035_adc.o ABSOLUTE
    plib035_can.c                            0x00000000   Number         0  plib035_can.o ABSOLUTE
    plib035_dma.c                            0x00000000   Number         0  plib035_dma.o ABSOLUTE
    plib035_ecap.c                           0x00000000   Number         0  plib035_ecap.o ABSOLUTE
    plib035_gpio.c                           0x00000000   Number         0  plib035_gpio.o ABSOLUTE
    plib035_i2c.c                            0x00000000   Number         0  plib035_i2c.o ABSOLUTE
    plib035_mflash.c                         0x00000000   Number         0  plib035_mflash.o ABSOLUTE
    plib035_pmu.c                            0x00000000   Number         0  plib035_pmu.o ABSOLUTE
    plib035_pwm.c                            0x00000000   Number         0  plib035_pwm.o ABSOLUTE
    plib035_qep.c                            0x00000000   Number         0  plib035_qep.o ABSOLUTE
    plib035_rcu.c                            0x00000000   Number         0  plib035_rcu.o ABSOLUTE
    plib035_spi.c                            0x00000000   Number         0  plib035_spi.o ABSOLUTE
    plib035_tmr.c                            0x00000000   Number         0  plib035_tmr.o ABSOLUTE
    plib035_uart.c                           0x00000000   Number         0  plib035_uart.o ABSOLUTE
    plib035_wdt.c                            0x00000000   Number         0  plib035_wdt.o ABSOLUTE
    retarget.c                               0x00000000   Number         0  retarget.o ABSOLUTE
    retarget_conf.c                          0x00000000   Number         0  retarget_conf.o ABSOLUTE
    sysclk.c                                 0x00000000   Number         0  sysclk.o ABSOLUTE
    system_K1921VK035.c                      0x00000000   Number         0  system_k1921vk035.o ABSOLUTE
    tmr.c                                    0x00000000   Number         0  tmr.o ABSOLUTE
    uart.c                                   0x00000000   Number         0  uart.o ABSOLUTE
    vk035_it.c                               0x00000000   Number         0  vk035_it.o ABSOLUTE
    RESET                                    0x00000000   Section      344  startup_k1921vk035.o(RESET)
    !!!main                                  0x00000158   Section        8  __main.o(!!!main)
    !!!scatter                               0x00000160   Section       52  __scatter.o(!!!scatter)
    !!dczerorl2                              0x00000194   Section       90  __dczerorl2.o(!!dczerorl2)
    !!handler_zi                             0x000001f0   Section       28  __scatter_zi.o(!!handler_zi)
    .ARM.Collect$$libinit$$00000000          0x0000020c   Section        2  libinit.o(.ARM.Collect$$libinit$$00000000)
    .ARM.Collect$$libinit$$00000001          0x0000020e   Section        4  libinit2.o(.ARM.Collect$$libinit$$00000001)
    .ARM.Collect$$libinit$$00000004          0x00000212   Section        0  libinit2.o(.ARM.Collect$$libinit$$00000004)
    .ARM.Collect$$libinit$$00000006          0x00000212   Section        0  libinit2.o(.ARM.Collect$$libinit$$00000006)
    .ARM.Collect$$libinit$$0000000C          0x00000212   Section        0  libinit2.o(.ARM.Collect$$libinit$$0000000C)
    .ARM.Collect$$libinit$$0000000E          0x00000212   Section        0  libinit2.o(.ARM.Collect$$libinit$$0000000E)
    .ARM.Collect$$libinit$$00000010          0x00000212   Section        0  libinit2.o(.ARM.Collect$$libinit$$00000010)
    .ARM.Collect$$libinit$$00000013          0x00000212   Section        0  libinit2.o(.ARM.Collect$$libinit$$00000013)
    .ARM.Collect$$libinit$$00000015          0x00000212   Section        0  libinit2.o(.ARM.Collect$$libinit$$00000015)
    .ARM.Collect$$libinit$$00000017          0x00000212   Section        0  libinit2.o(.ARM.Collect$$libinit$$00000017)
    .ARM.Collect$$libinit$$00000019          0x00000212   Section        0  libinit2.o(.ARM.Collect$$libinit$$00000019)
    .ARM.Collect$$libinit$$0000001B          0x00000212   Section        0  libinit2.o(.ARM.Collect$$libinit$$0000001B)
    .ARM.Collect$$libinit$$0000001D          0x00000212   Section        0  libinit2.o(.ARM.Collect$$libinit$$0000001D)
    .ARM.Collect$$libinit$$0000001F          0x00000212   Section        0  libinit2.o(.ARM.Collect$$libinit$$0000001F)
    .ARM.Collect$$libinit$$00000021          0x00000212   Section        0  libinit2.o(.ARM.Collect$$libinit$$00000021)
    .ARM.Collect$$libinit$$00000023          0x00000212   Section        0  libinit2.o(.ARM.Collect$$libinit$$00000023)
    .ARM.Collect$$libinit$$00000025          0x00000212   Section        0  libinit2.o(.ARM.Collect$$libinit$$00000025)
    .ARM.Collect$$libinit$$00000027          0x00000212   Section        0  libinit2.o(.ARM.Collect$$libinit$$00000027)
    .ARM.Collect$$libinit$$0000002E          0x00000212   Section        0  libinit2.o(.ARM.Collect$$libinit$$0000002E)
    .ARM.Collect$$libinit$$00000030          0x00000212   Section        0  libinit2.o(.ARM.Collect$$libinit$$00000030)
    .ARM.Collect$$libinit$$00000032          0x00000212   Section        0  libinit2.o(.ARM.Collect$$libinit$$00000032)
    .ARM.Collect$$libinit$$00000034          0x00000212   Section        0  libinit2.o(.ARM.Collect$$libinit$$00000034)
    .ARM.Collect$$libinit$$00000035          0x00000212   Section        2  libinit2.o(.ARM.Collect$$libinit$$00000035)
    .ARM.Collect$$libshutdown$$00000000      0x00000214   Section        2  libshutdown.o(.ARM.Collect$$libshutdown$$00000000)
    .ARM.Collect$$libshutdown$$00000002      0x00000216   Section        0  libshutdown2.o(.ARM.Collect$$libshutdown$$00000002)
    .ARM.Collect$$libshutdown$$00000004      0x00000216   Section        0  libshutdown2.o(.ARM.Collect$$libshutdown$$00000004)
    .ARM.Collect$$libshutdown$$00000007      0x00000216   Section        0  libshutdown2.o(.ARM.Collect$$libshutdown$$00000007)
    .ARM.Collect$$libshutdown$$0000000A      0x00000216   Section        0  libshutdown2.o(.ARM.Collect$$libshutdown$$0000000A)
    .ARM.Collect$$libshutdown$$0000000C      0x00000216   Section        0  libshutdown2.o(.ARM.Collect$$libshutdown$$0000000C)
    .ARM.Collect$$libshutdown$$0000000F      0x00000216   Section        0  libshutdown2.o(.ARM.Collect$$libshutdown$$0000000F)
    .ARM.Collect$$libshutdown$$00000010      0x00000216   Section        2  libshutdown2.o(.ARM.Collect$$libshutdown$$00000010)
    .ARM.Collect$$rtentry$$00000000          0x00000218   Section        0  __rtentry.o(.ARM.Collect$$rtentry$$00000000)
    .ARM.Collect$$rtentry$$00000002          0x00000218   Section        0  __rtentry2.o(.ARM.Collect$$rtentry$$00000002)
    .ARM.Collect$$rtentry$$00000004          0x00000218   Section        6  __rtentry4.o(.ARM.Collect$$rtentry$$00000004)
    .ARM.Collect$$rtentry$$00000009          0x0000021e   Section        0  __rtentry2.o(.ARM.Collect$$rtentry$$00000009)
    .ARM.Collect$$rtentry$$0000000A          0x0000021e   Section        4  __rtentry2.o(.ARM.Collect$$rtentry$$0000000A)
    .ARM.Collect$$rtentry$$0000000C          0x00000222   Section        0  __rtentry2.o(.ARM.Collect$$rtentry$$0000000C)
    .ARM.Collect$$rtentry$$0000000D          0x00000222   Section        8  __rtentry2.o(.ARM.Collect$$rtentry$$0000000D)
    .ARM.Collect$$rtexit$$00000000           0x0000022a   Section        2  rtexit.o(.ARM.Collect$$rtexit$$00000000)
    .ARM.Collect$$rtexit$$00000002           0x0000022c   Section        0  rtexit2.o(.ARM.Collect$$rtexit$$00000002)
    .ARM.Collect$$rtexit$$00000003           0x0000022c   Section        4  rtexit2.o(.ARM.Collect$$rtexit$$00000003)
    .ARM.Collect$$rtexit$$00000004           0x00000230   Section        6  rtexit2.o(.ARM.Collect$$rtexit$$00000004)
    $v0                                      0x00000238   Number         0  startup_k1921vk035.o(.text)
    .text                                    0x00000238   Section       64  startup_k1921vk035.o(.text)
    .text                                    0x00000278   Section        0  heapauxi.o(.text)
    .text                                    0x00000280   Section        8  libspace.o(.text)
    .text                                    0x00000288   Section       74  sys_stackheap_outer.o(.text)
    .text                                    0x000002d2   Section        0  exit.o(.text)
    .text                                    0x000002e4   Section        0  sys_exit.o(.text)
    .text                                    0x000002f0   Section        2  use_no_semi.o(.text)
    .text                                    0x000002f2   Section        0  indicate_semi.o(.text)
    [Anonymous Symbol]                       0x000002f4   Section        0  vk035_it.o(.text.ADC_DC_IRQHandler)
    [Anonymous Symbol]                       0x000002f8   Section        0  vk035_it.o(.text.ADC_SEQ0_IRQHandler)
    [Anonymous Symbol]                       0x000002fc   Section        0  vk035_it.o(.text.ADC_SEQ1_IRQHandler)
    [Anonymous Symbol]                       0x00000300   Section        0  vk035_it.o(.text.BusFault_Handler)
    [Anonymous Symbol]                       0x00000304   Section        0  vk035_it.o(.text.CAN0_IRQHandler)
    [Anonymous Symbol]                       0x00000308   Section        0  vk035_it.o(.text.CAN10_IRQHandler)
    [Anonymous Symbol]                       0x0000030c   Section        0  vk035_it.o(.text.CAN11_IRQHandler)
    [Anonymous Symbol]                       0x00000310   Section        0  vk035_it.o(.text.CAN12_IRQHandler)
    [Anonymous Symbol]                       0x00000314   Section        0  vk035_it.o(.text.CAN13_IRQHandler)
    [Anonymous Symbol]                       0x00000318   Section        0  vk035_it.o(.text.CAN14_IRQHandler)
    [Anonymous Symbol]                       0x0000031c   Section        0  vk035_it.o(.text.CAN15_IRQHandler)
    [Anonymous Symbol]                       0x00000320   Section        0  vk035_it.o(.text.CAN1_IRQHandler)
    [Anonymous Symbol]                       0x00000324   Section        0  vk035_it.o(.text.CAN2_IRQHandler)
    [Anonymous Symbol]                       0x00000328   Section        0  vk035_it.o(.text.CAN3_IRQHandler)
    [Anonymous Symbol]                       0x0000032c   Section        0  vk035_it.o(.text.CAN4_IRQHandler)
    [Anonymous Symbol]                       0x00000330   Section        0  vk035_it.o(.text.CAN5_IRQHandler)
    [Anonymous Symbol]                       0x00000334   Section        0  vk035_it.o(.text.CAN6_IRQHandler)
    [Anonymous Symbol]                       0x00000338   Section        0  vk035_it.o(.text.CAN7_IRQHandler)
    [Anonymous Symbol]                       0x0000033c   Section        0  vk035_it.o(.text.CAN8_IRQHandler)
    [Anonymous Symbol]                       0x00000340   Section        0  vk035_it.o(.text.CAN9_IRQHandler)
    [Anonymous Symbol]                       0x00000344   Section        0  system_k1921vk035.o(.text.ClkInit)
    [Anonymous Symbol]                       0x0000044c   Section        0  vk035_it.o(.text.DMA_CH0_IRQHandler)
    [Anonymous Symbol]                       0x00000450   Section        0  vk035_it.o(.text.DMA_CH10_IRQHandler)
    [Anonymous Symbol]                       0x00000454   Section        0  vk035_it.o(.text.DMA_CH11_IRQHandler)
    [Anonymous Symbol]                       0x00000458   Section        0  vk035_it.o(.text.DMA_CH12_IRQHandler)
    [Anonymous Symbol]                       0x0000045c   Section        0  vk035_it.o(.text.DMA_CH13_IRQHandler)
    [Anonymous Symbol]                       0x00000460   Section        0  vk035_it.o(.text.DMA_CH14_IRQHandler)
    [Anonymous Symbol]                       0x00000464   Section        0  vk035_it.o(.text.DMA_CH15_IRQHandler)
    [Anonymous Symbol]                       0x00000468   Section        0  vk035_it.o(.text.DMA_CH1_IRQHandler)
    [Anonymous Symbol]                       0x0000046c   Section        0  vk035_it.o(.text.DMA_CH2_IRQHandler)
    [Anonymous Symbol]                       0x00000470   Section        0  vk035_it.o(.text.DMA_CH3_IRQHandler)
    [Anonymous Symbol]                       0x00000474   Section        0  vk035_it.o(.text.DMA_CH4_IRQHandler)
    [Anonymous Symbol]                       0x00000478   Section        0  vk035_it.o(.text.DMA_CH5_IRQHandler)
    [Anonymous Symbol]                       0x0000047c   Section        0  vk035_it.o(.text.DMA_CH6_IRQHandler)
    [Anonymous Symbol]                       0x00000480   Section        0  vk035_it.o(.text.DMA_CH7_IRQHandler)
    [Anonymous Symbol]                       0x00000484   Section        0  vk035_it.o(.text.DMA_CH8_IRQHandler)
    [Anonymous Symbol]                       0x00000488   Section        0  vk035_it.o(.text.DMA_CH9_IRQHandler)
    [Anonymous Symbol]                       0x0000048c   Section        0  vk035_it.o(.text.DebugMon_Handler)
    [Anonymous Symbol]                       0x00000490   Section        0  vk035_it.o(.text.ECAP0_IRQHandler)
    [Anonymous Symbol]                       0x00000494   Section        0  vk035_it.o(.text.ECAP1_IRQHandler)
    [Anonymous Symbol]                       0x00000498   Section        0  vk035_it.o(.text.ECAP2_IRQHandler)
    [Anonymous Symbol]                       0x0000049c   Section        0  main.o(.text.Error_Handler)
    [Anonymous Symbol]                       0x000004ac   Section        0  system_k1921vk035.o(.text.FPUInit)
    [Anonymous Symbol]                       0x000004c4   Section        0  vk035_it.o(.text.FPU_IRQHandler)
    [Anonymous Symbol]                       0x000004c8   Section        0  vk035_it.o(.text.GPIOA_IRQHandler)
    [Anonymous Symbol]                       0x000004cc   Section        0  vk035_it.o(.text.GPIOB_IRQHandler)
    GPIO_AltFuncCmd                          0x000004d1   Thumb Code    40  plib035_gpio.o(.text.GPIO_AltFuncCmd)
    [Anonymous Symbol]                       0x000004d0   Section        0  plib035_gpio.o(.text.GPIO_AltFuncCmd)
    [Anonymous Symbol]                       0x000004f8   Section        0  plib035_gpio.o(.text.GPIO_DeInit)
    GPIO_DigitalCmd                          0x0000052d   Thumb Code    40  plib035_gpio.o(.text.GPIO_DigitalCmd)
    [Anonymous Symbol]                       0x0000052c   Section        0  plib035_gpio.o(.text.GPIO_DigitalCmd)
    [Anonymous Symbol]                       0x00000554   Section        0  plib035_gpio.o(.text.GPIO_DriveModeConfig)
    [Anonymous Symbol]                       0x00000574   Section        0  plib035_gpio.o(.text.GPIO_InModeConfig)
    [Anonymous Symbol]                       0x00000594   Section        0  plib035_gpio.o(.text.GPIO_Init)
    GPIO_ModeConfig                          0x000005f5   Thumb Code    94  plib035_gpio.o(.text.GPIO_ModeConfig)
    [Anonymous Symbol]                       0x000005f4   Section        0  plib035_gpio.o(.text.GPIO_ModeConfig)
    GPIO_OutCmd                              0x00000655   Thumb Code    40  plib035_gpio.o(.text.GPIO_OutCmd)
    [Anonymous Symbol]                       0x00000654   Section        0  plib035_gpio.o(.text.GPIO_OutCmd)
    [Anonymous Symbol]                       0x0000067c   Section        0  plib035_gpio.o(.text.GPIO_OutModeConfig)
    [Anonymous Symbol]                       0x0000069c   Section        0  plib035_gpio.o(.text.GPIO_PullModeConfig)
    [Anonymous Symbol]                       0x000006bc   Section        0  plib035_gpio.o(.text.GPIO_StructInit)
    GPIO_ToggleBits                          0x000006ed   Thumb Code    16  main.o(.text.GPIO_ToggleBits)
    [Anonymous Symbol]                       0x000006ec   Section        0  main.o(.text.GPIO_ToggleBits)
    [Anonymous Symbol]                       0x000006fc   Section        0  vk035_it.o(.text.HardFault_Handler)
    [Anonymous Symbol]                       0x00000700   Section        0  vk035_it.o(.text.I2C_IRQHandler)
    [Anonymous Symbol]                       0x00000704   Section        0  vk035_it.o(.text.MFLASH_IRQHandler)
    MFLASH_LatencyConfig                     0x00000709   Thumb Code    32  plib035_rcu.o(.text.MFLASH_LatencyConfig)
    [Anonymous Symbol]                       0x00000708   Section        0  plib035_rcu.o(.text.MFLASH_LatencyConfig)
    [Anonymous Symbol]                       0x00000728   Section        0  vk035_it.o(.text.MemManage_Handler)
    [Anonymous Symbol]                       0x0000072c   Section        0  vk035_it.o(.text.NMI_Handler)
    [Anonymous Symbol]                       0x00000730   Section        0  vk035_it.o(.text.PWM0_HD_IRQHandler)
    [Anonymous Symbol]                       0x00000734   Section        0  vk035_it.o(.text.PWM0_IRQHandler)
    [Anonymous Symbol]                       0x00000738   Section        0  vk035_it.o(.text.PWM0_TZ_IRQHandler)
    [Anonymous Symbol]                       0x0000073c   Section        0  vk035_it.o(.text.PWM1_HD_IRQHandler)
    [Anonymous Symbol]                       0x00000740   Section        0  vk035_it.o(.text.PWM1_IRQHandler)
    [Anonymous Symbol]                       0x00000744   Section        0  vk035_it.o(.text.PWM1_TZ_IRQHandler)
    [Anonymous Symbol]                       0x00000748   Section        0  vk035_it.o(.text.PWM2_HD_IRQHandler)
    [Anonymous Symbol]                       0x0000074c   Section        0  vk035_it.o(.text.PWM2_IRQHandler)
    [Anonymous Symbol]                       0x00000750   Section        0  vk035_it.o(.text.PWM2_TZ_IRQHandler)
    [Anonymous Symbol]                       0x00000754   Section        0  vk035_it.o(.text.PendSV_Handler)
    [Anonymous Symbol]                       0x00000758   Section        0  vk035_it.o(.text.QEP_IRQHandler)
    RCU_AHBClkCmd                            0x0000075d   Thumb Code    64  gpio.o(.text.RCU_AHBClkCmd)
    [Anonymous Symbol]                       0x0000075c   Section        0  gpio.o(.text.RCU_AHBClkCmd)
    RCU_AHBRstCmd                            0x0000079d   Thumb Code    64  gpio.o(.text.RCU_AHBRstCmd)
    [Anonymous Symbol]                       0x0000079c   Section        0  gpio.o(.text.RCU_AHBRstCmd)
    RCU_AHBRstCmd                            0x000007dd   Thumb Code    64  plib035_gpio.o(.text.RCU_AHBRstCmd)
    [Anonymous Symbol]                       0x000007dc   Section        0  plib035_gpio.o(.text.RCU_AHBRstCmd)
    RCU_APBClkCmd                            0x0000081d   Thumb Code    64  tmr.o(.text.RCU_APBClkCmd)
    [Anonymous Symbol]                       0x0000081c   Section        0  tmr.o(.text.RCU_APBClkCmd)
    RCU_APBRstCmd                            0x0000085d   Thumb Code    64  tmr.o(.text.RCU_APBRstCmd)
    [Anonymous Symbol]                       0x0000085c   Section        0  tmr.o(.text.RCU_APBRstCmd)
    RCU_BusyStatus                           0x0000089d   Thumb Code    16  plib035_rcu.o(.text.RCU_BusyStatus)
    [Anonymous Symbol]                       0x0000089c   Section        0  plib035_rcu.o(.text.RCU_BusyStatus)
    RCU_ClkOutCmd                            0x000008ad   Thumb Code    48  sysclk.o(.text.RCU_ClkOutCmd)
    [Anonymous Symbol]                       0x000008ac   Section        0  sysclk.o(.text.RCU_ClkOutCmd)
    RCU_ClkOutConfig                         0x000008dd   Thumb Code    60  sysclk.o(.text.RCU_ClkOutConfig)
    [Anonymous Symbol]                       0x000008dc   Section        0  sysclk.o(.text.RCU_ClkOutConfig)
    [Anonymous Symbol]                       0x00000918   Section        0  plib035_rcu.o(.text.RCU_GetOSEClkFreq)
    [Anonymous Symbol]                       0x00000924   Section        0  plib035_rcu.o(.text.RCU_GetOSIClkFreq)
    [Anonymous Symbol]                       0x00000930   Section        0  plib035_rcu.o(.text.RCU_GetPLLClkFreq)
    [Anonymous Symbol]                       0x00000990   Section        0  plib035_rcu.o(.text.RCU_GetPLLDivClkFreq)
    [Anonymous Symbol]                       0x000009b4   Section        0  plib035_rcu.o(.text.RCU_GetUARTClkFreq)
    [Anonymous Symbol]                       0x00000a1c   Section        0  vk035_it.o(.text.RCU_IRQHandler)
    [Anonymous Symbol]                       0x00000a20   Section        0  plib035_rcu.o(.text.RCU_PLL_AutoConfig)
    [Anonymous Symbol]                       0x00000ca0   Section        0  plib035_rcu.o(.text.RCU_PLL_Init)
    RCU_PLL_LockStatus                       0x00000d41   Thumb Code    16  plib035_rcu.o(.text.RCU_PLL_LockStatus)
    [Anonymous Symbol]                       0x00000d40   Section        0  plib035_rcu.o(.text.RCU_PLL_LockStatus)
    RCU_PLL_OutCmd                           0x00000d51   Thumb Code    38  plib035_rcu.o(.text.RCU_PLL_OutCmd)
    [Anonymous Symbol]                       0x00000d50   Section        0  plib035_rcu.o(.text.RCU_PLL_OutCmd)
    [Anonymous Symbol]                       0x00000d78   Section        0  plib035_rcu.o(.text.RCU_PLL_StructInit)
    [Anonymous Symbol]                       0x00000d9c   Section        0  plib035_rcu.o(.text.RCU_SysClkChangeCmd)
    RCU_SysClkConfig                         0x00000df9   Thumb Code    30  plib035_rcu.o(.text.RCU_SysClkConfig)
    [Anonymous Symbol]                       0x00000df8   Section        0  plib035_rcu.o(.text.RCU_SysClkConfig)
    RCU_SysClkStatus                         0x00000e19   Thumb Code    16  plib035_rcu.o(.text.RCU_SysClkStatus)
    [Anonymous Symbol]                       0x00000e18   Section        0  plib035_rcu.o(.text.RCU_SysClkStatus)
    RCU_UARTClkCmd                           0x00000e29   Thumb Code    42  uart.o(.text.RCU_UARTClkCmd)
    [Anonymous Symbol]                       0x00000e28   Section        0  uart.o(.text.RCU_UARTClkCmd)
    RCU_UARTClkConfig                        0x00000e55   Thumb Code    76  uart.o(.text.RCU_UARTClkConfig)
    [Anonymous Symbol]                       0x00000e54   Section        0  uart.o(.text.RCU_UARTClkConfig)
    RCU_UARTRstCmd                           0x00000ea1   Thumb Code    50  plib035_uart.o(.text.RCU_UARTRstCmd)
    [Anonymous Symbol]                       0x00000ea0   Section        0  plib035_uart.o(.text.RCU_UARTRstCmd)
    [Anonymous Symbol]                       0x00000ed4   Section        0  vk035_it.o(.text.SPI_RO_RT_IRQHandler)
    [Anonymous Symbol]                       0x00000ed8   Section        0  vk035_it.o(.text.SPI_RX_IRQHandler)
    [Anonymous Symbol]                       0x00000edc   Section        0  vk035_it.o(.text.SPI_TX_IRQHandler)
    [Anonymous Symbol]                       0x00000ee0   Section        0  vk035_it.o(.text.SVC_Handler)
    SysTick_Config                           0x00000ee5   Thumb Code    84  sysclk.o(.text.SysTick_Config)
    [Anonymous Symbol]                       0x00000ee4   Section        0  sysclk.o(.text.SysTick_Config)
    [Anonymous Symbol]                       0x00000f38   Section        0  vk035_it.o(.text.SysTick_Handler)
    [Anonymous Symbol]                       0x00000f40   Section        0  system_k1921vk035.o(.text.SystemCoreClockUpdate)
    [Anonymous Symbol]                       0x00001020   Section        0  system_k1921vk035.o(.text.SystemInit)
    [Anonymous Symbol]                       0x0000102c   Section        0  vk035_it.o(.text.TMR0_IRQHandler)
    [Anonymous Symbol]                       0x0000103c   Section        0  vk035_it.o(.text.TMR1_IRQHandler)
    [Anonymous Symbol]                       0x0000104c   Section        0  vk035_it.o(.text.TMR2_IRQHandler)
    [Anonymous Symbol]                       0x0000105c   Section        0  vk035_it.o(.text.TMR3_IRQHandler)
    TMR_ADCSOCCmd                            0x0000106d   Thumb Code    26  tmr.o(.text.TMR_ADCSOCCmd)
    [Anonymous Symbol]                       0x0000106c   Section        0  tmr.o(.text.TMR_ADCSOCCmd)
    TMR_Cmd                                  0x00001089   Thumb Code    26  tmr.o(.text.TMR_Cmd)
    [Anonymous Symbol]                       0x00001088   Section        0  tmr.o(.text.TMR_Cmd)
    TMR_DMAReqCmd                            0x000010a5   Thumb Code    26  tmr.o(.text.TMR_DMAReqCmd)
    [Anonymous Symbol]                       0x000010a4   Section        0  tmr.o(.text.TMR_DMAReqCmd)
    TMR_ExtInputConfig                       0x000010c1   Thumb Code    30  tmr.o(.text.TMR_ExtInputConfig)
    [Anonymous Symbol]                       0x000010c0   Section        0  tmr.o(.text.TMR_ExtInputConfig)
    [Anonymous Symbol]                       0x000010e0   Section        0  plib035_tmr.o(.text.TMR_FreqConfig)
    TMR_ITCmd                                0x000010fd   Thumb Code    34  tmr.o(.text.TMR_ITCmd)
    [Anonymous Symbol]                       0x000010fc   Section        0  tmr.o(.text.TMR_ITCmd)
    TMR_ITStatus                             0x00001121   Thumb Code    16  tmr.o(.text.TMR_ITStatus)
    [Anonymous Symbol]                       0x00001120   Section        0  tmr.o(.text.TMR_ITStatus)
    TMR_ITStatusClear                        0x00001131   Thumb Code    14  tmr.o(.text.TMR_ITStatusClear)
    [Anonymous Symbol]                       0x00001130   Section        0  tmr.o(.text.TMR_ITStatusClear)
    [Anonymous Symbol]                       0x00001140   Section        0  tmr.o(.text.TMR_Init)
    [Anonymous Symbol]                       0x000011f0   Section        0  plib035_tmr.o(.text.TMR_PeriodConfig)
    TMR_SetLoad                              0x00001219   Thumb Code    16  tmr.o(.text.TMR_SetLoad)
    [Anonymous Symbol]                       0x00001218   Section        0  tmr.o(.text.TMR_SetLoad)
    TMR_SetLoad                              0x00001229   Thumb Code    16  plib035_tmr.o(.text.TMR_SetLoad)
    [Anonymous Symbol]                       0x00001228   Section        0  plib035_tmr.o(.text.TMR_SetLoad)
    [Anonymous Symbol]                       0x00001238   Section        0  vk035_it.o(.text.UART0_E_RT_IRQHandler)
    [Anonymous Symbol]                       0x00001248   Section        0  vk035_it.o(.text.UART0_RX_IRQHandler)
    [Anonymous Symbol]                       0x00001258   Section        0  vk035_it.o(.text.UART0_TD_IRQHandler)
    [Anonymous Symbol]                       0x00001268   Section        0  vk035_it.o(.text.UART0_TX_IRQHandler)
    [Anonymous Symbol]                       0x00001278   Section        0  vk035_it.o(.text.UART1_E_RT_IRQHandler)
    [Anonymous Symbol]                       0x00001288   Section        0  vk035_it.o(.text.UART1_RX_IRQHandler)
    [Anonymous Symbol]                       0x00001298   Section        0  vk035_it.o(.text.UART1_TD_IRQHandler)
    [Anonymous Symbol]                       0x000012a8   Section        0  vk035_it.o(.text.UART1_TX_IRQHandler)
    [Anonymous Symbol]                       0x000012b8   Section        0  plib035_uart.o(.text.UART_AutoBaudConfig)
    UART_BaudDivConfig                       0x00001349   Thumb Code    24  plib035_uart.o(.text.UART_BaudDivConfig)
    [Anonymous Symbol]                       0x00001348   Section        0  plib035_uart.o(.text.UART_BaudDivConfig)
    UART_Cmd                                 0x00001361   Thumb Code    26  uart.o(.text.UART_Cmd)
    [Anonymous Symbol]                       0x00001360   Section        0  uart.o(.text.UART_Cmd)
    UART_DataWidthConfig                     0x0000137d   Thumb Code    34  plib035_uart.o(.text.UART_DataWidthConfig)
    [Anonymous Symbol]                       0x0000137c   Section        0  plib035_uart.o(.text.UART_DataWidthConfig)
    [Anonymous Symbol]                       0x000013a0   Section        0  plib035_uart.o(.text.UART_DeInit)
    UART_ErrorStatusClear                    0x000013e1   Thumb Code    16  uart.o(.text.UART_ErrorStatusClear)
    [Anonymous Symbol]                       0x000013e0   Section        0  uart.o(.text.UART_ErrorStatusClear)
    UART_FIFOCmd                             0x000013f1   Thumb Code    34  plib035_uart.o(.text.UART_FIFOCmd)
    [Anonymous Symbol]                       0x000013f0   Section        0  plib035_uart.o(.text.UART_FIFOCmd)
    UART_FlagStatus                          0x00001415   Thumb Code    24  uart.o(.text.UART_FlagStatus)
    [Anonymous Symbol]                       0x00001414   Section        0  uart.o(.text.UART_FlagStatus)
    UART_ITCmd                               0x0000142d   Thumb Code    54  uart.o(.text.UART_ITCmd)
    [Anonymous Symbol]                       0x0000142c   Section        0  uart.o(.text.UART_ITCmd)
    UART_ITFIFOLevelRxConfig                 0x00001465   Thumb Code    34  uart.o(.text.UART_ITFIFOLevelRxConfig)
    [Anonymous Symbol]                       0x00001464   Section        0  uart.o(.text.UART_ITFIFOLevelRxConfig)
    UART_ITFIFOLevelTxConfig                 0x00001489   Thumb Code    26  uart.o(.text.UART_ITFIFOLevelTxConfig)
    [Anonymous Symbol]                       0x00001488   Section        0  uart.o(.text.UART_ITFIFOLevelTxConfig)
    UART_ITStatusClear                       0x000014a5   Thumb Code    16  uart.o(.text.UART_ITStatusClear)
    [Anonymous Symbol]                       0x000014a4   Section        0  uart.o(.text.UART_ITStatusClear)
    [Anonymous Symbol]                       0x000014b4   Section        0  plib035_uart.o(.text.UART_Init)
    UART_ParityBitConfig                     0x00001509   Thumb Code    30  plib035_uart.o(.text.UART_ParityBitConfig)
    [Anonymous Symbol]                       0x00001508   Section        0  plib035_uart.o(.text.UART_ParityBitConfig)
    UART_RecieveData                         0x00001529   Thumb Code    14  uart.o(.text.UART_RecieveData)
    [Anonymous Symbol]                       0x00001528   Section        0  uart.o(.text.UART_RecieveData)
    UART_RxCmd                               0x00001539   Thumb Code    34  plib035_uart.o(.text.UART_RxCmd)
    [Anonymous Symbol]                       0x00001538   Section        0  plib035_uart.o(.text.UART_RxCmd)
    UART_SendData                            0x0000155d   Thumb Code    16  uart.o(.text.UART_SendData)
    [Anonymous Symbol]                       0x0000155c   Section        0  uart.o(.text.UART_SendData)
    UART_StopBitConfig                       0x0000156d   Thumb Code    34  plib035_uart.o(.text.UART_StopBitConfig)
    [Anonymous Symbol]                       0x0000156c   Section        0  plib035_uart.o(.text.UART_StopBitConfig)
    UART_TxCmd                               0x00001591   Thumb Code    34  plib035_uart.o(.text.UART_TxCmd)
    [Anonymous Symbol]                       0x00001590   Section        0  plib035_uart.o(.text.UART_TxCmd)
    [Anonymous Symbol]                       0x000015b4   Section        0  vk035_it.o(.text.UsageFault_Handler)
    [Anonymous Symbol]                       0x000015b8   Section        0  vk035_it.o(.text.WDT_IRQHandler)
    __NVIC_EnableIRQ                         0x000015bd   Thumb Code    48  tmr.o(.text.__NVIC_EnableIRQ)
    [Anonymous Symbol]                       0x000015bc   Section        0  tmr.o(.text.__NVIC_EnableIRQ)
    __NVIC_EnableIRQ                         0x000015ed   Thumb Code    48  uart.o(.text.__NVIC_EnableIRQ)
    [Anonymous Symbol]                       0x000015ec   Section        0  uart.o(.text.__NVIC_EnableIRQ)
    __NVIC_SetPriority                       0x0000161d   Thumb Code    66  sysclk.o(.text.__NVIC_SetPriority)
    [Anonymous Symbol]                       0x0000161c   Section        0  sysclk.o(.text.__NVIC_SetPriority)
    __uart_fifo_receive                      0x00001661   Thumb Code   166  uart.o(.text.__uart_fifo_receive)
    [Anonymous Symbol]                       0x00001660   Section        0  uart.o(.text.__uart_fifo_receive)
    __uart_fifo_transmit                     0x00001709   Thumb Code   200  uart.o(.text.__uart_fifo_transmit)
    [Anonymous Symbol]                       0x00001708   Section        0  uart.o(.text.__uart_fifo_transmit)
    getPeriphClkFreq                         0x000017d1   Thumb Code    72  plib035_rcu.o(.text.getPeriphClkFreq)
    [Anonymous Symbol]                       0x000017d0   Section        0  plib035_rcu.o(.text.getPeriphClkFreq)
    [Anonymous Symbol]                       0x00001818   Section        0  gpio.o(.text.gpio_get_init)
    [Anonymous Symbol]                       0x000018a0   Section        0  gpio.o(.text.gpio_init)
    [Anonymous Symbol]                       0x0000194c   Section        0  main.o(.text.heartbit)
    [Anonymous Symbol]                       0x0000196c   Section        0  main.o(.text.main)
    [Anonymous Symbol]                       0x000019f8   Section        0  sysclk.o(.text.millis)
    [Anonymous Symbol]                       0x00001a04   Section        0  sysclk.o(.text.millis_inc)
    [Anonymous Symbol]                       0x00001a14   Section        0  main.o(.text.periph_init)
    [Anonymous Symbol]                       0x00001a88   Section        0  main.o(.text.restart_receive)
    [Anonymous Symbol]                       0x00001ab8   Section        0  sysclk.o(.text.sysclk_init)
    [Anonymous Symbol]                       0x00001b0c   Section        0  tmr.o(.text.tmr_delay)
    [Anonymous Symbol]                       0x00001ba4   Section        0  tmr.o(.text.tmr_delay_done)
    [Anonymous Symbol]                       0x00001c30   Section        0  tmr.o(.text.tmr_delay_start)
    [Anonymous Symbol]                       0x00001c68   Section        0  tmr.o(.text.tmr_handler)
    [Anonymous Symbol]                       0x00001cb0   Section        0  tmr.o(.text.tmr_init)
    [Anonymous Symbol]                       0x00001d00   Section        0  tmr.o(.text.tmr_init_first)
    [Anonymous Symbol]                       0x00001de0   Section        0  tmr.o(.text.tmr_set_callback)
    [Anonymous Symbol]                       0x00001e18   Section        0  tmr.o(.text.tmr_start)
    [Anonymous Symbol]                       0x00001e48   Section        0  uart.o(.text.uart1_gpio_init)
    [Anonymous Symbol]                       0x00001ef0   Section        0  uart.o(.text.uart_handler)
    [Anonymous Symbol]                       0x00002004   Section        0  uart.o(.text.uart_init)
    [Anonymous Symbol]                       0x00002054   Section        0  uart.o(.text.uart_init_first)
    [Anonymous Symbol]                       0x000020b4   Section        0  uart.o(.text.uart_receive_it)
    [Anonymous Symbol]                       0x00002124   Section        0  uart.o(.text.uart_set_callback)
    [Anonymous Symbol]                       0x0000219c   Section        0  uart.o(.text.uart_start)
    [Anonymous Symbol]                       0x00002210   Section        0  uart.o(.text.uart_transmit)
    [Anonymous Symbol]                       0x000022a4   Section        0  uart.o(.text.uart_transmit_it)
    $v0                                      0x0000231c   Number         0  fpinit.o(x$fpl$fpinit)
    x$fpl$fpinit                             0x0000231c   Section       26  fpinit.o(x$fpl$fpinit)
    .L.str                                   0x00002336   Data          15  main.o(.rodata.str1.1)
    [Anonymous Symbol]                       0x00002336   Section        0  main.o(.rodata.str1.1)
    SYSCLK_Oscil_Type                        0x20000000   Data           1  sysclk.o(.data.SYSCLK_Oscil_Type)
    [Anonymous Symbol]                       0x20000000   Section        0  sysclk.o(.data.SYSCLK_Oscil_Type)
    gpioa_config                             0x20000004   Data         192  gpio.o(.data.gpioa_config)
    [Anonymous Symbol]                       0x20000004   Section        0  gpio.o(.data.gpioa_config)
    gpiob_config                             0x200000c4   Data         192  gpio.o(.data.gpiob_config)
    [Anonymous Symbol]                       0x200000c4   Section        0  gpio.o(.data.gpiob_config)
    tmr0_config                              0x20000184   Data          28  tmr.o(.data.tmr0_config)
    [Anonymous Symbol]                       0x20000184   Section        0  tmr.o(.data.tmr0_config)
    tmr1_config                              0x200001a0   Data          28  tmr.o(.data.tmr1_config)
    [Anonymous Symbol]                       0x200001a0   Section        0  tmr.o(.data.tmr1_config)
    tmr2_config                              0x200001bc   Data          28  tmr.o(.data.tmr2_config)
    [Anonymous Symbol]                       0x200001bc   Section        0  tmr.o(.data.tmr2_config)
    uart1_config                             0x200001d8   Data          28  uart.o(.data.uart1_config)
    [Anonymous Symbol]                       0x200001d8   Section        0  uart.o(.data.uart1_config)
    .bss                                     0x200001f8   Section       96  libspace.o(.bss)
    Heap_Mem                                 0x200002d0   Data         512  startup_k1921vk035.o(HEAP)
    HEAP                                     0x200002d0   Section      512  startup_k1921vk035.o(HEAP)
    Stack_Mem                                0x200004d0   Data        1024  startup_k1921vk035.o(STACK)
    STACK                                    0x200004d0   Section     1024  startup_k1921vk035.o(STACK)
    __initial_sp                             0x200008d0   Data           0  startup_k1921vk035.o(STACK)

    Global Symbols

    Symbol Name                              Value     Ov Type        Size  Object(Section)

    BuildAttributes$$THM_ISAv4$E$P$D$K$B$S$7EM$VFPi3$EXTD16$VFPS$VFMA$PE$A:L22UL41UL21$X:L11$S22US41US21$IEEE1$IW$~IW$USESV6$~STKCKD$USESV7$~SHL$OTIME$ROPI$IEEEX$EBA8$UX$STANDARDLIB$REQ8$PRES8$EABIv2 0x00000000   Number         0  anon$$obj.o ABSOLUTE
    __Vectors                                0x00000000   Data           4  startup_k1921vk035.o(RESET)
    __ARM_exceptions_init                     - Undefined Weak Reference
    __alloca_initialize                       - Undefined Weak Reference
    __arm_preinit_                            - Undefined Weak Reference
    __arm_relocate_pie_                       - Undefined Weak Reference
    __cpp_initialize__aeabi_                  - Undefined Weak Reference
    __cxa_finalize                            - Undefined Weak Reference
    __rt_locale                               - Undefined Weak Reference
    __sigvec_lookup                           - Undefined Weak Reference
    _atexit_init                              - Undefined Weak Reference
    _call_atexit_fns                          - Undefined Weak Reference
    _clock_init                               - Undefined Weak Reference
    _fp_trap_init                             - Undefined Weak Reference
    _fp_trap_shutdown                         - Undefined Weak Reference
    _get_lc_collate                           - Undefined Weak Reference
    _get_lc_ctype                             - Undefined Weak Reference
    _get_lc_monetary                          - Undefined Weak Reference
    _get_lc_numeric                           - Undefined Weak Reference
    _get_lc_time                              - Undefined Weak Reference
    _getenv_init                              - Undefined Weak Reference
    _handle_redirection                       - Undefined Weak Reference
    _init_alloc                               - Undefined Weak Reference
    _init_user_alloc                          - Undefined Weak Reference
    _initio                                   - Undefined Weak Reference
    _rand_init                                - Undefined Weak Reference
    _signal_finish                            - Undefined Weak Reference
    _signal_init                              - Undefined Weak Reference
    _terminate_alloc                          - Undefined Weak Reference
    _terminate_user_alloc                     - Undefined Weak Reference
    _terminateio                              - Undefined Weak Reference
    __Vectors_End                            0x00000158   Data           0  startup_k1921vk035.o(RESET)
    __Vectors_Size                           0x00000158   Number         0  startup_k1921vk035.o ABSOLUTE
    __main                                   0x00000159   Thumb Code     8  __main.o(!!!main)
    __scatterload                            0x00000161   Thumb Code     0  __scatter.o(!!!scatter)
    __scatterload_rt2                        0x00000161   Thumb Code    44  __scatter.o(!!!scatter)
    __scatterload_rt2_thumb_only             0x00000161   Thumb Code     0  __scatter.o(!!!scatter)
    __scatterload_null                       0x0000016f   Thumb Code     0  __scatter.o(!!!scatter)
    __decompress                             0x00000195   Thumb Code    90  __dczerorl2.o(!!dczerorl2)
    __decompress1                            0x00000195   Thumb Code     0  __dczerorl2.o(!!dczerorl2)
    __scatterload_zeroinit                   0x000001f1   Thumb Code    28  __scatter_zi.o(!!handler_zi)
    __rt_lib_init                            0x0000020d   Thumb Code     0  libinit.o(.ARM.Collect$$libinit$$00000000)
    __rt_lib_init_fp_1                       0x0000020f   Thumb Code     0  libinit2.o(.ARM.Collect$$libinit$$00000001)
    __rt_lib_init_alloca_1                   0x00000213   Thumb Code     0  libinit2.o(.ARM.Collect$$libinit$$00000030)
    __rt_lib_init_argv_1                     0x00000213   Thumb Code     0  libinit2.o(.ARM.Collect$$libinit$$0000002E)
    __rt_lib_init_atexit_1                   0x00000213   Thumb Code     0  libinit2.o(.ARM.Collect$$libinit$$0000001D)
    __rt_lib_init_clock_1                    0x00000213   Thumb Code     0  libinit2.o(.ARM.Collect$$libinit$$00000023)
    __rt_lib_init_cpp_1                      0x00000213   Thumb Code     0  libinit2.o(.ARM.Collect$$libinit$$00000034)
    __rt_lib_init_exceptions_1               0x00000213   Thumb Code     0  libinit2.o(.ARM.Collect$$libinit$$00000032)
    __rt_lib_init_fp_trap_1                  0x00000213   Thumb Code     0  libinit2.o(.ARM.Collect$$libinit$$00000021)
    __rt_lib_init_getenv_1                   0x00000213   Thumb Code     0  libinit2.o(.ARM.Collect$$libinit$$00000025)
    __rt_lib_init_heap_1                     0x00000213   Thumb Code     0  libinit2.o(.ARM.Collect$$libinit$$0000000C)
    __rt_lib_init_lc_collate_1               0x00000213   Thumb Code     0  libinit2.o(.ARM.Collect$$libinit$$00000013)
    __rt_lib_init_lc_ctype_1                 0x00000213   Thumb Code     0  libinit2.o(.ARM.Collect$$libinit$$00000015)
    __rt_lib_init_lc_monetary_1              0x00000213   Thumb Code     0  libinit2.o(.ARM.Collect$$libinit$$00000017)
    __rt_lib_init_lc_numeric_1               0x00000213   Thumb Code     0  libinit2.o(.ARM.Collect$$libinit$$00000019)
    __rt_lib_init_lc_time_1                  0x00000213   Thumb Code     0  libinit2.o(.ARM.Collect$$libinit$$0000001B)
    __rt_lib_init_preinit_1                  0x00000213   Thumb Code     0  libinit2.o(.ARM.Collect$$libinit$$00000006)
    __rt_lib_init_rand_1                     0x00000213   Thumb Code     0  libinit2.o(.ARM.Collect$$libinit$$00000010)
    __rt_lib_init_relocate_pie_1             0x00000213   Thumb Code     0  libinit2.o(.ARM.Collect$$libinit$$00000004)
    __rt_lib_init_return                     0x00000213   Thumb Code     0  libinit2.o(.ARM.Collect$$libinit$$00000035)
    __rt_lib_init_signal_1                   0x00000213   Thumb Code     0  libinit2.o(.ARM.Collect$$libinit$$0000001F)
    __rt_lib_init_stdio_1                    0x00000213   Thumb Code     0  libinit2.o(.ARM.Collect$$libinit$$00000027)
    __rt_lib_init_user_alloc_1               0x00000213   Thumb Code     0  libinit2.o(.ARM.Collect$$libinit$$0000000E)
    __rt_lib_shutdown                        0x00000215   Thumb Code     0  libshutdown.o(.ARM.Collect$$libshutdown$$00000000)
    __rt_lib_shutdown_cpp_1                  0x00000217   Thumb Code     0  libshutdown2.o(.ARM.Collect$$libshutdown$$00000002)
    __rt_lib_shutdown_fp_trap_1              0x00000217   Thumb Code     0  libshutdown2.o(.ARM.Collect$$libshutdown$$00000007)
    __rt_lib_shutdown_heap_1                 0x00000217   Thumb Code     0  libshutdown2.o(.ARM.Collect$$libshutdown$$0000000F)
    __rt_lib_shutdown_return                 0x00000217   Thumb Code     0  libshutdown2.o(.ARM.Collect$$libshutdown$$00000010)
    __rt_lib_shutdown_signal_1               0x00000217   Thumb Code     0  libshutdown2.o(.ARM.Collect$$libshutdown$$0000000A)
    __rt_lib_shutdown_stdio_1                0x00000217   Thumb Code     0  libshutdown2.o(.ARM.Collect$$libshutdown$$00000004)
    __rt_lib_shutdown_user_alloc_1           0x00000217   Thumb Code     0  libshutdown2.o(.ARM.Collect$$libshutdown$$0000000C)
    __rt_entry                               0x00000219   Thumb Code     0  __rtentry.o(.ARM.Collect$$rtentry$$00000000)
    __rt_entry_presh_1                       0x00000219   Thumb Code     0  __rtentry2.o(.ARM.Collect$$rtentry$$00000002)
    __rt_entry_sh                            0x00000219   Thumb Code     0  __rtentry4.o(.ARM.Collect$$rtentry$$00000004)
    __rt_entry_li                            0x0000021f   Thumb Code     0  __rtentry2.o(.ARM.Collect$$rtentry$$0000000A)
    __rt_entry_postsh_1                      0x0000021f   Thumb Code     0  __rtentry2.o(.ARM.Collect$$rtentry$$00000009)
    __rt_entry_main                          0x00000223   Thumb Code     0  __rtentry2.o(.ARM.Collect$$rtentry$$0000000D)
    __rt_entry_postli_1                      0x00000223   Thumb Code     0  __rtentry2.o(.ARM.Collect$$rtentry$$0000000C)
    __rt_exit                                0x0000022b   Thumb Code     0  rtexit.o(.ARM.Collect$$rtexit$$00000000)
    __rt_exit_ls                             0x0000022d   Thumb Code     0  rtexit2.o(.ARM.Collect$$rtexit$$00000003)
    __rt_exit_prels_1                        0x0000022d   Thumb Code     0  rtexit2.o(.ARM.Collect$$rtexit$$00000002)
    __rt_exit_exit                           0x00000231   Thumb Code     0  rtexit2.o(.ARM.Collect$$rtexit$$00000004)
    Reset_Handler                            0x00000239   Thumb Code     8  startup_k1921vk035.o(.text)
    __user_initial_stackheap                 0x00000255   Thumb Code     0  startup_k1921vk035.o(.text)
    __use_two_region_memory                  0x00000279   Thumb Code     2  heapauxi.o(.text)
    __rt_heap_escrow$2region                 0x0000027b   Thumb Code     2  heapauxi.o(.text)
    __rt_heap_expand$2region                 0x0000027d   Thumb Code     2  heapauxi.o(.text)
    __user_libspace                          0x00000281   Thumb Code     8  libspace.o(.text)
    __user_perproc_libspace                  0x00000281   Thumb Code     0  libspace.o(.text)
    __user_perthread_libspace                0x00000281   Thumb Code     0  libspace.o(.text)
    __user_setup_stackheap                   0x00000289   Thumb Code    74  sys_stackheap_outer.o(.text)
    exit                                     0x000002d3   Thumb Code    18  exit.o(.text)
    _sys_exit                                0x000002e5   Thumb Code     8  sys_exit.o(.text)
    __I$use$semihosting                      0x000002f1   Thumb Code     0  use_no_semi.o(.text)
    __use_no_semihosting_swi                 0x000002f1   Thumb Code     2  use_no_semi.o(.text)
    __semihosting_library_function           0x000002f3   Thumb Code     0  indicate_semi.o(.text)
    ADC_DC_IRQHandler                        0x000002f5   Thumb Code     2  vk035_it.o(.text.ADC_DC_IRQHandler)
    ADC_SEQ0_IRQHandler                      0x000002f9   Thumb Code     2  vk035_it.o(.text.ADC_SEQ0_IRQHandler)
    ADC_SEQ1_IRQHandler                      0x000002fd   Thumb Code     2  vk035_it.o(.text.ADC_SEQ1_IRQHandler)
    BusFault_Handler                         0x00000301   Thumb Code     4  vk035_it.o(.text.BusFault_Handler)
    CAN0_IRQHandler                          0x00000305   Thumb Code     2  vk035_it.o(.text.CAN0_IRQHandler)
    CAN10_IRQHandler                         0x00000309   Thumb Code     2  vk035_it.o(.text.CAN10_IRQHandler)
    CAN11_IRQHandler                         0x0000030d   Thumb Code     2  vk035_it.o(.text.CAN11_IRQHandler)
    CAN12_IRQHandler                         0x00000311   Thumb Code     2  vk035_it.o(.text.CAN12_IRQHandler)
    CAN13_IRQHandler                         0x00000315   Thumb Code     2  vk035_it.o(.text.CAN13_IRQHandler)
    CAN14_IRQHandler                         0x00000319   Thumb Code     2  vk035_it.o(.text.CAN14_IRQHandler)
    CAN15_IRQHandler                         0x0000031d   Thumb Code     2  vk035_it.o(.text.CAN15_IRQHandler)
    CAN1_IRQHandler                          0x00000321   Thumb Code     2  vk035_it.o(.text.CAN1_IRQHandler)
    CAN2_IRQHandler                          0x00000325   Thumb Code     2  vk035_it.o(.text.CAN2_IRQHandler)
    CAN3_IRQHandler                          0x00000329   Thumb Code     2  vk035_it.o(.text.CAN3_IRQHandler)
    CAN4_IRQHandler                          0x0000032d   Thumb Code     2  vk035_it.o(.text.CAN4_IRQHandler)
    CAN5_IRQHandler                          0x00000331   Thumb Code     2  vk035_it.o(.text.CAN5_IRQHandler)
    CAN6_IRQHandler                          0x00000335   Thumb Code     2  vk035_it.o(.text.CAN6_IRQHandler)
    CAN7_IRQHandler                          0x00000339   Thumb Code     2  vk035_it.o(.text.CAN7_IRQHandler)
    CAN8_IRQHandler                          0x0000033d   Thumb Code     2  vk035_it.o(.text.CAN8_IRQHandler)
    CAN9_IRQHandler                          0x00000341   Thumb Code     2  vk035_it.o(.text.CAN9_IRQHandler)
    ClkInit                                  0x00000345   Thumb Code   264  system_k1921vk035.o(.text.ClkInit)
    DMA_CH0_IRQHandler                       0x0000044d   Thumb Code     2  vk035_it.o(.text.DMA_CH0_IRQHandler)
    DMA_CH10_IRQHandler                      0x00000451   Thumb Code     2  vk035_it.o(.text.DMA_CH10_IRQHandler)
    DMA_CH11_IRQHandler                      0x00000455   Thumb Code     2  vk035_it.o(.text.DMA_CH11_IRQHandler)
    DMA_CH12_IRQHandler                      0x00000459   Thumb Code     2  vk035_it.o(.text.DMA_CH12_IRQHandler)
    DMA_CH13_IRQHandler                      0x0000045d   Thumb Code     2  vk035_it.o(.text.DMA_CH13_IRQHandler)
    DMA_CH14_IRQHandler                      0x00000461   Thumb Code     2  vk035_it.o(.text.DMA_CH14_IRQHandler)
    DMA_CH15_IRQHandler                      0x00000465   Thumb Code     2  vk035_it.o(.text.DMA_CH15_IRQHandler)
    DMA_CH1_IRQHandler                       0x00000469   Thumb Code     2  vk035_it.o(.text.DMA_CH1_IRQHandler)
    DMA_CH2_IRQHandler                       0x0000046d   Thumb Code     2  vk035_it.o(.text.DMA_CH2_IRQHandler)
    DMA_CH3_IRQHandler                       0x00000471   Thumb Code     2  vk035_it.o(.text.DMA_CH3_IRQHandler)
    DMA_CH4_IRQHandler                       0x00000475   Thumb Code     2  vk035_it.o(.text.DMA_CH4_IRQHandler)
    DMA_CH5_IRQHandler                       0x00000479   Thumb Code     2  vk035_it.o(.text.DMA_CH5_IRQHandler)
    DMA_CH6_IRQHandler                       0x0000047d   Thumb Code     2  vk035_it.o(.text.DMA_CH6_IRQHandler)
    DMA_CH7_IRQHandler                       0x00000481   Thumb Code     2  vk035_it.o(.text.DMA_CH7_IRQHandler)
    DMA_CH8_IRQHandler                       0x00000485   Thumb Code     2  vk035_it.o(.text.DMA_CH8_IRQHandler)
    DMA_CH9_IRQHandler                       0x00000489   Thumb Code     2  vk035_it.o(.text.DMA_CH9_IRQHandler)
    DebugMon_Handler                         0x0000048d   Thumb Code     2  vk035_it.o(.text.DebugMon_Handler)
    ECAP0_IRQHandler                         0x00000491   Thumb Code     2  vk035_it.o(.text.ECAP0_IRQHandler)
    ECAP1_IRQHandler                         0x00000495   Thumb Code     2  vk035_it.o(.text.ECAP1_IRQHandler)
    ECAP2_IRQHandler                         0x00000499   Thumb Code     2  vk035_it.o(.text.ECAP2_IRQHandler)
    Error_Handler                            0x0000049d   Thumb Code    14  main.o(.text.Error_Handler)
    FPUInit                                  0x000004ad   Thumb Code    24  system_k1921vk035.o(.text.FPUInit)
    FPU_IRQHandler                           0x000004c5   Thumb Code     2  vk035_it.o(.text.FPU_IRQHandler)
    GPIOA_IRQHandler                         0x000004c9   Thumb Code     2  vk035_it.o(.text.GPIOA_IRQHandler)
    GPIOB_IRQHandler                         0x000004cd   Thumb Code     2  vk035_it.o(.text.GPIOB_IRQHandler)
    GPIO_DeInit                              0x000004f9   Thumb Code    52  plib035_gpio.o(.text.GPIO_DeInit)
    GPIO_DriveModeConfig                     0x00000555   Thumb Code    30  plib035_gpio.o(.text.GPIO_DriveModeConfig)
    GPIO_InModeConfig                        0x00000575   Thumb Code    30  plib035_gpio.o(.text.GPIO_InModeConfig)
    GPIO_Init                                0x00000595   Thumb Code    96  plib035_gpio.o(.text.GPIO_Init)
    GPIO_OutModeConfig                       0x0000067d   Thumb Code    30  plib035_gpio.o(.text.GPIO_OutModeConfig)
    GPIO_PullModeConfig                      0x0000069d   Thumb Code    30  plib035_gpio.o(.text.GPIO_PullModeConfig)
    GPIO_StructInit                          0x000006bd   Thumb Code    46  plib035_gpio.o(.text.GPIO_StructInit)
    HardFault_Handler                        0x000006fd   Thumb Code     4  vk035_it.o(.text.HardFault_Handler)
    I2C_IRQHandler                           0x00000701   Thumb Code     2  vk035_it.o(.text.I2C_IRQHandler)
    MFLASH_IRQHandler                        0x00000705   Thumb Code     2  vk035_it.o(.text.MFLASH_IRQHandler)
    MemManage_Handler                        0x00000729   Thumb Code     4  vk035_it.o(.text.MemManage_Handler)
    NMI_Handler                              0x0000072d   Thumb Code     4  vk035_it.o(.text.NMI_Handler)
    PWM0_HD_IRQHandler                       0x00000731   Thumb Code     2  vk035_it.o(.text.PWM0_HD_IRQHandler)
    PWM0_IRQHandler                          0x00000735   Thumb Code     2  vk035_it.o(.text.PWM0_IRQHandler)
    PWM0_TZ_IRQHandler                       0x00000739   Thumb Code     2  vk035_it.o(.text.PWM0_TZ_IRQHandler)
    PWM1_HD_IRQHandler                       0x0000073d   Thumb Code     2  vk035_it.o(.text.PWM1_HD_IRQHandler)
    PWM1_IRQHandler                          0x00000741   Thumb Code     2  vk035_it.o(.text.PWM1_IRQHandler)
    PWM1_TZ_IRQHandler                       0x00000745   Thumb Code     2  vk035_it.o(.text.PWM1_TZ_IRQHandler)
    PWM2_HD_IRQHandler                       0x00000749   Thumb Code     2  vk035_it.o(.text.PWM2_HD_IRQHandler)
    PWM2_IRQHandler                          0x0000074d   Thumb Code     2  vk035_it.o(.text.PWM2_IRQHandler)
    PWM2_TZ_IRQHandler                       0x00000751   Thumb Code     2  vk035_it.o(.text.PWM2_TZ_IRQHandler)
    PendSV_Handler                           0x00000755   Thumb Code     2  vk035_it.o(.text.PendSV_Handler)
    QEP_IRQHandler                           0x00000759   Thumb Code     2  vk035_it.o(.text.QEP_IRQHandler)
    RCU_GetOSEClkFreq                        0x00000919   Thumb Code    10  plib035_rcu.o(.text.RCU_GetOSEClkFreq)
    RCU_GetOSIClkFreq                        0x00000925   Thumb Code    10  plib035_rcu.o(.text.RCU_GetOSIClkFreq)
    RCU_GetPLLClkFreq                        0x00000931   Thumb Code    96  plib035_rcu.o(.text.RCU_GetPLLClkFreq)
    RCU_GetPLLDivClkFreq                     0x00000991   Thumb Code    36  plib035_rcu.o(.text.RCU_GetPLLDivClkFreq)
    RCU_GetUARTClkFreq                       0x000009b5   Thumb Code   102  plib035_rcu.o(.text.RCU_GetUARTClkFreq)
    RCU_IRQHandler                           0x00000a1d   Thumb Code     2  vk035_it.o(.text.RCU_IRQHandler)
    RCU_PLL_AutoConfig                       0x00000a21   Thumb Code   638  plib035_rcu.o(.text.RCU_PLL_AutoConfig)
    RCU_PLL_Init                             0x00000ca1   Thumb Code   160  plib035_rcu.o(.text.RCU_PLL_Init)
    RCU_PLL_StructInit                       0x00000d79   Thumb Code    34  plib035_rcu.o(.text.RCU_PLL_StructInit)
    RCU_SysClkChangeCmd                      0x00000d9d   Thumb Code    92  plib035_rcu.o(.text.RCU_SysClkChangeCmd)
    SPI_RO_RT_IRQHandler                     0x00000ed5   Thumb Code     2  vk035_it.o(.text.SPI_RO_RT_IRQHandler)
    SPI_RX_IRQHandler                        0x00000ed9   Thumb Code     2  vk035_it.o(.text.SPI_RX_IRQHandler)
    SPI_TX_IRQHandler                        0x00000edd   Thumb Code     2  vk035_it.o(.text.SPI_TX_IRQHandler)
    SVC_Handler                              0x00000ee1   Thumb Code     2  vk035_it.o(.text.SVC_Handler)
    SysTick_Handler                          0x00000f39   Thumb Code     8  vk035_it.o(.text.SysTick_Handler)
    SystemCoreClockUpdate                    0x00000f41   Thumb Code   222  system_k1921vk035.o(.text.SystemCoreClockUpdate)
    SystemInit                               0x00001021   Thumb Code    12  system_k1921vk035.o(.text.SystemInit)
    TMR0_IRQHandler                          0x0000102d   Thumb Code    16  vk035_it.o(.text.TMR0_IRQHandler)
    TMR1_IRQHandler                          0x0000103d   Thumb Code    16  vk035_it.o(.text.TMR1_IRQHandler)
    TMR2_IRQHandler                          0x0000104d   Thumb Code    16  vk035_it.o(.text.TMR2_IRQHandler)
    TMR3_IRQHandler                          0x0000105d   Thumb Code    16  vk035_it.o(.text.TMR3_IRQHandler)
    TMR_FreqConfig                           0x000010e1   Thumb Code    28  plib035_tmr.o(.text.TMR_FreqConfig)
    TMR_Init                                 0x00001141   Thumb Code   176  tmr.o(.text.TMR_Init)
    TMR_PeriodConfig                         0x000011f1   Thumb Code    40  plib035_tmr.o(.text.TMR_PeriodConfig)
    UART0_E_RT_IRQHandler                    0x00001239   Thumb Code    16  vk035_it.o(.text.UART0_E_RT_IRQHandler)
    UART0_RX_IRQHandler                      0x00001249   Thumb Code    16  vk035_it.o(.text.UART0_RX_IRQHandler)
    UART0_TD_IRQHandler                      0x00001259   Thumb Code    16  vk035_it.o(.text.UART0_TD_IRQHandler)
    UART0_TX_IRQHandler                      0x00001269   Thumb Code    16  vk035_it.o(.text.UART0_TX_IRQHandler)
    UART1_E_RT_IRQHandler                    0x00001279   Thumb Code    16  vk035_it.o(.text.UART1_E_RT_IRQHandler)
    UART1_RX_IRQHandler                      0x00001289   Thumb Code    16  vk035_it.o(.text.UART1_RX_IRQHandler)
    UART1_TD_IRQHandler                      0x00001299   Thumb Code    16  vk035_it.o(.text.UART1_TD_IRQHandler)
    UART1_TX_IRQHandler                      0x000012a9   Thumb Code    16  vk035_it.o(.text.UART1_TX_IRQHandler)
    UART_AutoBaudConfig                      0x000012b9   Thumb Code   144  plib035_uart.o(.text.UART_AutoBaudConfig)
    UART_DeInit                              0x000013a1   Thumb Code    62  plib035_uart.o(.text.UART_DeInit)
    UART_Init                                0x000014b5   Thumb Code    82  plib035_uart.o(.text.UART_Init)
    UsageFault_Handler                       0x000015b5   Thumb Code     4  vk035_it.o(.text.UsageFault_Handler)
    WDT_IRQHandler                           0x000015b9   Thumb Code     2  vk035_it.o(.text.WDT_IRQHandler)
    gpio_get_init                            0x00001819   Thumb Code   136  gpio.o(.text.gpio_get_init)
    gpio_init                                0x000018a1   Thumb Code   172  gpio.o(.text.gpio_init)
    heartbit                                 0x0000194d   Thumb Code    30  main.o(.text.heartbit)
    main                                     0x0000196d   Thumb Code   140  main.o(.text.main)
    millis                                   0x000019f9   Thumb Code    12  sysclk.o(.text.millis)
    millis_inc                               0x00001a05   Thumb Code    16  sysclk.o(.text.millis_inc)
    periph_init                              0x00001a15   Thumb Code   114  main.o(.text.periph_init)
    restart_receive                          0x00001a89   Thumb Code    46  main.o(.text.restart_receive)
    sysclk_init                              0x00001ab9   Thumb Code    84  sysclk.o(.text.sysclk_init)
    tmr_delay                                0x00001b0d   Thumb Code   150  tmr.o(.text.tmr_delay)
    tmr_delay_done                           0x00001ba5   Thumb Code   140  tmr.o(.text.tmr_delay_done)
    tmr_delay_start                          0x00001c31   Thumb Code    54  tmr.o(.text.tmr_delay_start)
    tmr_handler                              0x00001c69   Thumb Code    72  tmr.o(.text.tmr_handler)
    tmr_init                                 0x00001cb1   Thumb Code    80  tmr.o(.text.tmr_init)
    tmr_init_first                           0x00001d01   Thumb Code   222  tmr.o(.text.tmr_init_first)
    tmr_set_callback                         0x00001de1   Thumb Code    56  tmr.o(.text.tmr_set_callback)
    tmr_start                                0x00001e19   Thumb Code    48  tmr.o(.text.tmr_start)
    uart1_gpio_init                          0x00001e49   Thumb Code   166  uart.o(.text.uart1_gpio_init)
    uart_handler                             0x00001ef1   Thumb Code   274  uart.o(.text.uart_handler)
    uart_init                                0x00002005   Thumb Code    80  uart.o(.text.uart_init)
    uart_init_first                          0x00002055   Thumb Code    96  uart.o(.text.uart_init_first)
    uart_receive_it                          0x000020b5   Thumb Code   112  uart.o(.text.uart_receive_it)
    uart_set_callback                        0x00002125   Thumb Code   120  uart.o(.text.uart_set_callback)
    uart_start                               0x0000219d   Thumb Code   114  uart.o(.text.uart_start)
    uart_transmit                            0x00002211   Thumb Code   146  uart.o(.text.uart_transmit)
    uart_transmit_it                         0x000022a5   Thumb Code   120  uart.o(.text.uart_transmit_it)
    _fp_init                                 0x0000231d   Thumb Code    26  fpinit.o(x$fpl$fpinit)
    __fplib_config_fpu_vfp                   0x00002335   Thumb Code     0  fpinit.o(x$fpl$fpinit)
    __fplib_config_pureend_doubles           0x00002335   Thumb Code     0  fpinit.o(x$fpl$fpinit)
    Region$$Table$$Base                      0x00002348   Number         0  anon$$obj.o(Region$$Table)
    Region$$Table$$Limit                     0x00002368   Number         0  anon$$obj.o(Region$$Table)
    __libspace_start                         0x200001f8   Data          96  libspace.o(.bss)
    SystemCoreClock                          0x20000258   Data           4  system_k1921vk035.o(.bss.SystemCoreClock)
    __temporary_stack_top$libspace           0x20000258   Data           0  libspace.o(.bss)
    htmr0                                    0x2000025c   Data           8  tmr.o(.bss.htmr0)
    htmr1                                    0x20000264   Data           8  tmr.o(.bss.htmr1)
    htmr2                                    0x2000026c   Data           8  tmr.o(.bss.htmr2)
    htmr3                                    0x20000274   Data           8  tmr.o(.bss.htmr3)
    huart0                                   0x2000027c   Data          32  uart.o(.bss.huart0)
    huart1                                   0x2000029c   Data          32  uart.o(.bss.huart1)
    rxbuff                                   0x200002bc   Data          10  main.o(.bss.rxbuff)
    uwTick                                   0x200002c8   Data           4  sysclk.o(.bss.uwTick)



==============================================================================

Memory Map of the image

  Image Entry point : 0x00000239

  Load Region LR_1 (Base: 0x00000000, Size: 0x0000255c, Max: 0xffffffff, ABSOLUTE, COMPRESSED[0x000023ac])

    Execution Region ER_RO (Exec base: 0x00000000, Load base: 0x00000000, Size: 0x00002368, Max: 0xffffffff, ABSOLUTE)

    Exec Addr    Load Addr    Size         Type   Attr      Idx    E Section Name        Object

    0x00000000   0x00000000   0x00000158   Data   RO          538    RESET               startup_k1921vk035.o
    0x00000158   0x00000158   0x00000008   Code   RO         1112  * !!!main             c_w.l(__main.o)
    0x00000160   0x00000160   0x00000034   Code   RO         1332    !!!scatter          c_w.l(__scatter.o)
    0x00000194   0x00000194   0x0000005a   Code   RO         1330    !!dczerorl2         c_w.l(__dczerorl2.o)
    0x000001ee   0x000001ee   0x00000002   PAD
    0x000001f0   0x000001f0   0x0000001c   Code   RO         1334    !!handler_zi        c_w.l(__scatter_zi.o)
    0x0000020c   0x0000020c   0x00000002   Code   RO         1195    .ARM.Collect$$libinit$$00000000  c_w.l(libinit.o)
    0x0000020e   0x0000020e   0x00000004   Code   RO         1204    .ARM.Collect$$libinit$$00000001  c_w.l(libinit2.o)
    0x00000212   0x00000212   0x00000000   Code   RO         1207    .ARM.Collect$$libinit$$00000004  c_w.l(libinit2.o)
    0x00000212   0x00000212   0x00000000   Code   RO         1209    .ARM.Collect$$libinit$$00000006  c_w.l(libinit2.o)
    0x00000212   0x00000212   0x00000000   Code   RO         1212    .ARM.Collect$$libinit$$0000000C  c_w.l(libinit2.o)
    0x00000212   0x00000212   0x00000000   Code   RO         1214    .ARM.Collect$$libinit$$0000000E  c_w.l(libinit2.o)
    0x00000212   0x00000212   0x00000000   Code   RO         1216    .ARM.Collect$$libinit$$00000010  c_w.l(libinit2.o)
    0x00000212   0x00000212   0x00000000   Code   RO         1219    .ARM.Collect$$libinit$$00000013  c_w.l(libinit2.o)
    0x00000212   0x00000212   0x00000000   Code   RO         1221    .ARM.Collect$$libinit$$00000015  c_w.l(libinit2.o)
    0x00000212   0x00000212   0x00000000   Code   RO         1223    .ARM.Collect$$libinit$$00000017  c_w.l(libinit2.o)
    0x00000212   0x00000212   0x00000000   Code   RO         1225    .ARM.Collect$$libinit$$00000019  c_w.l(libinit2.o)
    0x00000212   0x00000212   0x00000000   Code   RO         1227    .ARM.Collect$$libinit$$0000001B  c_w.l(libinit2.o)
    0x00000212   0x00000212   0x00000000   Code   RO         1229    .ARM.Collect$$libinit$$0000001D  c_w.l(libinit2.o)
    0x00000212   0x00000212   0x00000000   Code   RO         1231    .ARM.Collect$$libinit$$0000001F  c_w.l(libinit2.o)
    0x00000212   0x00000212   0x00000000   Code   RO         1233    .ARM.Collect$$libinit$$00000021  c_w.l(libinit2.o)
    0x00000212   0x00000212   0x00000000   Code   RO         1235    .ARM.Collect$$libinit$$00000023  c_w.l(libinit2.o)
    0x00000212   0x00000212   0x00000000   Code   RO         1237    .ARM.Collect$$libinit$$00000025  c_w.l(libinit2.o)
    0x00000212   0x00000212   0x00000000   Code   RO         1239    .ARM.Collect$$libinit$$00000027  c_w.l(libinit2.o)
    0x00000212   0x00000212   0x00000000   Code   RO         1243    .ARM.Collect$$libinit$$0000002E  c_w.l(libinit2.o)
    0x00000212   0x00000212   0x00000000   Code   RO         1245    .ARM.Collect$$libinit$$00000030  c_w.l(libinit2.o)
    0x00000212   0x00000212   0x00000000   Code   RO         1247    .ARM.Collect$$libinit$$00000032  c_w.l(libinit2.o)
    0x00000212   0x00000212   0x00000000   Code   RO         1249    .ARM.Collect$$libinit$$00000034  c_w.l(libinit2.o)
    0x00000212   0x00000212   0x00000002   Code   RO         1250    .ARM.Collect$$libinit$$00000035  c_w.l(libinit2.o)
    0x00000214   0x00000214   0x00000002   Code   RO         1285    .ARM.Collect$$libshutdown$$00000000  c_w.l(libshutdown.o)
    0x00000216   0x00000216   0x00000000   Code   RO         1313    .ARM.Collect$$libshutdown$$00000002  c_w.l(libshutdown2.o)
    0x00000216   0x00000216   0x00000000   Code   RO         1315    .ARM.Collect$$libshutdown$$00000004  c_w.l(libshutdown2.o)
    0x00000216   0x00000216   0x00000000   Code   RO         1318    .ARM.Collect$$libshutdown$$00000007  c_w.l(libshutdown2.o)
    0x00000216   0x00000216   0x00000000   Code   RO         1321    .ARM.Collect$$libshutdown$$0000000A  c_w.l(libshutdown2.o)
    0x00000216   0x00000216   0x00000000   Code   RO         1323    .ARM.Collect$$libshutdown$$0000000C  c_w.l(libshutdown2.o)
    0x00000216   0x00000216   0x00000000   Code   RO         1326    .ARM.Collect$$libshutdown$$0000000F  c_w.l(libshutdown2.o)
    0x00000216   0x00000216   0x00000002   Code   RO         1327    .ARM.Collect$$libshutdown$$00000010  c_w.l(libshutdown2.o)
    0x00000218   0x00000218   0x00000000   Code   RO         1128    .ARM.Collect$$rtentry$$00000000  c_w.l(__rtentry.o)
    0x00000218   0x00000218   0x00000000   Code   RO         1158    .ARM.Collect$$rtentry$$00000002  c_w.l(__rtentry2.o)
    0x00000218   0x00000218   0x00000006   Code   RO         1170    .ARM.Collect$$rtentry$$00000004  c_w.l(__rtentry4.o)
    0x0000021e   0x0000021e   0x00000000   Code   RO         1160    .ARM.Collect$$rtentry$$00000009  c_w.l(__rtentry2.o)
    0x0000021e   0x0000021e   0x00000004   Code   RO         1161    .ARM.Collect$$rtentry$$0000000A  c_w.l(__rtentry2.o)
    0x00000222   0x00000222   0x00000000   Code   RO         1163    .ARM.Collect$$rtentry$$0000000C  c_w.l(__rtentry2.o)
    0x00000222   0x00000222   0x00000008   Code   RO         1164    .ARM.Collect$$rtentry$$0000000D  c_w.l(__rtentry2.o)
    0x0000022a   0x0000022a   0x00000002   Code   RO         1196    .ARM.Collect$$rtexit$$00000000  c_w.l(rtexit.o)
    0x0000022c   0x0000022c   0x00000000   Code   RO         1256    .ARM.Collect$$rtexit$$00000002  c_w.l(rtexit2.o)
    0x0000022c   0x0000022c   0x00000004   Code   RO         1257    .ARM.Collect$$rtexit$$00000003  c_w.l(rtexit2.o)
    0x00000230   0x00000230   0x00000006   Code   RO         1258    .ARM.Collect$$rtexit$$00000004  c_w.l(rtexit2.o)
    0x00000236   0x00000236   0x00000002   PAD
    0x00000238   0x00000238   0x00000040   Code   RO          539  * .text               startup_k1921vk035.o
    0x00000278   0x00000278   0x00000006   Code   RO         1110    .text               c_w.l(heapauxi.o)
    0x0000027e   0x0000027e   0x00000002   PAD
    0x00000280   0x00000280   0x00000008   Code   RO         1179    .text               c_w.l(libspace.o)
    0x00000288   0x00000288   0x0000004a   Code   RO         1182    .text               c_w.l(sys_stackheap_outer.o)
    0x000002d2   0x000002d2   0x00000012   Code   RO         1184    .text               c_w.l(exit.o)
    0x000002e4   0x000002e4   0x0000000c   Code   RO         1251    .text               c_w.l(sys_exit.o)
    0x000002f0   0x000002f0   0x00000002   Code   RO         1274    .text               c_w.l(use_no_semi.o)
    0x000002f2   0x000002f2   0x00000000   Code   RO         1276    .text               c_w.l(indicate_semi.o)
    0x000002f2   0x000002f2   0x00000002   PAD
    0x000002f4   0x000002f4   0x00000002   Code   RO          260    .text.ADC_DC_IRQHandler  vk035_it.o
    0x000002f6   0x000002f6   0x00000002   PAD
    0x000002f8   0x000002f8   0x00000002   Code   RO          256    .text.ADC_SEQ0_IRQHandler  vk035_it.o
    0x000002fa   0x000002fa   0x00000002   PAD
    0x000002fc   0x000002fc   0x00000002   Code   RO          258    .text.ADC_SEQ1_IRQHandler  vk035_it.o
    0x000002fe   0x000002fe   0x00000002   PAD
    0x00000300   0x00000300   0x00000004   Code   RO          334    .text.BusFault_Handler  vk035_it.o
    0x00000304   0x00000304   0x00000002   Code   RO          262    .text.CAN0_IRQHandler  vk035_it.o
    0x00000306   0x00000306   0x00000002   PAD
    0x00000308   0x00000308   0x00000002   Code   RO          282    .text.CAN10_IRQHandler  vk035_it.o
    0x0000030a   0x0000030a   0x00000002   PAD
    0x0000030c   0x0000030c   0x00000002   Code   RO          284    .text.CAN11_IRQHandler  vk035_it.o
    0x0000030e   0x0000030e   0x00000002   PAD
    0x00000310   0x00000310   0x00000002   Code   RO          286    .text.CAN12_IRQHandler  vk035_it.o
    0x00000312   0x00000312   0x00000002   PAD
    0x00000314   0x00000314   0x00000002   Code   RO          288    .text.CAN13_IRQHandler  vk035_it.o
    0x00000316   0x00000316   0x00000002   PAD
    0x00000318   0x00000318   0x00000002   Code   RO          290    .text.CAN14_IRQHandler  vk035_it.o
    0x0000031a   0x0000031a   0x00000002   PAD
    0x0000031c   0x0000031c   0x00000002   Code   RO          292    .text.CAN15_IRQHandler  vk035_it.o
    0x0000031e   0x0000031e   0x00000002   PAD
    0x00000320   0x00000320   0x00000002   Code   RO          264    .text.CAN1_IRQHandler  vk035_it.o
    0x00000322   0x00000322   0x00000002   PAD
    0x00000324   0x00000324   0x00000002   Code   RO          266    .text.CAN2_IRQHandler  vk035_it.o
    0x00000326   0x00000326   0x00000002   PAD
    0x00000328   0x00000328   0x00000002   Code   RO          268    .text.CAN3_IRQHandler  vk035_it.o
    0x0000032a   0x0000032a   0x00000002   PAD
    0x0000032c   0x0000032c   0x00000002   Code   RO          270    .text.CAN4_IRQHandler  vk035_it.o
    0x0000032e   0x0000032e   0x00000002   PAD
    0x00000330   0x00000330   0x00000002   Code   RO          272    .text.CAN5_IRQHandler  vk035_it.o
    0x00000332   0x00000332   0x00000002   PAD
    0x00000334   0x00000334   0x00000002   Code   RO          274    .text.CAN6_IRQHandler  vk035_it.o
    0x00000336   0x00000336   0x00000002   PAD
    0x00000338   0x00000338   0x00000002   Code   RO          276    .text.CAN7_IRQHandler  vk035_it.o
    0x0000033a   0x0000033a   0x00000002   PAD
    0x0000033c   0x0000033c   0x00000002   Code   RO          278    .text.CAN8_IRQHandler  vk035_it.o
    0x0000033e   0x0000033e   0x00000002   PAD
    0x00000340   0x00000340   0x00000002   Code   RO          280    .text.CAN9_IRQHandler  vk035_it.o
    0x00000342   0x00000342   0x00000002   PAD
    0x00000344   0x00000344   0x00000108   Code   RO          523    .text.ClkInit       system_k1921vk035.o
    0x0000044c   0x0000044c   0x00000002   Code   RO          296    .text.DMA_CH0_IRQHandler  vk035_it.o
    0x0000044e   0x0000044e   0x00000002   PAD
    0x00000450   0x00000450   0x00000002   Code   RO          316    .text.DMA_CH10_IRQHandler  vk035_it.o
    0x00000452   0x00000452   0x00000002   PAD
    0x00000454   0x00000454   0x00000002   Code   RO          318    .text.DMA_CH11_IRQHandler  vk035_it.o
    0x00000456   0x00000456   0x00000002   PAD
    0x00000458   0x00000458   0x00000002   Code   RO          320    .text.DMA_CH12_IRQHandler  vk035_it.o
    0x0000045a   0x0000045a   0x00000002   PAD
    0x0000045c   0x0000045c   0x00000002   Code   RO          322    .text.DMA_CH13_IRQHandler  vk035_it.o
    0x0000045e   0x0000045e   0x00000002   PAD
    0x00000460   0x00000460   0x00000002   Code   RO          324    .text.DMA_CH14_IRQHandler  vk035_it.o
    0x00000462   0x00000462   0x00000002   PAD
    0x00000464   0x00000464   0x00000002   Code   RO          326    .text.DMA_CH15_IRQHandler  vk035_it.o
    0x00000466   0x00000466   0x00000002   PAD
    0x00000468   0x00000468   0x00000002   Code   RO          298    .text.DMA_CH1_IRQHandler  vk035_it.o
    0x0000046a   0x0000046a   0x00000002   PAD
    0x0000046c   0x0000046c   0x00000002   Code   RO          300    .text.DMA_CH2_IRQHandler  vk035_it.o
    0x0000046e   0x0000046e   0x00000002   PAD
    0x00000470   0x00000470   0x00000002   Code   RO          302    .text.DMA_CH3_IRQHandler  vk035_it.o
    0x00000472   0x00000472   0x00000002   PAD
    0x00000474   0x00000474   0x00000002   Code   RO          304    .text.DMA_CH4_IRQHandler  vk035_it.o
    0x00000476   0x00000476   0x00000002   PAD
    0x00000478   0x00000478   0x00000002   Code   RO          306    .text.DMA_CH5_IRQHandler  vk035_it.o
    0x0000047a   0x0000047a   0x00000002   PAD
    0x0000047c   0x0000047c   0x00000002   Code   RO          308    .text.DMA_CH6_IRQHandler  vk035_it.o
    0x0000047e   0x0000047e   0x00000002   PAD
    0x00000480   0x00000480   0x00000002   Code   RO          310    .text.DMA_CH7_IRQHandler  vk035_it.o
    0x00000482   0x00000482   0x00000002   PAD
    0x00000484   0x00000484   0x00000002   Code   RO          312    .text.DMA_CH8_IRQHandler  vk035_it.o
    0x00000486   0x00000486   0x00000002   PAD
    0x00000488   0x00000488   0x00000002   Code   RO          314    .text.DMA_CH9_IRQHandler  vk035_it.o
    0x0000048a   0x0000048a   0x00000002   PAD
    0x0000048c   0x0000048c   0x00000002   Code   RO          340    .text.DebugMon_Handler  vk035_it.o
    0x0000048e   0x0000048e   0x00000002   PAD
    0x00000490   0x00000490   0x00000002   Code   RO          230    .text.ECAP0_IRQHandler  vk035_it.o
    0x00000492   0x00000492   0x00000002   PAD
    0x00000494   0x00000494   0x00000002   Code   RO          232    .text.ECAP1_IRQHandler  vk035_it.o
    0x00000496   0x00000496   0x00000002   PAD
    0x00000498   0x00000498   0x00000002   Code   RO          234    .text.ECAP2_IRQHandler  vk035_it.o
    0x0000049a   0x0000049a   0x00000002   PAD
    0x0000049c   0x0000049c   0x0000000e   Code   RO           12    .text.Error_Handler  main.o
    0x000004aa   0x000004aa   0x00000002   PAD
    0x000004ac   0x000004ac   0x00000018   Code   RO          525    .text.FPUInit       system_k1921vk035.o
    0x000004c4   0x000004c4   0x00000002   Code   RO          294    .text.FPU_IRQHandler  vk035_it.o
    0x000004c6   0x000004c6   0x00000002   PAD
    0x000004c8   0x000004c8   0x00000002   Code   RO          194    .text.GPIOA_IRQHandler  vk035_it.o
    0x000004ca   0x000004ca   0x00000002   PAD
    0x000004cc   0x000004cc   0x00000002   Code   RO          196    .text.GPIOB_IRQHandler  vk035_it.o
    0x000004ce   0x000004ce   0x00000002   PAD
    0x000004d0   0x000004d0   0x00000028   Code   RO          710    .text.GPIO_AltFuncCmd  plib035_gpio.o
    0x000004f8   0x000004f8   0x00000034   Code   RO          702    .text.GPIO_DeInit   plib035_gpio.o
    0x0000052c   0x0000052c   0x00000028   Code   RO          712    .text.GPIO_DigitalCmd  plib035_gpio.o
    0x00000554   0x00000554   0x0000001e   Code   RO          700    .text.GPIO_DriveModeConfig  plib035_gpio.o
    0x00000572   0x00000572   0x00000002   PAD
    0x00000574   0x00000574   0x0000001e   Code   RO          696    .text.GPIO_InModeConfig  plib035_gpio.o
    0x00000592   0x00000592   0x00000002   PAD
    0x00000594   0x00000594   0x00000060   Code   RO          706    .text.GPIO_Init     plib035_gpio.o
    0x000005f4   0x000005f4   0x0000005e   Code   RO          694    .text.GPIO_ModeConfig  plib035_gpio.o
    0x00000652   0x00000652   0x00000002   PAD
    0x00000654   0x00000654   0x00000028   Code   RO          708    .text.GPIO_OutCmd   plib035_gpio.o
    0x0000067c   0x0000067c   0x0000001e   Code   RO          692    .text.GPIO_OutModeConfig  plib035_gpio.o
    0x0000069a   0x0000069a   0x00000002   PAD
    0x0000069c   0x0000069c   0x0000001e   Code   RO          698    .text.GPIO_PullModeConfig  plib035_gpio.o
    0x000006ba   0x000006ba   0x00000002   PAD
    0x000006bc   0x000006bc   0x0000002e   Code   RO          714    .text.GPIO_StructInit  plib035_gpio.o
    0x000006ea   0x000006ea   0x00000002   PAD
    0x000006ec   0x000006ec   0x00000010   Code   RO           10    .text.GPIO_ToggleBits  main.o
    0x000006fc   0x000006fc   0x00000004   Code   RO          330    .text.HardFault_Handler  vk035_it.o
    0x00000700   0x00000700   0x00000002   Code   RO          228    .text.I2C_IRQHandler  vk035_it.o
    0x00000702   0x00000702   0x00000002   PAD
    0x00000704   0x00000704   0x00000002   Code   RO          192    .text.MFLASH_IRQHandler  vk035_it.o
    0x00000706   0x00000706   0x00000002   PAD
    0x00000708   0x00000708   0x00000020   Code   RO          994    .text.MFLASH_LatencyConfig  plib035_rcu.o
    0x00000728   0x00000728   0x00000004   Code   RO          332    .text.MemManage_Handler  vk035_it.o
    0x0000072c   0x0000072c   0x00000004   Code   RO          328    .text.NMI_Handler   vk035_it.o
    0x00000730   0x00000730   0x00000002   Code   RO          238    .text.PWM0_HD_IRQHandler  vk035_it.o
    0x00000732   0x00000732   0x00000002   PAD
    0x00000734   0x00000734   0x00000002   Code   RO          236    .text.PWM0_IRQHandler  vk035_it.o
    0x00000736   0x00000736   0x00000002   PAD
    0x00000738   0x00000738   0x00000002   Code   RO          240    .text.PWM0_TZ_IRQHandler  vk035_it.o
    0x0000073a   0x0000073a   0x00000002   PAD
    0x0000073c   0x0000073c   0x00000002   Code   RO          244    .text.PWM1_HD_IRQHandler  vk035_it.o
    0x0000073e   0x0000073e   0x00000002   PAD
    0x00000740   0x00000740   0x00000002   Code   RO          242    .text.PWM1_IRQHandler  vk035_it.o
    0x00000742   0x00000742   0x00000002   PAD
    0x00000744   0x00000744   0x00000002   Code   RO          246    .text.PWM1_TZ_IRQHandler  vk035_it.o
    0x00000746   0x00000746   0x00000002   PAD
    0x00000748   0x00000748   0x00000002   Code   RO          250    .text.PWM2_HD_IRQHandler  vk035_it.o
    0x0000074a   0x0000074a   0x00000002   PAD
    0x0000074c   0x0000074c   0x00000002   Code   RO          248    .text.PWM2_IRQHandler  vk035_it.o
    0x0000074e   0x0000074e   0x00000002   PAD
    0x00000750   0x00000750   0x00000002   Code   RO          252    .text.PWM2_TZ_IRQHandler  vk035_it.o
    0x00000752   0x00000752   0x00000002   PAD
    0x00000754   0x00000754   0x00000002   Code   RO          342    .text.PendSV_Handler  vk035_it.o
    0x00000756   0x00000756   0x00000002   PAD
    0x00000758   0x00000758   0x00000002   Code   RO          254    .text.QEP_IRQHandler  vk035_it.o
    0x0000075a   0x0000075a   0x00000002   PAD
    0x0000075c   0x0000075c   0x00000040   Code   RO           26    .text.RCU_AHBClkCmd  gpio.o
    0x0000079c   0x0000079c   0x00000040   Code   RO           28    .text.RCU_AHBRstCmd  gpio.o
    0x000007dc   0x000007dc   0x00000040   Code   RO          704    .text.RCU_AHBRstCmd  plib035_gpio.o
    0x0000081c   0x0000081c   0x00000040   Code   RO           43    .text.RCU_APBClkCmd  tmr.o
    0x0000085c   0x0000085c   0x00000040   Code   RO           45    .text.RCU_APBRstCmd  tmr.o
    0x0000089c   0x0000089c   0x00000010   Code   RO         1006    .text.RCU_BusyStatus  plib035_rcu.o
    0x000008ac   0x000008ac   0x00000030   Code   RO          165    .text.RCU_ClkOutCmd  sysclk.o
    0x000008dc   0x000008dc   0x0000003c   Code   RO          163    .text.RCU_ClkOutConfig  sysclk.o
    0x00000918   0x00000918   0x0000000a   Code   RO          960    .text.RCU_GetOSEClkFreq  plib035_rcu.o
    0x00000922   0x00000922   0x00000002   PAD
    0x00000924   0x00000924   0x0000000a   Code   RO          958    .text.RCU_GetOSIClkFreq  plib035_rcu.o
    0x0000092e   0x0000092e   0x00000002   PAD
    0x00000930   0x00000930   0x00000060   Code   RO          962    .text.RCU_GetPLLClkFreq  plib035_rcu.o
    0x00000990   0x00000990   0x00000024   Code   RO          964    .text.RCU_GetPLLDivClkFreq  plib035_rcu.o
    0x000009b4   0x000009b4   0x00000066   Code   RO          972    .text.RCU_GetUARTClkFreq  plib035_rcu.o
    0x00000a1a   0x00000a1a   0x00000002   PAD
    0x00000a1c   0x00000a1c   0x00000002   Code   RO          190    .text.RCU_IRQHandler  vk035_it.o
    0x00000a1e   0x00000a1e   0x00000002   PAD
    0x00000a20   0x00000a20   0x0000027e   Code   RO          988    .text.RCU_PLL_AutoConfig  plib035_rcu.o
    0x00000c9e   0x00000c9e   0x00000002   PAD
    0x00000ca0   0x00000ca0   0x000000a0   Code   RO          992    .text.RCU_PLL_Init  plib035_rcu.o
    0x00000d40   0x00000d40   0x00000010   Code   RO         1000    .text.RCU_PLL_LockStatus  plib035_rcu.o
    0x00000d50   0x00000d50   0x00000026   Code   RO          998    .text.RCU_PLL_OutCmd  plib035_rcu.o
    0x00000d76   0x00000d76   0x00000002   PAD
    0x00000d78   0x00000d78   0x00000022   Code   RO          990    .text.RCU_PLL_StructInit  plib035_rcu.o
    0x00000d9a   0x00000d9a   0x00000002   PAD
    0x00000d9c   0x00000d9c   0x0000005c   Code   RO          996    .text.RCU_SysClkChangeCmd  plib035_rcu.o
    0x00000df8   0x00000df8   0x0000001e   Code   RO         1004    .text.RCU_SysClkConfig  plib035_rcu.o
    0x00000e16   0x00000e16   0x00000002   PAD
    0x00000e18   0x00000e18   0x00000010   Code   RO          968    .text.RCU_SysClkStatus  plib035_rcu.o
    0x00000e28   0x00000e28   0x0000002a   Code   RO          103    .text.RCU_UARTClkCmd  uart.o
    0x00000e52   0x00000e52   0x00000002   PAD
    0x00000e54   0x00000e54   0x0000004c   Code   RO          101    .text.RCU_UARTClkConfig  uart.o
    0x00000ea0   0x00000ea0   0x00000032   Code   RO         1057    .text.RCU_UARTRstCmd  plib035_uart.o
    0x00000ed2   0x00000ed2   0x00000002   PAD
    0x00000ed4   0x00000ed4   0x00000002   Code   RO          222    .text.SPI_RO_RT_IRQHandler  vk035_it.o
    0x00000ed6   0x00000ed6   0x00000002   PAD
    0x00000ed8   0x00000ed8   0x00000002   Code   RO          224    .text.SPI_RX_IRQHandler  vk035_it.o
    0x00000eda   0x00000eda   0x00000002   PAD
    0x00000edc   0x00000edc   0x00000002   Code   RO          226    .text.SPI_TX_IRQHandler  vk035_it.o
    0x00000ede   0x00000ede   0x00000002   PAD
    0x00000ee0   0x00000ee0   0x00000002   Code   RO          338    .text.SVC_Handler   vk035_it.o
    0x00000ee2   0x00000ee2   0x00000002   PAD
    0x00000ee4   0x00000ee4   0x00000054   Code   RO          167    .text.SysTick_Config  sysclk.o
    0x00000f38   0x00000f38   0x00000008   Code   RO          344    .text.SysTick_Handler  vk035_it.o
    0x00000f40   0x00000f40   0x000000de   Code   RO          521    .text.SystemCoreClockUpdate  system_k1921vk035.o
    0x0000101e   0x0000101e   0x00000002   PAD
    0x00001020   0x00001020   0x0000000c   Code   RO          527    .text.SystemInit    system_k1921vk035.o
    0x0000102c   0x0000102c   0x00000010   Code   RO          198    .text.TMR0_IRQHandler  vk035_it.o
    0x0000103c   0x0000103c   0x00000010   Code   RO          200    .text.TMR1_IRQHandler  vk035_it.o
    0x0000104c   0x0000104c   0x00000010   Code   RO          202    .text.TMR2_IRQHandler  vk035_it.o
    0x0000105c   0x0000105c   0x00000010   Code   RO          204    .text.TMR3_IRQHandler  vk035_it.o
    0x0000106c   0x0000106c   0x0000001a   Code   RO           79    .text.TMR_ADCSOCCmd  tmr.o
    0x00001086   0x00001086   0x00000002   PAD
    0x00001088   0x00001088   0x0000001a   Code   RO           57    .text.TMR_Cmd       tmr.o
    0x000010a2   0x000010a2   0x00000002   PAD
    0x000010a4   0x000010a4   0x0000001a   Code   RO           77    .text.TMR_DMAReqCmd  tmr.o
    0x000010be   0x000010be   0x00000002   PAD
    0x000010c0   0x000010c0   0x0000001e   Code   RO           81    .text.TMR_ExtInputConfig  tmr.o
    0x000010de   0x000010de   0x00000002   PAD
    0x000010e0   0x000010e0   0x0000001c   Code   RO         1042    .text.TMR_FreqConfig  plib035_tmr.o
    0x000010fc   0x000010fc   0x00000022   Code   RO           75    .text.TMR_ITCmd     tmr.o
    0x0000111e   0x0000111e   0x00000002   PAD
    0x00001120   0x00001120   0x00000010   Code   RO           69    .text.TMR_ITStatus  tmr.o
    0x00001130   0x00001130   0x0000000e   Code   RO           71    .text.TMR_ITStatusClear  tmr.o
    0x0000113e   0x0000113e   0x00000002   PAD
    0x00001140   0x00001140   0x000000b0   Code   RO           51    .text.TMR_Init      tmr.o
    0x000011f0   0x000011f0   0x00000028   Code   RO         1038    .text.TMR_PeriodConfig  plib035_tmr.o
    0x00001218   0x00001218   0x00000010   Code   RO           73    .text.TMR_SetLoad   tmr.o
    0x00001228   0x00001228   0x00000010   Code   RO         1040    .text.TMR_SetLoad   plib035_tmr.o
    0x00001238   0x00001238   0x00000010   Code   RO          212    .text.UART0_E_RT_IRQHandler  vk035_it.o
    0x00001248   0x00001248   0x00000010   Code   RO          208    .text.UART0_RX_IRQHandler  vk035_it.o
    0x00001258   0x00001258   0x00000010   Code   RO          206    .text.UART0_TD_IRQHandler  vk035_it.o
    0x00001268   0x00001268   0x00000010   Code   RO          210    .text.UART0_TX_IRQHandler  vk035_it.o
    0x00001278   0x00001278   0x00000010   Code   RO          220    .text.UART1_E_RT_IRQHandler  vk035_it.o
    0x00001288   0x00001288   0x00000010   Code   RO          216    .text.UART1_RX_IRQHandler  vk035_it.o
    0x00001298   0x00001298   0x00000010   Code   RO          214    .text.UART1_TD_IRQHandler  vk035_it.o
    0x000012a8   0x000012a8   0x00000010   Code   RO          218    .text.UART1_TX_IRQHandler  vk035_it.o
    0x000012b8   0x000012b8   0x00000090   Code   RO         1051    .text.UART_AutoBaudConfig  plib035_uart.o
    0x00001348   0x00001348   0x00000018   Code   RO         1053    .text.UART_BaudDivConfig  plib035_uart.o
    0x00001360   0x00001360   0x0000001a   Code   RO          115    .text.UART_Cmd      uart.o
    0x0000137a   0x0000137a   0x00000002   PAD
    0x0000137c   0x0000137c   0x00000022   Code   RO         1061    .text.UART_DataWidthConfig  plib035_uart.o
    0x0000139e   0x0000139e   0x00000002   PAD
    0x000013a0   0x000013a0   0x0000003e   Code   RO         1055    .text.UART_DeInit   plib035_uart.o
    0x000013de   0x000013de   0x00000002   PAD
    0x000013e0   0x000013e0   0x00000010   Code   RO          131    .text.UART_ErrorStatusClear  uart.o
    0x000013f0   0x000013f0   0x00000022   Code   RO         1067    .text.UART_FIFOCmd  plib035_uart.o
    0x00001412   0x00001412   0x00000002   PAD
    0x00001414   0x00001414   0x00000018   Code   RO          145    .text.UART_FlagStatus  uart.o
    0x0000142c   0x0000142c   0x00000036   Code   RO          125    .text.UART_ITCmd    uart.o
    0x00001462   0x00001462   0x00000002   PAD
    0x00001464   0x00001464   0x00000022   Code   RO          111    .text.UART_ITFIFOLevelRxConfig  uart.o
    0x00001486   0x00001486   0x00000002   PAD
    0x00001488   0x00001488   0x0000001a   Code   RO          113    .text.UART_ITFIFOLevelTxConfig  uart.o
    0x000014a2   0x000014a2   0x00000002   PAD
    0x000014a4   0x000014a4   0x00000010   Code   RO          133    .text.UART_ITStatusClear  uart.o
    0x000014b4   0x000014b4   0x00000052   Code   RO         1059    .text.UART_Init     plib035_uart.o
    0x00001506   0x00001506   0x00000002   PAD
    0x00001508   0x00001508   0x0000001e   Code   RO         1065    .text.UART_ParityBitConfig  plib035_uart.o
    0x00001526   0x00001526   0x00000002   PAD
    0x00001528   0x00001528   0x0000000e   Code   RO          147    .text.UART_RecieveData  uart.o
    0x00001536   0x00001536   0x00000002   PAD
    0x00001538   0x00001538   0x00000022   Code   RO         1071    .text.UART_RxCmd    plib035_uart.o
    0x0000155a   0x0000155a   0x00000002   PAD
    0x0000155c   0x0000155c   0x00000010   Code   RO          149    .text.UART_SendData  uart.o
    0x0000156c   0x0000156c   0x00000022   Code   RO         1063    .text.UART_StopBitConfig  plib035_uart.o
    0x0000158e   0x0000158e   0x00000002   PAD
    0x00001590   0x00001590   0x00000022   Code   RO         1069    .text.UART_TxCmd    plib035_uart.o
    0x000015b2   0x000015b2   0x00000002   PAD
    0x000015b4   0x000015b4   0x00000004   Code   RO          336    .text.UsageFault_Handler  vk035_it.o
    0x000015b8   0x000015b8   0x00000002   Code   RO          188    .text.WDT_IRQHandler  vk035_it.o
    0x000015ba   0x000015ba   0x00000002   PAD
    0x000015bc   0x000015bc   0x00000030   Code   RO           49    .text.__NVIC_EnableIRQ  tmr.o
    0x000015ec   0x000015ec   0x00000030   Code   RO          105    .text.__NVIC_EnableIRQ  uart.o
    0x0000161c   0x0000161c   0x00000042   Code   RO          177    .text.__NVIC_SetPriority  sysclk.o
    0x0000165e   0x0000165e   0x00000002   PAD
    0x00001660   0x00001660   0x000000a6   Code   RO          135    .text.__uart_fifo_receive  uart.o
    0x00001706   0x00001706   0x00000002   PAD
    0x00001708   0x00001708   0x000000c8   Code   RO          119    .text.__uart_fifo_transmit  uart.o
    0x000017d0   0x000017d0   0x00000048   Code   RO          974    .text.getPeriphClkFreq  plib035_rcu.o
    0x00001818   0x00001818   0x00000088   Code   RO           30    .text.gpio_get_init  gpio.o
    0x000018a0   0x000018a0   0x000000ac   Code   RO           24    .text.gpio_init     gpio.o
    0x0000194c   0x0000194c   0x0000001e   Code   RO            6    .text.heartbit      main.o
    0x0000196a   0x0000196a   0x00000002   PAD
    0x0000196c   0x0000196c   0x0000008c   Code   RO            8    .text.main          main.o
    0x000019f8   0x000019f8   0x0000000c   Code   RO          169    .text.millis        sysclk.o
    0x00001a04   0x00001a04   0x00000010   Code   RO          171    .text.millis_inc    sysclk.o
    0x00001a14   0x00001a14   0x00000072   Code   RO            2    .text.periph_init   main.o
    0x00001a86   0x00001a86   0x00000002   PAD
    0x00001a88   0x00001a88   0x0000002e   Code   RO            4    .text.restart_receive  main.o
    0x00001ab6   0x00001ab6   0x00000002   PAD
    0x00001ab8   0x00001ab8   0x00000054   Code   RO          161    .text.sysclk_init   sysclk.o
    0x00001b0c   0x00001b0c   0x00000096   Code   RO           61    .text.tmr_delay     tmr.o
    0x00001ba2   0x00001ba2   0x00000002   PAD
    0x00001ba4   0x00001ba4   0x0000008c   Code   RO           65    .text.tmr_delay_done  tmr.o
    0x00001c30   0x00001c30   0x00000036   Code   RO           63    .text.tmr_delay_start  tmr.o
    0x00001c66   0x00001c66   0x00000002   PAD
    0x00001c68   0x00001c68   0x00000048   Code   RO           67    .text.tmr_handler   tmr.o
    0x00001cb0   0x00001cb0   0x00000050   Code   RO           47    .text.tmr_init      tmr.o
    0x00001d00   0x00001d00   0x000000de   Code   RO           41    .text.tmr_init_first  tmr.o
    0x00001dde   0x00001dde   0x00000002   PAD
    0x00001de0   0x00001de0   0x00000038   Code   RO           53    .text.tmr_set_callback  tmr.o
    0x00001e18   0x00001e18   0x00000030   Code   RO           55    .text.tmr_start     tmr.o
    0x00001e48   0x00001e48   0x000000a6   Code   RO           99    .text.uart1_gpio_init  uart.o
    0x00001eee   0x00001eee   0x00000002   PAD
    0x00001ef0   0x00001ef0   0x00000112   Code   RO          129    .text.uart_handler  uart.o
    0x00002002   0x00002002   0x00000002   PAD
    0x00002004   0x00002004   0x00000050   Code   RO          107    .text.uart_init     uart.o
    0x00002054   0x00002054   0x00000060   Code   RO           97    .text.uart_init_first  uart.o
    0x000020b4   0x000020b4   0x00000070   Code   RO          127    .text.uart_receive_it  uart.o
    0x00002124   0x00002124   0x00000078   Code   RO          137    .text.uart_set_callback  uart.o
    0x0000219c   0x0000219c   0x00000072   Code   RO          109    .text.uart_start    uart.o
    0x0000220e   0x0000220e   0x00000002   PAD
    0x00002210   0x00002210   0x00000092   Code   RO          117    .text.uart_transmit  uart.o
    0x000022a2   0x000022a2   0x00000002   PAD
    0x000022a4   0x000022a4   0x00000078   Code   RO          123    .text.uart_transmit_it  uart.o
    0x0000231c   0x0000231c   0x0000001a   Code   RO         1268    x$fpl$fpinit        fz_wm.l(fpinit.o)
    0x00002336   0x00002336   0x0000000f   Data   RO           15    .rodata.str1.1      main.o
    0x00002345   0x00002345   0x00000003   PAD
    0x00002348   0x00002348   0x00000020   Data   RO         1329    Region$$Table       anon$$obj.o


    Execution Region ER_RW (Exec base: 0x20000000, Load base: 0x00002368, Size: 0x000001f4, Max: 0xffffffff, ABSOLUTE, COMPRESSED[0x00000044])

    Exec Addr    Load Addr    Size         Type   Attr      Idx    E Section Name        Object

    0x20000000   COMPRESSED   0x00000001   Data   RW          179    .data.SYSCLK_Oscil_Type  sysclk.o
    0x20000001   COMPRESSED   0x00000003   PAD
    0x20000004   COMPRESSED   0x000000c0   Data   RW           32    .data.gpioa_config  gpio.o
    0x200000c4   COMPRESSED   0x000000c0   Data   RW           33    .data.gpiob_config  gpio.o
    0x20000184   COMPRESSED   0x0000001c   Data   RW           84    .data.tmr0_config   tmr.o
    0x200001a0   COMPRESSED   0x0000001c   Data   RW           86    .data.tmr1_config   tmr.o
    0x200001bc   COMPRESSED   0x0000001c   Data   RW           88    .data.tmr2_config   tmr.o
    0x200001d8   COMPRESSED   0x0000001c   Data   RW          152    .data.uart1_config  uart.o


    Execution Region ER_ZI (Exec base: 0x200001f8, Load base: 0x000023ac, Size: 0x000006d8, Max: 0xffffffff, ABSOLUTE)

    Exec Addr    Load Addr    Size         Type   Attr      Idx    E Section Name        Object

    0x200001f8        -       0x00000060   Zero   RW         1180    .bss                c_w.l(libspace.o)
    0x20000258        -       0x00000004   Zero   RW          529    .bss.SystemCoreClock  system_k1921vk035.o
    0x2000025c        -       0x00000008   Zero   RW           83    .bss.htmr0          tmr.o
    0x20000264        -       0x00000008   Zero   RW           85    .bss.htmr1          tmr.o
    0x2000026c        -       0x00000008   Zero   RW           87    .bss.htmr2          tmr.o
    0x20000274        -       0x00000008   Zero   RW           89    .bss.htmr3          tmr.o
    0x2000027c        -       0x00000020   Zero   RW          153    .bss.huart0         uart.o
    0x2000029c        -       0x00000020   Zero   RW          151    .bss.huart1         uart.o
    0x200002bc        -       0x0000000a   Zero   RW           14    .bss.rxbuff         main.o
    0x200002c6   0x000023ac   0x00000002   PAD
    0x200002c8        -       0x00000004   Zero   RW          180    .bss.uwTick         sysclk.o
    0x200002cc   0x000023ac   0x00000004   PAD
    0x200002d0        -       0x00000200   Zero   RW          537    HEAP                startup_k1921vk035.o
    0x200004d0        -       0x00000400   Zero   RW          536    STACK               startup_k1921vk035.o


==============================================================================

Image component sizes


      Code (inc. data)   RO Data    RW Data    ZI Data      Debug   Object Name

       436          0          0        384          0      21301   gpio.o
       360          0         15          0         10      16182   main.o
       592          0          0          0          0      22487   plib035_gpio.o
      1398          4          0          0          0      12580   plib035_rcu.o
        84          0          0          0          0       1926   plib035_tmr.o
       562          4          0          0          0      10575   plib035_uart.o
        64         26        344          0       1536        916   startup_k1921vk035.o
       370          0          0          1          4      10534   sysclk.o
       522          0          0          0          4       8515   system_k1921vk035.o
      1362          4          0         84         32      12698   tmr.o
      1986          4          0         28         64      32187   uart.o
       342          0          0          0          0       6665   vk035_it.o

    ----------------------------------------------------------------------
      8296         42        394        500       1656     156566   Object Totals
         0          0         32          0          0          0   (incl. Generated)
       218          0          3          3          6          0   (incl. Padding)

    ----------------------------------------------------------------------

      Code (inc. data)   RO Data    RW Data    ZI Data      Debug   Library Member Name

        90          0          0          0          0          0   __dczerorl2.o
         8          0          0          0          0         68   __main.o
         0          0          0          0          0          0   __rtentry.o
        12          0          0          0          0          0   __rtentry2.o
         6          0          0          0          0          0   __rtentry4.o
        52          8          0          0          0          0   __scatter.o
        28          0          0          0          0          0   __scatter_zi.o
        18          0          0          0          0         80   exit.o
         6          0          0          0          0        152   heapauxi.o
         0          0          0          0          0          0   indicate_semi.o
         2          0          0          0          0          0   libinit.o
         6          0          0          0          0          0   libinit2.o
         2          0          0          0          0          0   libshutdown.o
         2          0          0          0          0          0   libshutdown2.o
         8          4          0          0         96         68   libspace.o
         2          0          0          0          0          0   rtexit.o
        10          0          0          0          0          0   rtexit2.o
        12          4          0          0          0         68   sys_exit.o
        74          0          0          0          0         80   sys_stackheap_outer.o
         2          0          0          0          0         68   use_no_semi.o
        26          0          0          0          0        116   fpinit.o

    ----------------------------------------------------------------------
       374         16          0          0         96        700   Library Totals
         8          0          0          0          0          0   (incl. Padding)

    ----------------------------------------------------------------------

      Code (inc. data)   RO Data    RW Data    ZI Data      Debug   Library Name

       340         16          0          0         96        584   c_w.l
        26          0          0          0          0        116   fz_wm.l

    ----------------------------------------------------------------------
       374         16          0          0         96        700   Library Totals

    ----------------------------------------------------------------------

==============================================================================


      Code (inc. data)   RO Data    RW Data    ZI Data      Debug   

      8670         58        394        500       1752     156910   Grand Totals
      8670         58        394         68       1752     156910   ELF Image Totals (compressed)
      8670         58        394         68          0          0   ROM Totals

==============================================================================

    Total RO  Size (Code + RO Data)                 9064 (   8.85kB)
    Total RW  Size (RW Data + ZI Data)              2252 (   2.20kB)
    Total ROM Size (Code + RO Data + RW Data)       9132 (   8.92kB)

==============================================================================

